:020000040000FA
:040000006FD00400B9
:101000006F00507B000000000000000090200020D6
:10101000AA220020A9BDF9F56C23002000000000E1
:10102000000000006C230020902000200000000041
:101030000000000090200020000000009020002010
:101040000000000090200020902000209020002030
:101050009020002090200020242F00205E240020DB
:101060000000000090200020902000200424002098
:1010700090200020D22300209020002090200020EB
:101080009020002090200020902000209020002020
:101090009020002001A04111B7170040985F3AC688
:1010A000945F3247E39CE6FE3245410182800111A4
:1010B00013078008F337078093F787083EC20100C3
:1010C0000100B7170040930570052380B70413068D
:1010D00080FA2380C7040100010083C6B70493F699
:1010E000F60DA385D704238007049246F3A6068055
:1010F0000100010093760502D5CEF336078093F602
:10110000860836C4010001002380B7042380C70489
:1011100001000100B70614007D89558D88C70100C4
:1011200001000100010023800704A246F3A6068007
:101130000100010073370780137787083AC6010062
:1011400001002380B7042380C704010001000100CF
:1011500001003727004093061005A303D7802380A2
:101160000704B247F3A70780010001009307800836
:10117000F3B7078093F787083ECE01000100B71749
:101180000040130770052380E704130780FA2380CB
:10119000E7040100010003C7B70413670708A3852C
:1011A000E70423800704F247F3A70780010001004A
:1011B0000561828093760504BDC6F336078093F6F9
:1011C000860836C8010001002380B7042380C704C5
:1011D00001000100B7061400938606047D89558D31
:1011E00088C7010001000100010023800704C246F6
:1011F000F3A6068001000100733707801377870884
:101200003ACA010001002380B7042380C70401000B
:1012100001003727004093062005A303D7802380D1
:101220000704D24781B773370780137787083ACC12
:10123000010001002380B7042380C70401000100DE
:1012400098471367070C98C723800704E24719BF24
:101250000111814601468145114506CE97000000E7
:10126000E780005593078008F3B7078093F7870856
:101270003EC601000100B717004013077005238028
:10128000E704130780FA2380E7040100010003C785
:101290006704136717002383E70423800704B2471A
:1012A000F3A7078001000100F2400561828041112F
:1012B000814601468145114597000000E780404F77
:1012C00013078008F337078093F787083EC40100AF
:1012D0000100B7170040130670052380C70493066A
:1012E00080FA2380D70401000100FD552396B70240
:1012F00023800704A245F3A5058001000100733790
:101300000780137787083AC6010001002380C704CD
:101310002380D7040100010003C767041367170087
:101320002383E70423800704B247F3A70780010063
:10133000010001A0BD473305F50201007D1575FDD3
:101340008280411122C426C206C6AA8401446317C2
:101350009400B24022449244410182800504130566
:10136000803E420497000000E78000FD4180C5B741
:101370009305000273A04580824573901534924016
:101380002242B2424243D2436244F2440255925551
:101390002256B2564257D2576258F25806499649D9
:1013A000264AB64A464BD64B664CF64C065D965DD1
:1013B000265EB65E465FD65F09617300203041113C
:1013C000B7170040985F3AC6945F3247E39CE6FE49
:1013D000324541018280B71700401307000323887C
:1013E000E702854717170000232EF74273002030CD
:1013F000411122C406C637040020976000E0E78050
:1014000020CC1C408297D5BF373700408347470028
:101410009146BD8B6389D70099466394D700834773
:101420005740730020309736000083C6662C9387A0
:10143000160017360000230DF62A0347870097375A
:1014400000009387E71AB6972380E700B7E7040008
:10145000BC4F0946894517150000034565F482977E
:10146000C9B7B787004003C76700098B6309071036
:1014700003C777009306000313770703630DD708AC
:10148000173800000348586217360000130606613B
:101490000547B30606012380E60083C577001737AA
:1014A000000013072760429793F5F50F2300B7005C
:1014B00003C58700973500009385855EC295137537
:1014C000F50F2380A5000347070089451377F7032D
:1014D000630CB70C63E7E50A6306071A8545630CDE
:1014E000B7129737000083C7375C3307F60003470E
:1014F00007001377F70F19CB850793F7F70F0D4701
:101500006363F71A17370000A300F75AB787004044
:1015100009472383E700B787004083C77700E207C6
:10152000E18763DE07049737000083C7F757173753
:1015300000001307A7563E9785462300D7001737AC
:101540000000130727563E97930600032300D70099
:10155000173700001307C7543E97A146850723009D
:10156000D70093F7F70F0D476364F71417370000A0
:10157000A30CF752B787004009472383E7007300A5
:101580002030930610026300D70E930620026305F5
:10159000D70693060002E316D7F403C72702137792
:1015A000C70F13672700D5A803C767001377070481
:1015B00065CB03C7A702173800001308A82F1735FB
:1015C00000001305E526134707082385E70203C734
:1015D000A7021377370F136787002385E702814738
:1015E00013070004B305F5008C41B306F80091071A
:1015F0008CC2E399E7FEF5B503C7A70213470704BA
:101600002385E70203C7A7021377C70F13672700D5
:101610002385E702F9B503C767001377070449C3B9
:1016200003C76702173800001308881C173500002D
:101630001305C513134707082383E70203C767028F
:101640001377370F136787002383E7028147130758
:101650000004B305F5008C41B306F80091078CC275
:10166000E399E7FEBDBD03C7670213470704238361
:10167000E70203C767021377C70F136727002383A7
:10168000E70285B503C767001377070411CB03C7CB
:1016900027021377370F136787002381E70291B57D
:1016A000238006003DBD97370000A38F073EB9BDDC
:1016B00097370000A38A073E75BD230304801547B2
:1016C0002303E48001002302A480828083076480D6
:1016D000E3CE07FE23030480828083076480E3CE89
:1016E00007FE03454480828083076480E3CE07FEC3
:1016F0002302A4808280411126C44AC24EC006C67D
:101700001377F50BAD47AA892E899544630CF70032
:10171000194597000000E78080FA97000000E780F5
:1017200020FB8D444E8597000000E78040F9FD596D
:10173000FD1463983401B240A24412498249410128
:101740008280135509011375F50F97000000E7809B
:10175000E0F92209F1BF011126CC06CEB70408003A
:1017600097000000E780C0F6154597000000E7806D
:1017700000F597000000E78080F697000000E78002
:1017800000F62AC697000000E78080F43245937780
:10179000150089EB136515001375F50FF240E2444F
:1017A00005618280FD14E9F00145CDBF397126DC69
:1017B0004ADA4ED852D656D45AD25ED006DE62CE1F
:1017C00066CCB7E700E07D5783AA070022C603AACC
:1017D000470023A0E71823A2E718B7170040130714
:1017E00070052380E704130780FA2380E70483C78A
:1017F0004704930B75FFB684E20793FBFB0F854606
:10180000AA892E8B328937240040E187015763FA79
:1018100076016308D5008946130700026313D500DB
:101820000157D98F93F7F70FB71C00402382FC04B0
:1018300011472303E4801305F00F97000000E780B1
:1018400000E8094C97000000E78080E863657C159C
:10185000B7050700DA9537870700795563FEE50479
:10186000B3879500636AF704370B0800A94733EB89
:1018700065016395F90881E8814497000000E780DD
:1018800020E5268515A8DA85094597000000E78040
:10189000C0E605090345F9FFFD14050B970000009C
:1018A000E780C0E481C49377FB0FE5F79700000061
:1018B000E780A0EA69F17D55B7170040130770056E
:1018C0002380E704130780FA2380E70403C7470453
:1018D000418B2382E704F250B7E700E023A05711C1
:1018E00023A24711E25432445259C259325AA25AE1
:1018F000125B825B724CE24C21618280A547639B44
:10190000F90685691309F00FB3069900B3742B012A
:10191000B6941349F9FFB3749900856B3379690163
:10192000416B9387F9FFB3F7270199E363FC340117
:1019300093D94900C147E3E637FF3DBF0569C16957
:101940007D19D9B71305800D63886901130500025D
:101950006384790113051008CA8597000000E780A9
:10196000C0D997000000E78040DF31D54E99B3849D
:1019700034416DBFDA852D4597000000E780E0D740
:10198000CA94E30B99EE050997000000E78020D583
:10199000A30FA9FEFDB79387F9FF93F7F70F636DC8
:1019A000FC0C83C71C04130730086315F7063707C0
:1019B00008006361EB06B3079B00B706100063FBEA
:1019C000D704334BEB0089476399F9068980D549E1
:1019D000E38404EADA85094597000000E780E0D156
:1019E00011090327C9FF91472320E480030764807E
:1019F000E34E07FE23033481FD17EDFBFD14110BAD
:101A000081C49377FB0FE9FF97000000E780E0D4E3
:101A100061F155B5B717004003C75704B707080071
:101A20001377070219E3B78707007955E376FBE8D8
:101A300033079B00E3F9E7F841B58547E380F9F008
:101A4000DA852D4597000000E78020CB9389F4FFCD
:101A5000E38404E297000000E78060C893F7390050
:101A600091EB832604800327090093074900E3963E
:101A7000E6E03E89CE84D9BFB5476399F9001305E6
:101A8000900B97000000E78080C3FDB3B1471305BA
:101A9000B00AE388F9FE99476397F904B70508008F
:101AA000B365BB002D4597000000E78000C5814469
:101AB0008D4BA14997000000E78060C263967401D6
:101AC000832704802320F9008504E39534FF8327CE
:101AD000048013172B01635507002312F90069BB1B
:101AE0002322F90051BB9D47639FF90281451305ED
:101AF000B00497000000E78040C0BD4423200900E7
:101B000023220900FD5997000000E78040BD93F7AC
:101B10007400CA9703C70700FD14398D2380A700FE
:101B2000E39334FF91BBA1476397F9069700000048
:101B3000E780A0C28144630D0B008D479304C0036E
:101B40006308FB009304000563048B0193044004C5
:101B50001375C507E30295D2194597000000E78089
:101B600000B697000000E780A0B60545970000008A
:101B7000E780E0B4268597000000E78020B709459C
:101B800097000000E78080B697000000E780E0BC87
:101B9000E31405CE0DB39147639FF900130560066A
:101BA00097000000E780A0B197000000E78040B2F6
:101BB00013059009F9B5E38109CCF1547DB9BD66EF
:101BC0000147173600001306660B938606A6854567
:101BD0008347060093F7F70F91C382800507E3F967
:101BE000E6FE97370000238BB708DDB77D16620647
:101BF000618693178601E18763D4070001458280DF
:101C0000931726003307F500AE9718439C4363E70C
:101C1000E7007D16E37FF7FC7D55828005458280D5
:101C2000FD15E205E18513978501618793F7F50FAF
:101C300063480700FD15139725002A97584365D779
:101C4000138517006205618582803308B5021C4246
:101C500083A80600B335B502C29733B50701AE9825
:101C6000469585486367B5006394A50063E3070163
:101C700081480C43C6950CC388C21CC28280814730
:101C80001397870161876343B7008280139727000A
:101C90002A97232007008507E5B7814701479396D8
:101CA0008701E18663C5B6001335170082809396DD
:101CB0002700AA9694428507558FD5B793D75540EC
:101CC0008A07AA979C4305453315B5007D8D828010
:101CD00017F3FFDFE702A33D2A8497000000E780A7
:101CE00060F405C5931725003E940327C4FF814780
:101CF00011EB7D1516053E954205418517F3FFDF73
:101D00006700233D05838507E5B70145C5BF8147CA
:101D10001397870161876343C70082801397270069
:101D2000B386E50094422A97850714C3D5B77D167C
:101D300062066186014793178601E18763D5070034
:101D400013351700828093172600B306F500AE976F
:101D500094429C437D16B58F5D8FF1BF8A05AA958D
:101D600001476363B500828083A6C5FFF11593D751
:101D70001600D98F9CC11397F601E5B72A83014855
:101D8000014701456343D7008280B387050183A8DB
:101D90000700B30706019C43C697AA976384F8001F
:101DA00033B517010507B3080301620723A0F80044
:101DB00061871108C1BF2A8301478147014563C379
:101DC000D70082803388E50083280800330EE600C0
:101DD000032E0E003388A8403308C84163840801ED
:101DE00033B508018507B308E300E20723A0080123
:101DF000E1871107E9B717F3FFDFE702432B011172
:101E0000B286B2842E86AA850A8597000000E780F4
:101E1000C0FA2A84A6850A8597000000E78020E89A
:101E200033348000060413351500018D056117F366
:101E3000FFDF6700032A17F3FFDFE702C324411126
:101E4000AA89AE8A328BB68402C202C402C6014499
:101E5000131C8401135C8C4163499C02939B140006
:101E6000FD1B0549138CF4FFF15C33048901620406
:101E700061846340740792478E04CE9423AEF4FECF
:101E8000410117F3FFDF6700832313192400B30B0D
:101E90002B01014A93172A00D69783A50B0088438C
:101EA00078003400500097000000E78040DA050A0F
:101EB00093178A01E187F11BE35EFCFC92474E9980
:101EC00005042320F900A2473EC2B24702C63EC421
:101ED00041B7131A8901135A8A41131D240093171D
:101EE0008A01E18763CF970092470A044E941CC091
:101EF000A24705091379F90F3EC2B24702C63EC494
:101F0000ADB7B3079A0313152A0056950841780018
:101F100034005000050AEA97DA978C4397000000D6
:101F2000E780E0D26DBF0000197106C212C416C668
:101F30001AC81ECA22CC26CE2AD02ED232D436D6E9
:101F40003AD83EDA42DC46DECAC0CEC2D2C4D6C6D9
:101F5000DAC8DECAE2CCE6CEEAD0EED2F2D4F6D6C9
:101F6000FAD8FEDA971500009385458B8841E70083
:101F7000050092402242B2424243D2436244F244BC
:101F8000025592552256B2564257D2576258F258CD
:101F900006499649264AB64A464BD64B664CF64CFD
:101FA000065D965D265EB65E465FD65F096173008C
:101FB00020300000972100209381C1041751002098
:101FC0001301418417F5FFFF130505049705002051
:101FD00093854503171600201306C6FD63FAC50056
:101FE0008322050023A0550011059105E3EAC5FEF3
:101FF00017050200130545CC97150020938585FB36
:10200000171600201306066563FAC5008322050033
:1020100023A0550011059105E3EAC5FE1715002020
:102020001305456397450020938545116377B500F7
:10203000232005001105E36DB5FEFD42739002BC3F
:102040008D4273904280B722000093828288739001
:102050000230970200209382E2FA93E232007390FA
:102060005230975200009382A281739012346FB065
:10207000347973002030397101436EC619A039716B
:1020800041536AC866CA62CC5ECE19A03971015349
:102090005AD056D252D44ED64AD826DA22DC06DEA0
:1020A00033016140828241114AC026C222C406C661
:1020B0008282B24D4101024D924C224CB24B410101
:1020C000024B924A224AB2494101024992442244B7
:1020D000B240410182803D432A876373C3029377F4
:1020E000F700BDEFADE5937606FF3D8ABA960CC3C7
:1020F0004CC30CC74CC74107E36BD7FE11E282808B
:10210000B306C3408A069702000096966780A60031
:102110002307B700A306B7002306B700A305B7003F
:102120002305B700A304B7002304B700A303B70037
:102130002303B700A302B7002302B700A301B7002F
:102140002301B700A300B7002300B700828093F5F6
:10215000F50F93968500D58D93960501D58D61B7C2
:10216000939627009702000096968682E78086FA6B
:102170009680C1171D8F3E96E374C3F8A5B73367E9
:10218000B500FD530D8B79E7B7877F7F9387F7F70E
:1021900010419441B372F6003363F600BE92B3E28D
:1021A00062006397720C6318D6065041D441B37233
:1021B000F6003363F600BE92B3E262006398720ADF
:1021C000631BD60410459445B372F6003363F600E2
:1021D000BE92B3E262006391720A631ED60250455A
:1021E000D445B372F6003363F600BE92B3E26200E8
:1021F000639A72086311D60210499449B372F600CB
:102200003363F600BE92B3E2620063937208510535
:10221000D105E30FD6F61317060193970601631C49
:10222000F7001357060193D706013305F74093755E
:10223000F50F91E982804183C1833305F74093759F
:10224000F50F91E182801377F70F93F7F70F3305BE
:10225000F74082800346050083C605000505850515
:102260006313D60065FA3305D640828011059105C7
:10227000E312D6FE014582802105A105E31CD6FCB0
:10228000014582803105B105E316D6FC0145828007
:102290004105C105E310D6FC01458280B717004017
:1022A00003C777051377E70FA38BE704130700F83D
:1022B000A38DE7043D47238CE70413075003A38C49
:1022C000E70403C7A7051377D70F238DE7048280A0
:1022D000B717004003C7E7020D8941111377C70FF5
:1022E000498F93068008F3B6068093F6860836C6B3
:1022F00001000100930670052380D704930680FA3D
:102300002380D704010001002387E702238007040C
:10231000B247F3A70780010001004101828041110B
:102320002A83014E930E407E130F0019930F40062F
:1023300063E56E129308001913034006B378150382
:10234000854E0D4FA14F337365020D89133515006E
:1023500063EFBE121308F6FF7946729842081358CD
:1023600008013307C70213D61700BE07329761462C
:10237000B3F6C60213068070B386C6023697A1660E
:10238000F58F42075D8FB716004083C7F60293F7BB
:102390000708A303F1000346710083C7F60293F711
:1023A0000708E394C7FE83477100B716004093F710
:1023B000F70F6388071293078008F3B7078093F736
:1023C00087083EC401000100B7170040930670055E
:1023D0002380D704930680FA2380D70401000100EC
:1023E00023AA070383C6170393E60608A388D70228
:1023F00023800704A247F3A70780010001001166AC
:10240000B71700407D16D45BC85F93854703A98E3C
:10241000F18EF5FA93068008F3B6068093F68608E7
:1024200036C601000100930670052380D704930689
:1024300080FA2380D7040100010098C103C7170365
:1024400013670704A388E70223800704B247F3A7B2
:10245000078001000100410182807D133368E3039E
:102460009308E016630E08003368F3039308D01650
:10247000630808009378330093B818009388D8163F
:1024800033081E01131E0801135E0E0155B5639338
:10249000E5030548638608000148630303002A88B2
:1024A00071087298FD15131E0801C205135E0E0116
:1024B000C18179BD13F8150063F4BF007908D5B761
:1024C00013381800E5BF83C7F60293F70708A30384
:1024D000F1000346710083C7F60293F70708E394FF
:1024E000C7FE8347710093F7F70FF1DFE9B531714C
:1024F0004AD966CB06DF22DD26DB4ED752D556D32E
:102500005AD15ECF62CD6AC96EC7AA8C02D8971025
:102510000000E780009F2A8993078008F3B70780AF
:1025200093F787083EDA01000100B7170040130750
:1025300070052380E704130780FA2380E704010075
:10254000010003C7F7021377770FA387E70203C7DA
:10255000F70213678700A387E70223800704D25797
:10256000F3A7078001000100054597000000E78000
:1025700060D6130780C13347E902116A93070AE85E
:1025800093065002BD69930BA004814A014B1304CA
:102590008008930470057D1AB347F9023307D70208
:1025A0003EC0FD873ECC938709A69309803E334702
:1025B000F7023AC27D873AC4334739038549B39954
:1025C000990193D93940B306D702B30B7703B3C649
:1025D000F602B3CBFB0236C6FD8636C893D6FB4166
:1025E00036CEB7460F00938606243349D902856656
:1025F000938606FAB3969601B389E90213076055EC
:102600003309D90293060010B389E9023349D9028C
:10261000B3C9F9029316390036CA37190040FD864E
:1026200036D0930D090493D7F9413ED2F336048096
:1026300093F6860836DC01000100930770052380BD
:10264000FD00930680FA2380DD000100010083462F
:10265000390593F6860FA309D9048346390593E615
:102660001600A309D90423800D00E256F3A60680C4
:1026700001000100130C80FA116DF336048093F60B
:10268000860836DE01000100930770052380FD00F7
:1026900023808D010100010083463905216693E600
:1026A0000602A309D90483560905B3E6A601231837
:1026B000D90483560905D18E2318D90423800D002F
:1026C000F256F3A60680010001008346390593F611
:1026D00006026381061A03463905218A6DDE081851
:1026E00097100000E780E085733604801376860833
:1026F000B2C20100010023809D0023808D010100F2
:102700000100B717004003C637051376F60DA389FD
:10271000C70403C6370513660602A389C704835698
:1027200009052166B3E6A6012318D90483560905D5
:10273000D18E2318D90423800D009646F3A6068077
:10274000010001008346390593F60602638B0614E7
:1027500083463905A18AEDFE97000020E780A0930B
:10276000AA8636D497000020E780E092A256E30ABA
:10277000D5FE835609054255B3E6A6012318D904B0
:1027800097000000E780A07D83463905A18AEDDE31
:10279000035609058346290582473376CA00B306E6
:1027A000DA0293D5F641B296B388F640E24733B8E1
:1027B000C6002E983308F840A247B3B61601330876
:1027C000D84063C70701631DF800924763FA1701F9
:1027D000C247634FF80E63950701B24763EAF80EEC
:1027E000894663E9660FF2469315180013D3F80182
:1027F0005E8613951800B365B30042D646D497B0F1
:102800000100E780006A3258050B137BFB0F63471A
:102810000001631A0838A2586387083813081500A6
:10282000B336A800B69513D6F5013298B336C80072
:10283000AE9613581800FE06B3E606017336048000
:1028400013768608B2C60100010023809D00238014
:102850008D01010001000356C902B296C206C18271
:102860002316D90223800D00B646F3A60680010088
:10287000010021B5F336048093F68608B6C0010046
:10288000010023809D0023808D010100010083460B
:10289000390593E60602A309D90423800D00864674
:1028A0000DB5F336048093F68608B6C40100010026
:1028B00023809D0023808D0101000100834639059E
:1028C00093E60602A309D90423800D00A646BDB5F0
:1028D000E30B0BF0F336048093F68608B6C80100CC
:1028E0000100930680FA23809D002380DD00010013
:1028F00001008346390593F5FC0F93F6860FA30973
:10290000D90483463905CD8EA309D90423800D004F
:10291000C646F3A6068001000100130580FA0346AF
:102920003905930639051D8A631C96297336048080
:1029300013768608B2CC01000100130680FA2380CA
:102940009D002380CD000100010003C60600137620
:10295000F60D2380C60003C6060013660602238018
:10296000C600835609051166D18E2318D9048356F3
:1029700009052166D18E2318D90423800D00E6466F
:10298000F3A6068001000100130680FA834639058C
:1029900093F606026380062683463905130C390533
:1029A000A18AFDDA081897000000E7808059F33605
:1029B000048093F68608B6D001000100930680FAE1
:1029C00023809D002380DD000100010083460C0070
:1029D000116693F6F60D2300DC0083460C0093E6A7
:1029E00006022300DC0083560905D18E2318D90482
:1029F000835609052166D18E2318D90423800D0042
:102A00008656F3A6068001000100130680FA83466D
:102A1000390593F60602638A062083463905A18AA2
:102A2000EDFE97F0FF1FE78000672A8C97F0FF1FED
:102A3000E7806066E30C85FF835609051166425501
:102A4000D18E2318D90497000000E78040518346B7
:102A5000390513063905A18AFDDAF336048093F6A9
:102A60008608B6D401000100930680FA23809D00F9
:102A70002380DD00010001008346060093F6F60D79
:102A80002300D60023800D00A656F3A60680010081
:102A900001008356090503462905D247B376DA00BB
:102AA0003306CA021305800C9355F6413696330D52
:102AB000F6408257333CD6002E9C3336A601330CA9
:102AC000FC40330CCC403308850392564E86B33518
:102AD000A5033305A503C29597B00100E780603CCC
:102AE00063468001631E0C16630C0D161306150059
:102AF0003335A6002E959356F5013696B335D6009C
:102B0000AA959396F50105828585D18E6346B0001E
:102B1000639D051A638B061A0356C9021582330595
:102B2000D6003336C500B2956348B00063910524E2
:102B30001306F00F637DA622894663F356159307AB
:102B40008008F3B7078093F78708BED6010001001D
:102B500037170040930770052300F704930780FAA6
:102B60002300F704010001008356C702896781171B
:102B7000D58FC207C1832316F70223000704B65777
:102B8000F3A7078001000100FA506A54DA544A5949
:102B9000BA592A5A9A5A0A5BFA4B6A4CDA4C4A4D8D
:102BA000BA4D296182801308F5FF3335A800FD1561
:102BB0002E951356F5013298B336C800AA9695B9EA
:102BC000F336048093F68608B6CA0100010023801C
:102BD0009D002380AD000100010083463905CD8EA4
:102BE000A309D90423800D00D646F3A60680010070
:102BF000010035B3F336048093F68608B6CE0100A3
:102C0000010023809D002380CD0001000100834648
:102C1000390593E60602A309D90423800D00F64680
:102C2000F3A606800100010095B3F336048093F605
:102C30008608B6D20100010023809D002380CD00CC
:102C4000010001008346390593E60602A309D90471
:102C500023800D009656F3A606800100010045BBB7
:102C60009306F5FF33B5A600FD152E959355F50196
:102C7000AE96B3B5B600AA951396F501858269B5EF
:102C8000F336048093F68608B6D801000100930657
:102C900080FA23809D002380DD000100010083561F
:102CA000C9020566011693F6F60FD18EC206C182DF
:102CB0002316D90223800D00C656F3A60680010014
:102CC0000100850A93FAFA0F95B233E6B60045C2C1
:102CD0000356C9023305D0403338A000B305B040D5
:102CE000B385054115826345B000D1E16371A60843
:102CF000894663F0560593078008F3B7078093F77A
:102D00008708BEDA01000100B717004013077005FD
:102D10002380E704130780FA2380E7040100010001
:102D200003D7C7027D8B2396E70223800704D6577B
:102D300081BDF336048093F68608B6DC01000100FD
:102D4000930680FA23809D002380DD0001000100AE
:102D50008356C9020566011693F6F60FD18EC20698
:102D6000C1822316D90223800D00E656B9B7930716
:102D70008008F3B7078093F78708BEDE01000100E3
:102D800037170040930770052300F704930780FA74
:102D90002300F704010001000356C7029397560071
:102DA000B297C207C1832316F70223000704F65720
:102DB000C1BB914763EEB70217D70100130707FAAB
:102DC0008A05BA959C41BA978287B717004003A736
:102DD000470B1345F5FF698F23AAE70A03A7070BE3
:102DE000698F23A8E70A03A7070A798D23A0A70AFA
:102DF0008280B717004083A6470B1347F5FFF98E73
:102E000023AAD70A83A6070B558D23A8A70A83A652
:102E1000070A758F23A0E70A8280B717004003A72F
:102E2000470B498F23AAE70A03A7070B1345F5FFB2
:102E300045BFB717004083A6470B1347F5FF758FB3
:102E400023AAE70A03A7070A598D4DB7B717004011
:102E500003A7470B498FEDB7914763EEB70217D72A
:102E600001001307E7F08A05BA959C41BA9782875B
:102E7000B717004003A7470D1345F5FF698F23AA35
:102E8000E70C03A7070D698F23A8E70C03A7070C1E
:102E9000798D23A0A70C8280B717004083A6470D29
:102EA0001347F5FFF98E23AAD70C83A6070D558D7E
:102EB00023A8A70C83A6070C758F23A0E70C82809C
:102EC000B717004003A7470D498F23AAE70C03A7B4
:102ED000070D1345F5FF45BFB717004083A6470D03
:102EE0001347F5FF758F23AAE70C03A7070C598D2D
:102EF0004DB7B717004003A7470D498FEDB7B71778
:102F000000408847420541819377050491EB937710
:102F1000F5013755E801130505803345F502828038
:102F20009377050C130700046397E7009377F50187
:102F300037459C1CCDB72165130505D0828037E746
:102F400000E01C435443A183E206D58F1CC1FD570A
:102F50002320F7182322F718828013178500B7E77C
:102F600000E023A0E710618123A2A7108280B7F7B9
:102F700000E08847CC478280814737370040A14630
:102F800063C4C700328582800345B740E38EA6FE46
:102F90003385F5000345050085072304A740CDB719
:102FA00097070020938707019C43173700201307DA
:102FB000E7183E95636EE500173700201307876416
:102FC0006368A700170700202326A7FE3E8582809E
:102FD000FD57EDBF8280411122C406C62A849700A6
:102FE0000000E78000F22947B307E502B2408D8375
:102FF000B3D7870222449507B3D7E702373700409B
:10300000C207C1832316F700410182807165411117
:103010001305052006C697000000E78000FCB737BF
:103020000040130770F82381E7000D47A381E700F4
:1030300013070004A380E70005472387E700B24099
:103040004101828037370040834727001A0593F7F4
:10305000F703C98F93F7F70F2301F7008280B73783
:10306000004003C7170019C9D98DA380B70003C753
:103070000700136787002380E700828093C5F5FF70
:10308000F98DA380B7008280AE872A87B7360040CB
:1030900021463738004089E7170300006700C3F373
:1030A00083C8B600E30916FF05078348F7FFFD173D
:1030B000C20723041801C183F9BF411122C406C607
:1030C0002A8497000000E780C0E32947B307E502A0
:1030D000B2408D83B3D7870222449507B3D7E70266
:1030E00037370040C207C1832316F7404101828071
:1030F000716541111305052006C697000000E780A1
:1031000000FCB7370040130770F82381E7400D47F4
:10311000A381E74013070004A380E7400547238706
:10312000E740B24041018280CC41411106C6328560
:1031300003C6150083C5050022064D8E42068D6527
:103140004186138875A2630C0611634BC80413886B
:1031500045A26300060D634AC800938535A263014A
:10316000B6082390060029464DA0138855A2630592
:10317000060D938565A2E316B6FE8D451D4663E6F2
:10318000E5081146198E63F3C7003E86B7E70400D1
:103190002390C600FC4797D501009385A5BF9DA04D
:1031A000138895A263030611634E060D1388A5A22A
:1031B00063000613938505A5E315B6FA99451D46E8
:1031C00063E5E504198E63F3C7003E86B7E70400A4
:1031D0002390C600FC47970500209385E5E71DA0D6
:1031E0009D451D4663E3E5022146198E63F3C70042
:1031F0003E86B7E70400FC472390C60097050020F1
:103200009385C545BA9582970146B2403285410102
:103210008280AD451D46E3EAE5FE3146198E63F333
:10322000C7003E86B7E704002390C600FC4797D549
:1032300001009385A5B8F9B7B1451D46E3E7E5FC64
:103240003546198E63F3C7003E86B7E70400239026
:10325000C600FC4797D50100938545B765B78D45F6
:103260001D46E3E4E5FA1146198E63F3C7003E8676
:10327000B7E704002390C600FC4797D5010093856B
:1032800025B249B78D451D46E3E1E5F81146198E93
:1032900063F3C7003E86B7E704002390C600FC47EF
:1032A00097D50100938545B4B1BFA5451D46E3EE12
:1032B000E5F42946198E63F3C7003E86B7E704009C
:1032C0002390C600FC4797D50100938525AE1DBF0E
:1032D000B5451D46E3EBE5F23946198E63F3C700A9
:1032E0003E86B7E704002390C600FC4797D501004F
:1032F000938545A901BFB7E7040003A30713970609
:103300000020938666D44146A54517050020130585
:10331000A5CA02832D455DE703C505000947631F64
:10332000E50803A84500411106C603471800328589
:103330000346080022074168518F930828FE63075F
:10334000170563E9E80005186303070323900600E7
:10335000294591A8130648FE630AC7041518E31708
:1033600007FF15463E87637BF600154701A8130645
:1033700000023E876374F60013070002B7E70400FB
:103380002390E600FC471316070111A83E8691C35F
:103390000546B7E70400FC472390C6004206CC452B
:1033A000418282970145B2404101828013060008A4
:1033B0003E87E375F6FC13070008C9B723900600A3
:1033C000054582808280416779176304E5044111D5
:1033D00022C406C685472A84639FF500B7E7040028
:1033E00022852244B24003A38713970500209385CA
:1033F00025414101028389476399F500B7E704003D
:1034000083A7070B8545829771D9B24022444101B9
:1034100082808280797122D452CC2E842A8A97D5D8
:1034200001009385659E17D50100130565A006D69A
:103430003AC626D24AD0B68432894ECE97B0010021
:10344000E78060F1A68517D501001305659F97B049
:103450000100E78040F0294597B00100E78080F443
:103460008347840093F70702E1E783490400894713
:10347000054532476396F908544083C7160083C652
:103480000600A207D58FC166138616FE638CC7029D
:103490008D16638FD7068D66938626902945639196
:1034A000D706B7E70400A285225403A34714B250FD
:1034B000F249A6864A86925402595285624A854745
:1034C000456102832D450DEF93070002354563E901
:1034D0009702B7E70400FC47484413060002CA8578
:1034E0008297814997070020938747329C43014583
:1034F00081CB9C4391C74E852686CA85829701451C
:10350000B250225492540259F249624A4561828073
:103510002D457DF79307700F3545E3E397FEB7E739
:103520000400FC4748441306700FCA8582975DBFAC
:103530002145F9B7411122C437E4040083278413DD
:1035400026C2AA84416506C6970500209385452BAF
:103550007D1582978327C40A170500001305E5E649
:103560008588829795C0032304132244B240924475
:10357000970600209386C6BF4146C5451705002023
:10358000130505AE41010283B24022449244014535
:103590004101828019C59707002023A9A72601456C
:1035A0008280454582801147636AA70A97D6010049
:1035B000938646840A0536951841411106C636970A
:1035C000AE87B2850287130700026145639DE7005D
:1035D000B7E70400FC471306000217050020130597
:1035E000650882970145B2404101828005476145E7
:1035F000E39BE7FEB7E70400FC47054617050020FC
:1036000013054508F9BF1307700F6145E39DE7FCFB
:10361000B7E70400FC471306700F170500201305D9
:10362000A506C1B7130700086145E39EE7FAB7E7AF
:103630000400FC4713060008170500201305451475
:103640004DB715476145E390E7FAB7E70400FC473B
:103650001546170500201305E51A61B70945828054
:10366000411126C2B7E4040083A7C41322C44AC090
:1036700006C62E8497050020938585182A8982978F
:10368000058905C5970700209387879D83D7A70BDA
:10369000A28503A3440D2310F4002244B2409244B7
:1036A0004A850249014641010283B24022449244C4
:1036B000024949454101828097070020238A071467
:1036C0009707002023A80714B717004003A7070C8B
:1036D000B706C0FFFD16758F23A0E70C03A7070DE3
:1036E000B7064000558F23A8E70C03A7070C3D9BA6
:1036F00023A0E70C03A7070D1367070123A8E70C16
:103700008280B717004003A5470C83A7470C598157
:1037100013451500C18B058999E3136525009707AB
:10372000002083C7E70E6380A7029707002023814C
:10373000A70E11C9970700209387C70D03A30700A1
:103740006303030002838280114517F3FFFF6700C4
:1037500043DA411193962500AA852D4506C697F0B8
:10376000FF1FE780A004B2400145410182800111A2
:1037700022CC06CE3714004026CA4AC84EC652C4D0
:1037800083447405034AB4058349840503499405B9
:1037900097F0FFFFE780C0B08347A40593F4F40FD0
:1037A000137AFA0F93E71700230DF40493F9F90F36
:1037B0001379F90FB717004003C7A705058B6DFFF5
:1037C00003D5C705A38D4705238C3705A38C270593
:1037D000A38B9704F2406244D2444249B249224A40
:1037E0000561828041119397050122C406C626C255
:1037F000C1872E8463DC0700B7E40400FC54829781
:1038000019C1BC5482972165218D15A893F7150025
:1038100013C515008DE793F725009DC7970000009D
:10382000E78060EEB7E70400BC4F1306000A894545
:1038300017050020034585FE829713452400B240FA
:1038400022449244410182809397250163D8070264
:10385000B7E4040083A7C41E829797000000E780A6
:10386000E0EEBC4C37F60200130606E0896517054A
:1038700000200345A5FA8297096579B7939715014A
:103880000145E3DE07FA17C501001305656397B02C
:103890000100E78020C4B7E70400BC4F13060064B2
:1038A000916517050020034565F782971165A9BF4B
:1038B0002D71232A9110FD74E98C232C811023286B
:1038C0002111232631112A84AE89328993060010F2
:1038D0000A86A6852D45232E111097F0FF1FE7803D
:1038E000E0EC13154401B7E70400FC4751810A05D9
:1038F00013962900CA850A958297A6858566014692
:10390000254597F0FF1FE78060EA0A86A6859306A3
:103910000010294597F0FF1FE78040E98320C1117F
:103920000324811183244111032901118329C1102A
:1039300015618280B7F7070003C70701411106C66A
:1039400022C426C24AC0A547631DF70097000000A5
:10395000E78040F6B24022449244024901454101C9
:10396000828013942500AA843289A286AA85014602
:10397000254597F0FF1FE78060E3A2864A86A6856B
:10398000294597F0FF1FE78060E2E9B71D71A2CCDF
:1039900037E404005C5C485886CE494697C5010070
:1039A0009385854D829711E917C501001305054ED2
:1039B00097B00100E78000B201A0B7F600E07957A8
:1039C00098CAFD57DCCA0567B7E700E023A0E710F7
:1039D0001306F00290C223A0E71801000100370788
:1039E000002018471306000481459706002023A5F0
:1039F000E6E24157A38AE7403C44080882979707CC
:103A000000209387677E3EC8856713870740231A87
:103A1000E1001D673ACC37070105130707103ACEBE
:103A20009387B7D31307B00F2310E1022312F102DB
:103A3000054797F7FFFF9387C7532301E1023ED85D
:103A400017070000130727D197070000938767D255
:103A5000B7F50700BAC23EDC170700001307C7ED31
:103A600097070000938787CE81463000E10519450E
:103A7000BAC43EDE97F0FF1FE78040D318088147A5
:103A8000994630003E960346060085070507A30BBE
:103A9000C700E398D7FEC24791C703574101856726
:103AA0006373F70001A0B7E7040083A7470A08087B
:103AB0008297AA8511C917C501001305653E97B005
:103AC0000100E780408901A0F640664425618280BC
:103AD000411126C2B7E4040083A7040806C622C425
:103AE00017050000130545D0829717040020130422
:103AF000E4D22300A40097000000E7808002970032
:103B00000000E780A0BB03450400224403A3840512
:103B1000B2409244130600328965410102837971F3
:103B200006D622D413078008F337078093F7870857
:103B30003EC201000100B7170040930570052380C5
:103B4000B704130680FA2380C7040100010083C66E
:103B5000F70293F6A60FA387D702238007049246A5
:103B6000F3A60680010001007337078013778708EA
:103B70003AC4010001002380B7042380C704010078
:103B8000010003C7F70213672700A387E70223801A
:103B90000704A247F3A7078001000100054597E04D
:103BA000FFFFE780207397000000E78020BA0147FD
:103BB00081468147054685451305407E97E0FFFF16
:103BC000E780207637E404003C4468005146814594
:103BD0008297B707C0A83EC8B787E803938707D086
:103BE0003ECA97E7FF1F9387877D3EC67C586800D3
:103BF0008297B250225445618280411197D50100CD
:103C00009385459217C501001305852206C697A026
:103C10000100E780407417D50100130565A997A03E
:103C20000100E7804073B2402945410117A301001C
:103C300067004377411197D501009385E58F17C53C
:103C400001001305E51E06C697A00100E780A070DD
:103C500017D50100130585A497A00100E780A06F88
:103C6000B2402945410117A301006700A373411128
:103C700022C406C6834705002A849DC797D5010044
:103C80009385459117C501001305851A97A001007A
:103C9000E780606C4C4017D501001305A5B597A0CF
:103CA0000100E780406B3DA058410DEF97D5010022
:103CB0009385458E17C501001305851797A0010050
:103CC000E780606917D50100130545B497A001008E
:103CD000E78060682244B2402945410117A30100F2
:103CE0006700436CA1679386D7036313D70297D508
:103CF00001009385258A17C501001305651397A058
:103D00000100E780406517D50100130525B17DBF8F
:103D1000ED0797D501009385E58717C501001305C9
:103D20002511631BF70097A00100E780C06217D53B
:103D300001001305E5AF59BF97A00100E780A0611E
:103D40004C4017D501001305A5B091BF411197C58F
:103D500001009385A57F17C501001305650D06C6F3
:103D600097A00100E780205FB2402945410117A3D9
:103D7000010067002363797122D426D24AD02E84B1
:103D80002A898145B2844800714606D697E0FFFF34
:103D9000E780A03497F7FF1F9387475EDC4783D700
:103DA0000700231421012313F10097400000E7804E
:103DB000A07C9547A305F1009307401F3EC6FD5721
:103DC0002305A100230AF10097500000E780008F2F
:103DD0002686A285480097400000E780C07CB2504C
:103DE00022549254025945618280972700202390E3
:103DF0000790971700202389077EB7E70400BC4788
:103E0000411106C641468145170500201305452C82
:103E1000829797200000E780E05D97200000E78010
:103E20002039014597500000E780C01B170700208C
:103E30000347072C9307F00A6315F7029307F0F87E
:103E40008945170500201305A52A1707002023011F
:103E5000F72A97070020A38D072897500000E780D6
:103E6000604897500000E780405A814537050400BC
:103E70009707002023AC07249707002023960724E8
:103E80009707002023830724970700202394071C0B
:103E9000970700202392071A9707002023950722EF
:103EA00097070020239E072297300000E780A0C0DC
:103EB000014597500000E780E04B97C501009385CE
:103EC000656B17C501001305A5F697A00100E780F3
:103ED000804817D501001305E59D97A00100E780F4
:103EE0008047B2402945410117A301006700834B79
:103EF000411122C406C626C293F715002E84638F93
:103F00000710814617F6FF1F1306864485451705DF
:103F100000200355251297C00000E78080B515C921
:103F200097C501009385C56517C50100130545F0C8
:103F300097A00100E780204217C50100130505077F
:103F400097A00100E7802041294597A00100E78064
:103F5000604597C501009385A56217C5010013054B
:103F600025ED97A00100E780003F17C5010013056C
:103F7000250597A00100E780003E294597A0010094
:103F8000E780404217F5FF1F1305453F5C45054795
:103F90002390E70097300100E780006697C5010095
:103FA0009385055E17C50100130585E897A00100FC
:103FB000E780603A17C501001305C50197A001000D
:103FC000E7806039294597A00100E780A03D93076D
:103FD00010F817070020230DF7109707002083D74C
:103FE000270517070020A305F71017050020130564
:103FF0002510A183914517070020230CF70E970782
:104000000020A388070E97500000E780A02D1345DD
:104010001400B240224492444101828093F725006B
:10402000E1C3170700200357270A45CB9706002056
:104030009386C609944297D701009387A7891706EC
:104040000020034686088145170500201305450812
:1040500097700000E78040C1AA8441C197C5010064
:104060009385C55817C50100130585DC97A001008D
:10407000E780602EA68517C50100130525F797A0D8
:104080000100E780402D294597A00100E78080319D
:1040900097070020239A0702930710F817070020BC
:1040A0002308F7049707002083D787F81707002015
:1040B000A300F704A18317070020230CF702914502
:1040C0008D47170500201305A50217070020A3023E
:1040D000F70297500000E780E0201345240015BF49
:1040E00093F74500D1C397C501009385255017C5A7
:1040F00001001305E5D397A00100E780C02517C58F
:104100000100130565F097A00100E780C024294550
:1041100097A00100E7800029930720F817070020E7
:104120002308F7FC9707002083D7C7F21707002062
:10413000A300F7FCA18317070020230CF7FA85479B
:1041400017070020A307F7FA97400000E780005701
:10415000170500201305C5F9914597500000E78029
:1041600060181345440075B593F78500A9C797C536
:1041700001009385A54717C50100130565CB97A0DE
:104180000100E780401D17C50100130525E997A030
:104190000100E780401C294597A00100E7808020AE
:1041A00097070020239207F297700000E780A0BBDA
:1041B00013458400B9BD93F70501D1C385451705A3
:1041C0000020035525E997500100E780C06D97C591
:1041D00001009385A54117C50100130565C597A08A
:1041E0000100E780401717C50100130565E497A09B
:1041F0000100E7804016294597A00100E780801A5A
:10420000930730F8170700202304F7EE97070020E4
:1042100083D747E417070020A30CF7EC170500200D
:10422000130505EDA1838D45170700202303F7EC47
:1042300097500000E780000B13450401D9BB93F7AA
:104240000502D1C797C501009385453A17C50100FE
:10425000130505BE97A00100E780E00F17C5010018
:10426000130545DF97A00100E780E00E294597A0E0
:104270000100E7802013930740F817070020230967
:10428000F7E69707002083D727DB17070020A30155
:10429000F7E6A18317070020230DF7E485471707EA
:1042A0000020A308F7E497070020239707D897403A
:1042B0000000E780A04017050020130565E3914545
:1042C00097500000E78000021345040299B393F76A
:1042D0000504FDC397C501009385453117C501004D
:1042E000130505B597A00100E780E00617C501009A
:1042F0001305C5D797A00100E780E005294597A0E1
:104300000100E780200A9707002083C767DE1307B4
:10431000700A6386E7061307800A638CE7081307B1
:10432000600A6393E704930760F8170700202301EE
:10433000F7DC9707002083D707D917070020A309C8
:10434000F7DAA183170700202305F7DA8547170757
:104350000020A304F7DAB14517050020130545D95D
:1043600097500000E78000F897400000E780003594
:104370001345040497070020239707D459B99307DE
:1043800070F8170700202305F7D69707002083D77A
:1043900087D317070020A30DF7D4A18317070020A8
:1043A0002309F7D4854717070020A305F7D49945BB
:1043B00065B7930780F8F1B793F705080145E38ADD
:1043C00007C497C501009385652217C50100130531
:1043D00025A697A00100E78000F817C50100130586
:1043E00065CA97A00100E78000F7294597A0010062
:1043F000E78040FB9307A0F817070020230AF7CEB9
:104400009707002083D7C7CD17070020A302F7CE58
:10441000A18317070020230EF7CC8547170700203C
:10442000A309F7CC97070020239C07CA97400000F8
:10443000E780C02817050020130585CB91459750CC
:104440000000E78020EA13450408E1B6411122C4C8
:1044500097C50100938545152A8417C501001305EA
:10446000259D06C697A00100E780E0EE4C4017C5E9
:1044700001001305A53597A00100E780C0ED29458F
:1044800097A00100E78000F2034704009307F00FB4
:10449000631FF70297C501009385051117C5010039
:1044A0001305059997A00100E780E0EA4C4017C585
:1044B00001001305A53297A00100E780C0E922445E
:1044C000B2402945410117A301006700A3EDB240A6
:1044D000224441018280B1C1411122C417C50100AB
:1044E000130505952E8497C501009385E50606C63C
:1044F00097A00100E78020E6A28517C501001305FB
:10450000253997A00100E78000E52244B240294503
:10451000410117A301006700E3E88280411122C432
:1045200026C22E84AA8497C501009385A50317C5CA
:1045300001001305E58F06C697A00100E780A0E102
:1045400017C501001305853597A00100E780A0E09D
:10455000294597A00100E780E0E497C50100938515
:10456000650097070020239797AC17C50100130536
:10457000258C854497070020239C87AA9707002055
:10458000239997AA971700202393871697A00100D5
:10459000E78060DC9715002083D5651517C50100FD
:1045A0001305453097A00100E780E0DA294597A080
:1045B0000100E78020DF97170020238797029720CC
:1045C0000000E780E0BE228597500000E78080A1D0
:1045D000054597500000E780E0D997F7FF1F9387C4
:1045E000E7D9DC4703D70700C167FD176312F7025D
:1045F0002244B7E70400B240924403A3870517F5AD
:10460000FF1F034525221306000A85454101028349
:10461000B2402244924441018280011122CC37E40D
:1046200004005C5C06CE26CA354697C5010093851A
:10463000650917D501001305E5CD829711E917C566
:1046400001001305A58497A00100E780A0E801A060
:1046500097F7FF1F9387C71D3EC4B7F5070085670F
:1046600093870780814617F6FF1F1306E61BE105B7
:1046700019453EC697E0FF1FE78040137C4419466A
:1046800097F5FF1F9385451A170500201305C59C54
:104690008297340017F6FF1F1306061997C501000D
:1046A0009385455A17C501001305455B97600000C7
:1046B000E7808030AA8421C197C50100938505F267
:1046C00017B501001305C57697A00100E780A0C8C3
:1046D000A68517C501001305E5FF97A00100E78037
:1046E00080C7294597A00100E780C0CBF240624413
:1046F000D2440561828097E00000E780C09217C530
:104700000100130525F497500000E780A02497A02E
:104710000000E78000E797500100E780804B17F525
:10472000FF1F130525C297500100E780203417C5ED
:104730000100130525F297500100E780004CAA8480
:1047400097600000E780E08A97000100E78060231F
:1047500097800100E78080BC97700000E78020E32D
:1047600097600000E780E00097300100E780C0E438
:1047700097C50100938585E617B501001305456BC4
:1047800099C897A00100E78000BDA68517C5010064
:10479000130585F699B797A00100E780C0BB17C540
:1047A00001001305A5F797A00100E780C0BA2945CD
:1047B00097A00100E78000BF97300100E780A0C00C
:1047C00097F00000E78060DF630F0510854537052F
:1047D000040097200000E780002E97C50100938514
:1047E000E5DF17B501001305A56497A00100E78078
:1047F00080B617C501001305E5F397A00100E78017
:1048000080B5294597A00100E780C0B997F7FF1F41
:10481000938787A683D70700171700202319F7EC83
:104820008547171700202301F7DC97200000E78059
:10483000E0B697200000E780A097171500200355E9
:1048400005EB97400000E780E0799707002083C7D9
:104850007799ADEBA303010083274417130671007A
:10486000854513055030829797C50100938505D77C
:1048700017B501001305C55B97A00100E780A0AD47
:1048800017C50100130545ED97A00100E780A0AC16
:10489000294597A00100E780E0B097C50100938506
:1048A000E5D317B501001305A55897A00100E780CF
:1048B00080AA17C50100130525F097A00100E78025
:1048C00080A905B597C50100938545D117B50100AD
:1048D0001305055697A00100E780E0A717C5010062
:1048E000130505EB55B797C50100938525CF17B57F
:1048F00001001305E55397A00100E780C0A517C587
:104900000100130525FB97A00100E780C0A42945FD
:1049100097A00100E78000A9014597500000E780BB
:1049200060A5A5BF411122C437E404008327041AFF
:1049300006C6829797400000E780E073832704084B
:1049400017F5FFFF1305055B829797F7FF1F238B72
:10495000A7EC17F5FF1F130565A297400000E7803D
:1049600080082244B240410117030000670023CBB6
:10497000B7E70400FC471171A2DDCAD986DFA6DBC8
:10498000CED72E8432892E86AA8517F5FF1F1305F0
:104990002576829717F7FF1F130787758347070050
:1049A000930680029387E70793F7F70FE3ECF6107F
:1049B000BA898A0717B701001307C750BA979C43F3
:1049C000BA9782878D4797C50100938565C317B550
:1049D00001001305E545630FF40097A00100E7808F
:1049E000809717C501001305658097A00100E78037
:1049F0008096BDA497A00100E780E09517C501004F
:104A00001305458097A00100E780E094294597A011
:104A10000100E7802099930720F8114697F5FF1FC2
:104A20009385056D4A8517F7FF1F2303F76C97F7EA
:104A3000FF1FA380076C97F0FFFFE78000342A84F4
:104A40001DC997C501009385A5BB17B501001305C6
:104A5000253E97A00100E7800090A28517B50100D0
:104A60001305057E97A00100E780E08E294597A0F9
:104A70000100E780209397C50100938565B817B5BD
:104A800001001305E53A97A00100E780C08C17B537
:104A900001001305257C97A00100E780C08B294504
:104AA00097A00100E78000904165930730FA054622
:104AB00097F5FF1F9385C5637D1517F7FF1F230922
:104AC000F76297F0FFFFE780402B2A841DC997C546
:104AD00001009385E5B217B501001305653597A070
:104AE0000100E7804087A28517B5010013054575D1
:104AF00097A00100E7802086294597A00100E78064
:104B0000608AB7E70400BC4F0566130606C8A145D6
:104B100017F5FF1F034505D18297FE506E54DE54F2
:104B20004E59BE591161828091476303F40297C5C3
:104B300001009385E5AC17B501001305652F97A01B
:104B40000100E780408117B501001305E57371BDD1
:104B5000B7E70400FC4F914517F5FF1F034585CCCF
:104B6000829797C501009385A5A917B50100130584
:104B7000252C97900100E780007E17B501001305F2
:104B8000657297900100E780007D294597A001009C
:104B9000E780408197400000E78040B2914535A40E
:104BA00085476303F40297C50100938565A517B592
:104BB00001001305E52797900100E780C07917B53C
:104BC00001001305A56F15B597F7FF1F239427491B
:104BD000B7E704000566BC4F130606C8C1450DBF04
:104BE0008D476303F40297C50100938565A117B54E
:104BF00001001305E52397900100E780C07517B504
:104C000001001305656DD5B3930740F8114697F57C
:104C1000FF1F9385E54D4A8517F7FF1F230AF74CC1
:104C200097F7FF1FA387074C97F0FFFFE780E0147B
:104C30002A84E30405EE97C501009385659C17B5AA
:104C400001001305E51E97900100E780C070A28562
:104C500017B501001305C55E97900100E780A06FAE
:104C6000294597900100E780E07345BD9147E31C1B
:104C7000F4F6B7E70400FC4F9305000217F5FF1F99
:104C8000034545BA829797C501009385659717B587
:104C900001001305E51997900100E780C06B17B577
:104CA00001001305E564F1BD894763E3870297C5F9
:104CB00001009385E59417B50100130565179790DA
:104CC0000100E780406917B501001305A56331BBFA
:104CD00097F4FF1F83C4E44197F7FF1F83C7574131
:104CE00097C501009385C591A20417B5010013056E
:104CF0002514DD8C97900100E780E065A28517B54B
:104D000001001305656197900100E780C064C2044B
:104D1000294597900100E780E068C1849305D4FF9E
:104D200093960401C1824A8693F5F50F17F5FF1F8C
:104D30001305353C97200000E780A0DBE35F90DCA3
:104D4000930750F817F7FF1F2304F73A83C739007A
:104D5000228697F5FF1F9385A53985074A8517F7A2
:104D6000FF1FA308F73897F0FFFFE78000012A84B0
:104D7000E30505DA97C501009385858817B501001D
:104D80001305050B97900100E780E05CA28517C52D
:104D900001001305E5AEC9B5894763E3870297C5EE
:104DA00001009385E58517B5010013056508979007
:104DB0000100E780405A17B501001305A55735B12A
:104DC00097400000E780808FA28517F5FF1F13052D
:104DD000253297400000E780E05081B38D476303A0
:104DE000F40297C501009385A58117B5010013054D
:104DF000250497900100E780005617B501001305C0
:104E00002555E5B6B76602000146B77502000545AF
:104E100097E0FF1FE7808099930760F817F7FF1F5F
:104E20002308F72C97F7FF1FA385072C930700068D
:104E300017F7FF1F2300F72C894717F7FF1FA30B56
:104E4000F72A97F7FF1F2388072A97F7FF1FA384E6
:104E5000072AC14717F7FF1F2300F72A930720F9F6
:104E600017F7FF1FA30AF728314697F7FF1FA386FE
:104E7000A72897F5FF1F9385A5274A8597F7FF1F5A
:104E8000238D072697F0FFFFE78020EF2A84E306B3
:104E900005C897B501009385A57617B501001305E0
:104EA00025F997900100E780004BA28517B5010016
:104EB0001305854B55B3B1476303F40297B5010061
:104EC0009385057417B50100130585F697900100C9
:104ED000E780604817B501001305C54A39B6B7E742
:104EE0000400FC4F9305000417F5FF1F034585934D
:104EF000829797300000E780607CB145F9B5914713
:104F000063E3870297B501009385856F17B50100AC
:104F1000130505F297900100E780E04317B5010003
:104F200013050548D9B497F4FF1F83C4A41C97F751
:104F3000FF1F83C7171CA204DD8C8E04B777020005
:104F40006D14BE942286A68517B50100130585460B
:104F500097900100E7802040B7E70400FC472286D5
:104F600097F5FF1F93851519280082979316040162
:104F7000C1823000A685094597E0FF1FE7800083C6
:104F80002A8409C917B501001305854497900100CB
:104F9000E7804054930770F8194697F5FF1F9385F3
:104FA00025154A8517F7FF1F2304F71497F7FF1FEE
:104FB000A382871497F0FFFFE78020DC2A84E30EAA
:104FC00005B497B501009385A56317B501001305D6
:104FD00025E697900100E7800038A28517B501000B
:104FE0001305054095B99947630BF41297B5010075
:104FF0009385056117B50100130585E397900100BE
:10500000E780603517B501001305053FF9BA9147F0
:1050100063E3870297B501009385855E17B50100AC
:10502000130505E197900100E780E03217B5010014
:105030001305053E5DBA97F4FF1F83C4A40B97F7D1
:10504000FF1F83C7170BA204DD8C8E04B777020005
:105050006D14BE942286A68517B501001305853C04
:1050600097900100E780202FB7E70400FC472286D5
:1050700097F5FF1F93851508280082979316040162
:10508000C1823000A6850D4597D0FF1FE7800072D2
:105090002A8409C917B501001305853A97900100C4
:1050A000E7804043930780F8194697F5FF1F9385E3
:1050B00025044A8517F7FF1F230CF70297F7FF1FF8
:1050C000A38A870297F0FFFFE78020CB2A84E306BC
:1050D00005A497B501009385A55217B501001305E6
:1050E00025D597900100E7800027A28517B501001C
:1050F0001305453695B699476303F40297B5010049
:105100009385055017B50100130585D297900100CE
:10511000E780602417B5010013054535F9B0B7E7FE
:105120000400FC4F9305000417E5FF1F0345856F3E
:10513000829797300000E7806058994579B18D4794
:105140006303F40297B501009385854B17B5010001
:10515000130505CE97900100E780E01F17B5010009
:105160001305453259B017B501001305A5329790C4
:105170000100E78020361305C01297D0FF1FE7809B
:10518000401C014597E0FFFFE780A0DB0D4597102D
:105190000000E780009F294597D0FF1FE780601A35
:1051A00097D0FF1FE780C00A8DBA99476303F402C6
:1051B00097B501009385C54417B50100130545C790
:1051C00097900100E780201917B501001305452DC0
:1051D00029B817F7FF1F0347F7F197F7FF1F83C79A
:1051E00067F122075D8F9166BA96C2061166C18289
:1051F0001306F6EF8D476365D60297E7FF1F938787
:10520000E7179C4B17F6FF1F0346B6EE9386C700C1
:105210002DC203D6070069CA8907E39CD7FE8947D8
:105220001307A0F8114697F5FF1F938565EC4A8593
:1052300097F6FF1F238EE6EA17F7FF1FA30BF7EA87
:1052400097F0FFFFE78060B32A84E308058C97B5E9
:1052500001009385E53A17B50100130565BD9790E8
:105260000100E780400FA28517B5010013058524D2
:10527000E5B203D60700630EE60A8907E39BF6FE54
:105280008D4779BF91476304F40297B50100938578
:10529000253717B501001305A5B997900100E780E0
:1052A000800B17B50100130565226FF00FF4B7E707
:1052B0000400FC4F9305000817E5FF1F03458556C2
:1052C0008297C9B897B501009385853317B501005A
:1052D000130505B697900100E780E00717B50100B8
:1052E000130545206FF06FF02390E70017E5FF1FCF
:1052F0001305C50897200100E780603297B50100CB
:105300009385053017B50100130585B2979001000C
:10531000E780600417B501001305C51D97900100D3
:10532000E7806003294597900100E780A007814747
:10533000C5BD2390070017E5FF1F1305250497201F
:105340000100E780C02D97B501009385652B17B547
:1053500001001305E5AD97900100E780C0FF17B588
:1053600001001305A51A5DBF411122C406C683477B
:1053700005002A849DC797B501009385252417B59C
:1053800001001305E5AA97900100E780C0FC4C409E
:1053900017B501001305055597900100E780A0FBA4
:1053A000E1A05841B707CF009387777D631DF706CB
:1053B00097B501009385852017B50100130545A712
:1053C00097900100E78020F91C448356E400835540
:1053D000C40003C6070017B50100130525529790B6
:1053E0000100E78040F7294597900100E78080FBA6
:1053F0000357E4009707002083D7672F6309F7005E
:105400008355C400084497E0FFFFE78020C8035697
:10541000E4008355C40008442244B240410117F31C
:10542000FFFF67002355B707CC009387777D63158F
:10543000F70497B501009385651817B501001305AA
:10544000259F97900100E78000F11C448356E400FB
:105450008355C40003C6070017B501001305054AAC
:1054600097900100E78020EF2244B2402945410196
:1054700017930100670003F3B707CE009387777D8A
:105480006304F70297B501009385451317B5010032
:105490001305059A97900100E780E0EB4C4017B5A3
:1054A00001001305E53ACDBDB2402244410182809E
:1054B000B7E70400FC4741112E8606C622C426C267
:1054C0004AC02E842A89AA8517F5FF1F130545C2F5
:1054D000829797B501009385651417B501001305F0
:1054E000259597900100E78000E797F5FF1F83C59A
:1054F00025C017B50100130565BA97900100E78034
:1055000080E5294597900100E780C0E997F4FF1FE7
:10551000938404BE83C7040041479387070693F72B
:10552000F70F636AF75C17B701001307E7A38A0751
:10553000BA979C43BA9782879D476307F40297B551
:1055400001009385A50D17B501001305658E979091
:105550000100E78040E017B501001305A5B497905E
:105560000100E78040DFADAC97F7FF1F83C757B856
:10557000DDCB17F7FF1F0347D7B797F7FF1F83C789
:1055800047B722075D8F97F7FF1F83C7A7B6C207EC
:105590005D8F97F7FF1F83C7F7B5E207D98F17F71E
:1055A000FF1F2325F7B283C7640097B501009385D9
:1055B000E50617B501001305A58717F7FF1F23069A
:1055C000F7B097900100E78000D997F7FF1F938706
:1055D000E7AF8C4317F6FF1F034626AF17B5010050
:1055E000130505AE97900100E780E0D62945979016
:1055F0000100E78020DB97F7FF1FA38B07AE224453
:10560000B24092440249930700F817F7FF1F2301A5
:10561000F7AE9D4517F5FF1F130585AD41011743F3
:105620000000670023CC97600000E780408397F775
:10563000FF1F2380A7AC9357850017F7FF1FA30A0E
:10564000F7AA935705012A8417F7FF1F2304F7AA27
:1056500093578501014517F7FF1FA30DF7A8976022
:105660000000E780808097F7FF1F2386A7A897B5E3
:1056700001009385A5FA17A501001305657B979096
:105680000100E78040CD17F6FF1F0346C6A6A2859E
:1056900017B50100130545A4B1B7CD476303F40264
:1056A00097B50100938585F717A501001305457887
:1056B00097900100E78020CA17B50100130545A3A4
:1056C00079BD37E404007C44414697F5FF1F93857C
:1056D00035A217F5FF1F1305A59F829717F5FF1F2A
:1056E0001305059F97100000E78060C49710000025
:1056F000E78000AC97F7FF1F83C7A7A017F7FF1F2E
:10570000034717A0A20703238405D98F17F7FF1FAC
:10571000231CF79A1306000A89452244B24092449A
:10572000024917E5FF1F0345E50F410102838D473D
:105730006303F40297B50100938545EE17A50100B8
:105740001305056F97900100E780E0C017B50100D1
:105750001305C5A929B517F4FF1F0344849997F7CA
:10576000FF1F83C7F79897B50100938525EB2204A7
:1057700017A501001305C56B5D8C97900100E780AC
:1057800080BDA28517B5010013050598979001000B
:10579000E78060BC294597900100E780A0C00D46D6
:1057A00097F5FF1F9385C594228597E0FFFFE7805B
:1057B000C05CAA8421C197B50100938525E617A591
:1057C00001001305E56697900100E780C0B8A68543
:1057D00017B501001305859497900100E780A0B7E5
:1057E0002244B240924402492945410117930100E5
:1057F000670043BB97F7FF1F239E8784B7E704002A
:10580000116603A38705130606E8914539B78D474E
:105810006303F40297B50100938545E017A50100E5
:105820001305056197900100E780E0B217B501000C
:10583000130585AA2DB317F4FF1F0344848B97F734
:10584000FF1F83C7F78A97B50100938525DD2204E2
:1058500017A501001305C55D5D8C97900100E780D9
:1058600080AFA28517B501001305858C97900100C4
:10587000E78060AE294597900100E780A0B20D4611
:1058800097F5FF1F9385C586228597E0FFFFE78088
:10589000C04EAA841DC197B50100938525D817A5D0
:1058A00001001305E55897900100E780C0AAA6857E
:1058B00017B501001305058905B797E7FF1F239D5D
:1058C0008776B7E70400116603A38705130606E889
:1058D0009305000299B5894763E3870297B50100F4
:1058E0009385C5D317A50100130585549790010032
:1058F000E78060A617B501001305C5A08DB197E438
:10590000FF1F83C4047F97E7FF1F83C7777E97B588
:1059100001009385A5D0A20417A5010013054551E8
:10592000DD8C97900100E78000A3A68517B50100E4
:105930001305C58297900100E780E0A12945979063
:105940000100E78020A6228697E5FF1F9385457A10
:10595000268597E0FFFFE78040422A84630E051A00
:1059600097B50100938585CB17A501001305454C1C
:1059700097900100E780209EA28517A501001305DE
:10598000257F99BD854763F987188345190022440F
:10599000B24092440249B335B00097E7FF1F238518
:1059A000B76C17A501001305E57D410117930100B0
:1059B0006700639AA2852244B24092444A85024914
:1059C0004101170300006700032299476303F402B3
:1059D00097B50100938585C417A5010013054545BA
:1059E00097900100E780209717B50100130545AB9C
:1059F000BDB617E4FF1F0344C46F97E7FF1F83C7BB
:105A0000376F97B50100938565C1220417A5010082
:105A1000130505425D8C97900100E780C093A28535
:105A200017A501001305857797900100E780A092E4
:105A3000294597900100E780E096194697E5FF1FFA
:105A40009385056B228597E0FFFFE7800033AA84EA
:105A50001DC197B50100938565BC17A5010013050D
:105A6000253D97900100E780008FA68517A50100CE
:105A70001305C57395B397E7FF1F23938766B7E7B1
:105A80000400116603A38705130606E893050008C2
:105A900069B1854797B50100938545B817A5010001
:105AA00013050539630BF40097900100E780A08A85
:105AB00017A501001305C5705DB497900100E7803C
:105AC000808917A501001305257197900100E780D3
:105AD0008088294597900100E780C08C2244B2401D
:105AE0009244024997E7FF1F2390075E4101175335
:105AF00000006700432797B50100938525B217A5DD
:105B000001001305E53297900100E780C08417B5C6
:105B100001001305259DA1B4B240224492440249DC
:105B200041018280411106C622C497E0FFFFE78051
:105B3000C0249377F50FA1C32A8497B501009385FC
:105B400065AF17A501001305A52E97900100E7800A
:105B500080809375F40F17B50100130565D2978007
:105B60000100E780407F2244B2402945410117935C
:105B7000010067002383B240224441018280411129
:105B800022C491462A8417E6FF1F1306A6649D656A
:105B90002D4506C697D0FF1FE78040C1B7F7070025
:105BA00003C70701A5476313F70001A09306001080
:105BB00001469D65254597D0FF1FE78020BF97E7E9
:105BC000FF1F238987602244B240914617E6FF1FDA
:105BD000130646609D652945410117D3FF1F6700E5
:105BE000E3BC5171CAD137E904008327C904A2D5A7
:105BF0002E8686D7A6D32E84AA8517E5FF1F130508
:105C0000254F829797E7FF1F83C7874E1307700AB8
:105C10006387E710636CF7001307600A6384E70487
:105C2000BE502E549E540E596D6182801307800A17
:105C30006388E7161307900AE394E7FE8D4763092C
:105C4000F41C97B501009385E5D617A5010013054F
:105C5000251E97800100E780007017B5010013052D
:105C6000A5D225A08D47630CF40297B5010093855A
:105C700065D417A501001305A51B97800100E780D7
:105C8000806D17B50100130565C997800100E78095
:105C9000806C294597800100E780C07051B7854727
:105CA00017B50100130545C917E7FF1F230EF73A83
:105CB00097900100E7800082B7750200B766020086
:105CC0000146054597D0FF1FE78040AE930760F877
:105CD00017E7FF1F230EF74097E7FF1FA38B07402F
:105CE0009307002617E7FF1F2326F740E5779387E2
:105CF000072117E7FF1F2311F740B14597E7FF1F63
:105D0000238D073E97E7FF1FA389A73E17E5FF1FD7
:105D10001305053E97300000E780C05C11B791473E
:105D200063E3870297B501009385C5C817A50100F5
:105D30001305051097800100E780E06117B50100A9
:105D4000130585C199B797E4FF1F83C4A43A97E769
:105D5000FF1F83C7173AA204DD8C8327C9046D1483
:105D6000228697E5FF1F9385F538280082978E04D9
:105D700093160401B7750200C1823000A69509454B
:105D800097D0FF1FE78080A2930770F817E7FF1FE7
:105D90002300F736994597E7FF1FA38DA734BDB7BA
:105DA000914763E3870297B501009385A5C017A5C6
:105DB00001001305E50797800100E780C05917B57A
:105DC00001001305E5BAD1B597E4FF1F83C48432FF
:105DD00097E7FF1F83C7F731A204DD8C8327C9042F
:105DE0006D14228697E5FF1F9385D5302800829792
:105DF0008E0493160401B7750200C1823000A69587
:105E00000D4597D0FF1FE780609A930780F8BDBFCC
:105E100017B50100130585B897800100E780806BF6
:105E20001305C01297C0FF1FE780A051014597D00E
:105E3000FFFFE78000110D4597000000E78060D468
:105E4000294597C0FF1FE780C04F97C0FF1FE7801D
:105E50002040F9B341114AC09706002083D6268915
:105E6000328917D6FF1F0356865322C426C206C6A0
:105E70002A84AE8497000000E780A05F35C12DC062
:105E8000994763FF97048347140003470400A20760
:105E9000D98F13978700A183D98FC2073167C18338
:105EA0001307C755639EE70297D7FF1F83D7274F76
:105EB000A301F400A1832302F4009707002083D7F5
:105EC000078391C7A302F400A1832303F400A685EE
:105ED00017B50100130505B297800100E780A047C0
:105EE00097F7FF1F83C74770B9CF97D5FF1F83D59B
:105EF000054B17B501001305A5B197800100E78098
:105F000080452686A28517D5FF1F03554549970072
:105F10000000E78060C16301090497E7FF1F83C7A2
:105F2000672C9DCB95C897E7FF1F83C7E7138DE7C5
:105F300022852244B2400249A6859244410117338A
:105F400000006700233A17B50100130565AD97807F
:105F50000100E7802058C1B7B24022449244024970
:105F600041018280834755008345450017B50100F4
:105F7000130505A7A207DD8D178301006700A33D68
:105F800017B501001305C5A41783010067008354EA
:105F90008D4763FBB70A011126CA06CE22CC034403
:105FA000350097E4FF1F83C4F42397B50100938560
:105FB000E5A7B337800017E7FF1FA305F72209C441
:105FC00097B50100938545A717B50100130545A7AF
:105FD00097800100E780203897E7FF1F83C797204D
:105FE0006386970097000000E780602697E7FF1F11
:105FF00083C7571F8DC785472306F100B7E7040005
:1060000083A747177000854513055030829717B551
:1060100001001305E5A397800100E780A04B996775
:10602000938757EE2316F100680085479145A30733
:1060300081002307F10097300000E780A02AF2409A
:106040006244D244056182808280894763F7B70841
:10605000011122CC06CE26CA8344250085472A8416
:10606000639DF404914763F5B704034545008347F6
:10607000340022055D8D97D7FF1F2392A73297002A
:106080000000E780E0479967938767EE2314F100EB
:106090008347340023059100A305F10083474400A2
:1060A000954528002306F10097300000E780802303
:1060B000F2406244D24405618280FDF8996793877B
:1060C00067EE2314F10097D7FF1F83D7472DA30551
:1060D000F10023050100A183E1B7828001119967D6
:1060E00022CCD51717F4FF1F130404502314F1001A
:1060F0008347040026CA97F4FF1F9384445F230557
:10610000F10083D7040028009545A305F100A18381
:1061100006CE2306F10097300000E780A01C03D6CE
:1061200004008345040017B501001305E59397802B
:106130000100E7804022F2406244D244056182803F
:106140009D677971D9172316F10097F7FF1F83C751
:10615000A74906D62307F100A9C3B7E70400FC4707
:10616000414697E5FF1F9385A5F61305F100829739
:106170006800CD4597300000E780C01697F5FF1FF7
:1061800083C5854617B50100130505919780010069
:10619000E780601CB25045618280B7E70400BC47CD
:1061A000414681451305F1008297D9B7B7670204CC
:1061B0005D71938757AA3EC0930700302312F10008
:1061C00097F7FF1F9387474283C70700A2C4A30323
:1061D00001002303F10097F7FF1F9387475183D7EF
:1061E000070037E4040086C62314F10097D7FF1F89
:1061F0009387E71A83D70700414668002315F1000B
:106200007C4497E5FF1F9385A5EC8297F1450A85AD
:1062100097000000E780E021231EA1007C448A85CE
:106220000810794682973C441305E10309468145ED
:106230008297101093050002014597D0FFFFE78079
:10624000C036B640264461618280B7C7A55A0111A5
:106250009387C7333EC497E7FF1F83C7B7F83EC68F
:10626000B7F7070003C7070106CE22CCA547631383
:10627000F70001A01164930504F093060010014695
:10628000254597C0FF1FE78060523000930504F05A
:10629000A146294597C0FF1FE780405197E5FF1FA2
:1062A00083C555F417B501001305C58F978001000C
:1062B000E780600AF24062440561828001119165C5
:1062C000A1463000938505F02D4506CE97C0FF1FEF
:1062D000E780C04D2247B7C7A55A9387C7336314D9
:1062E000F702B24517A501001305057FB335B000CD
:1062F00097E7FF1FA388B7EE97800100E780A0050E
:10630000F24005618280814517A501001305057FD4
:1063100097E7FF1FA38807EC97800100E780A003A1
:1063200097000000E780A0F2E1BFB7C7A55A7971D6
:106330009387F7353EC6B7E70400FC47AA8506D623
:1063400022D4414608088297B7F7070003C7070120
:10635000A5476313F70001A01164930504E89306B1
:1063600000100146254597C0FF1FE78020447000BC
:10637000930504E8D146294597C0FF1FE7800043F5
:1063800017B501001305C58597800100E7808014CB
:10639000B25022544561828079719165D146700076
:1063A000938505E82D4506D697C0FF1FE78000407E
:1063B0003247B7C7A55A9387F73517A501001305CC
:1063C000E57B6310F702B7E70400FC4717E5FF1F02
:1063D000130505D041460C08829717A50100130547
:1063E000E57797800100E780E00EB250456182803A
:1063F000B7F7070003C70701A5476313F70001A01C
:1064000091654111930600100146938505E82545E5
:1064100006C697C0FF1FE7806039B24017A501008C
:106420001305C5694101178301006700A30AC1670D
:1064300069768146FD17050613970601418363645B
:10644000B7003E8582803307D50003470700B98F28
:10645000214713F81700858363050800B18FC20731
:10646000C1837D171377F70F6DF78506F1B741C527
:10647000A547054763F2B7088347150003470500A2
:106480003168A207D98F13978700A183D98FC207DC
:10649000C1831308C855054763900707411106C615
:1064A00022C426C203442500914763F08704930762
:1064B000540063ECF502A301C50021822302C5004C
:1064C0009304340091C6A302D500A1822303D50012
:1064D0002A84A68597000000E780A0F52694230073
:1064E000A4002181A300A4000147B24022449244A9
:1064F0003A854101828005473A858280B7C7A55A0F
:1065000001119387E7343EC42AC6B7F7070003C7D3
:10651000070106CE22CC26CAA5476313F70001A0C7
:1065200091642A84938504EE930600100146254564
:1065300097C0FF1FE78080273000A146938504EEB7
:10654000294597C0FF1FE7806026A28517A5010097
:106550001305456797800100E780E0DF97000000A2
:10656000E78000C5F2406244D24405618280011197
:106570009165A1463000938505EE2D4506CE97C066
:10658000FF1FE780A0222247B7C7A55A9387E734A9
:106590006318F702B24517A501001305255897D7D0
:1065A000FF1F239EB7DEC205C18197800100E780EF
:1065B00080DA97000000E780A0BFF240056182808A
:1065C000D147D14517A501001305455717D7FF1F20
:1065D0002317F7DC97800100E780E0D717D5FF1F6E
:1065E0000355E5DB97000000E78080F1F9B7011162
:1065F00026CA06CE22CC93F71500AE848DCBAD67AC
:10660000371700409387A7AA1CC3B7E70400BC4F05
:1066100013060019854517D5FF1F034525D8829716
:1066200013C51400F2406244D2440561828093F79E
:1066300025006386071897A501009385655E2D46A2
:10664000480097800100E780A0C597F5FF1F83C52C
:10665000E509854793C4240063E5B7049DC98545D2
:1066600017F5FF1F130585F897200000E78060A944
:1066700097E7FF1F83C707B789CF97F5FF1F83C52C
:10668000E50617F5FF1F130565F697300000E78054
:1066900060C51395040197F7FF1F23890704418103
:1066A00051B717F4FF1F034464F497F7FF1F83C724
:1066B000F7F322045D8CAD67C2059387B755C1819E
:1066C000630DF40C63E18704A9679387A755630FF3
:1066D000F40C17F5FF1F130565F197200000E78004
:1066E00040A297E7FF1F83C7E7AFD1CF97F5FF1F02
:1066F00083C5C5FF17F5FF1F130545EF9730000051
:10670000E78040BE49A0B1679387C7556302F40490
:10671000B5679387D755E31EF4FA17F5FF1F1305E6
:10672000E5EC97300000E780E0BB97F5FF1F83C5DD
:10673000E5FB894763F9B704F915C205C18117F56F
:10674000FF1F1305C5EA97200000E780809B25A85E
:10675000054617F5FF1F130565E997F0FFFFE78072
:10676000A06F97F7FF1F83C727E891EF4800978036
:106770000100E780E0DE93150501C181480097D054
:10678000FFFFE780A090A28517A5010013054547EC
:1067900097800100E78020BCEDBD17F5FF1F1305B2
:1067A000E5E497F0FFFFE780207CF1BF17F5FF1FBE
:1067B0001305C5E397F0FFFFE780C07CE9B793F7C7
:1067C00045000145E38007E617A501001305854450
:1067D00097800100E78000D097300000E780A0C4D8
:1067E00013C5440081B5411122C437E404005C5C48
:1067F00006C6354697A501009385C5EC17B501007F
:10680000130545B1829711E917A50100130505424B
:1068100097800100E78000CC01A08327041C8297A9
:106820002A84054597B00000E780407F976001000B
:10683000E780600497600100E78060D997B00000AE
:10684000E780C0902285B2402244410182801567D2
:10685000B71700401307575598C3D8439D66558F07
:10686000D8C3D843FD76758FD8C3D8431367F70FC5
:10687000D8C335671307C7CC98C38280411113056D
:10688000800406C622C426C297C0FF1FE78020826C
:1068900085457D5597C0FFFFE780E05185457D55D3
:1068A00097C0FFFFE780805B371400408327840A8E
:1068B0008D451305002093E707202324F40A97C091
:1068C000FFFFE780404FB7E4040097D0FFFFE78069
:1068D0006082C85897800100E780C0BF17B50100EB
:1068E000130545A397800100E780C0BE8327840C71
:1068F0008545414593E707082324F40C97C0FFFF23
:10690000E780C0558D451305000897C0FFFFE7805D
:10691000E05497C0FFFFE780A06F014597C0FFFFDD
:10692000E780807285450545894717F7FF1F2301DA
:10693000F7DC97C0FFFFE780C07237070004B7E7B6
:1069400000E023A0E71097D0FFFFE780600497D016
:10695000FFFFE780201897000000E78000E997001C
:106960000000E780E09597000000E78080C097E096
:10697000FFFFE78060FB97000000E7806010970052
:106980000000E780600B83A70408170500001305CB
:1069900045C6829797D7FF1F2382A7A0BC4C13063A
:1069A00000648545829797000000E78080EA97C0E1
:1069B000FF1FE780E0A301458280B7F7070003C708
:1069C0000701A547AE866316F7009397450191C36B
:1069D00001A0AA850146254517C3FF1F670003DDF7
:1069E0004111B2862E86AA852D4506C697C0FF1F87
:1069F000E780C0DBB240014541018280930700047B
:106A000063E8C7021D71A2CC2A84080886CE32C66C
:106A100097800100E780C088B2461008A28529450A
:106A200097C0FF1FE78080D8F640664425618280CA
:106A30003955828041110D658D4506C697C0FFFF0F
:106A4000E7806037B71700408D6623A6D70A17F591
:106A5000FF1F130525CA1387C70A9387870A1CC11E
:106A60005CC5856689675CC958C114C518C9B7E794
:106A70000400B24003A3871E4101028397F7FF1F62
:106A800083C7C7C899EF411106C697100000E78079
:106A90006061B240854717F7FF1F2309F7C6410120
:106AA0008280828011C589C517C3FFFF6700035E1E
:106AB0008280411126C2AE848D4522C406C62A8436
:106AC00097C0FFFFE7808039B717004099C803A53A
:106AD000C70C418D23A6A70CB24022449244410129
:106AE000828003A5870C418D23A4A70CF5B78347AB
:106AF000050003471500A207D98FC2076177C18738
:106B000013072720639AE700834525003705040013
:106B100017030000670023FA828017F6FF1F130691
:106B200026BF8147B2861303F00FA9483308F60049
:106B30000348080013F7F70F6307A80C6306680003
:106B40008507E39517FF2947B387E6002380A70051
:106B500097F7FF1F938787BC5DA8411113D7650086
:106B60001347170006C693F63500058B954791CA63
:106B7000054699476387C60009469D476383C6005B
:106B8000A14713F645003336C00093F6850305068A
:106B900085C2A145638BB604E145638AB6049305BB
:106BA00080026388B604930580036393B600914620
:106BB00097F5FF1F2389F5DC97F5FF1F2384C5DCBC
:106BC00097F5FF1FA380D5DCBE8517A5010013052F
:106BD000650F97700100E7800078B240854717F78E
:106BE000FF1FA302F7DA410182808546D1B78946AB
:106BF000C1B78D4675BF17A501001305250F177383
:106C000001006700437517F7FF1F130727B1BA97F5
:106C10002380B700E147E302F5F493077002E30C29
:106C2000F5FC82802A8723800500814717F5FF1F26
:106C3000130505AE1308F00F2946B306F50083C609
:106C400006006396E60297F6FF1F938626ADB69779
:106C500083C7070005452380F5009947636EF70257
:106C60009D4763FDE700E147630DF7008280638580
:106C700006018507E393C7FC0145C5B723800500DE
:106C80008280B737004003C7370083C7050093F7FA
:106C90000704D98F2380F5008280797126D24AD0EB
:106CA00097F4FF1F83C404E017F9FF1F1309C9DE1F
:106CB00006D622D44ECE52CC56CA5AC8B307990033
:106CC00083C7070093F7F70FA5C79387140093F7BF
:106CD000F70F0D476361F70C17F7FF1F2304F7DC6D
:106CE00097F7FF1F9387C7DBA69783C70700130794
:106CF000100293F7F703638FE7286363F70A0544ED
:106D000063808720E389076E09476389E7141307C7
:106D10000002E38EE758B7E700E03707400023A002
:106D2000E71801000100CA942380040023A0E710A3
:106D3000B787004003C76700058BE30F077897F616
:106D4000FF1F83C646D60547E39AE6762947238187
:106D5000E70209472383E7022385E70297F7FF1F2E
:106D6000A38407C297F7FF1FA38F07D2B7870040FE
:106D7000A381070017F7FF1FA30A07C00547238356
:106D8000E700B250225492540259F249624AD24A60
:106D9000424B4561828097F7FF1F238507D089B753
:106DA000130730026386E70A63E6E714130740021D
:106DB000638AE70813070003E39FE7F497F7FF1FD1
:106DC0009387C7CDA69703C70700A1471377F70F8F
:106DD000E31AF71C17FAFF1F130A0A9583476A0084
:106DE00097F6FF1F2388F6B897F7FF1F83C73794DE
:106DF00091C7FD5797F6FF1F238EF6B697F5FF1F35
:106E000083C5959297F7FF1FA386B7B697F7FF1F25
:106E100083C7879193F907089306000493F7070641
:106E20006393D7529307A009638DF51A63EAB716E7
:106E30009307F005638AF54E930750096388F52E92
:106E4000014479ABFD5717F7FF1F2304F7B2E1B5F3
:106E5000FD5717F7FF1F230DF7B075BD17A50100EC
:106E6000130545FA97700100E780C06697F7FF1F8A
:106E70009387C7C2A69703C40700814917FAFF1F6B
:106E8000130A0AA31374F40F97AA0100938A0AF84D
:106E900063C78904294597700100E780A0508547A2
:106EA00017F7FF1FA304F7A017F7FF1F230187A001
:106EB00017F7FF1F230AF7AC37E700E0B7064000DB
:106EC0002320D71801000100378600408347A6021F
:106ED00093F7370F2305F6022320D7102DBDB307F4
:106EE0003A0183C507005685850997700100E78040
:106EF000804679BF854717F7FF1F2309F79A21BD01
:106F000017A50100130505F097700100E780805C6C
:106F100097F7FF1F938787B8A69703C40700814997
:106F200017FAFF1F130A8A8C1374F40F97AA010033
:106F3000938ACAED63C58904294597700100E780EB
:106F40006046854717F7FF1FA300F78A17F7FF1F53
:106F5000230D878817F7FF1F2308F7A237E700E004
:106F6000B70640002320D7180100010037860040F3
:106F70008347660293F7370F2303F602B1BFB307C7
:106F80003A0183C507005685850997700100E7809F
:106F9000803C4DB7854717F7FF1F2307F784A5BB34
:106FA0009307400A638DF5349307200B6388F53609
:106FB0009307100AE396F5E883072A00014463D19A
:106FC000074297E7FF1F83C7577693F63700638E14
:106FD000061A0546638EC62209466399C61A1D47DE
:106FE00075A217E5FF1F03454574C94717EAFF1F40
:106FF000034ABA7397E5FF1F83C5457317E4FF1F64
:107000000344D4726319F510CD476316FA10930741
:107010007008639CF5021307300FB7170E00630862
:10702000E4001307900DB7B704006314E40817F7E2
:10703000FF1F2327F794BE8517A50100130585DDE3
:1070400097700100E7802031E5BB93078008639DBE
:10705000F50033048040B77746001374F40F93872C
:1070600087CDB3D78702E1B793079008639AF500FD
:107070003304804091671374F40F9387C766D5B7C4
:107080009307A008639BF50033048040B7173D00C9
:107090001374F40F93870790E9B79307B008639AC6
:1070A000F5003304804091671374F40F938797D0F1
:1070B0004DBF93F5F5078D47639BF5003304804082
:1070C000B7975B001374F40F938707D859BF8947AC
:1070D000639BF50033048040B7770B001374F40F03
:1070E0009387071BBDBF8547639AF5003304804033
:1070F000DD671374F40F938767E3A5B789E9330459
:1071000080408D671374F40F938777DC99BFF16724
:107110009387072029BF97000000E78040A0A28541
:10712000528597000000E780809F19BB930561009E
:1071300017E5FF1F0345655F17E4FF1F0344F45E77
:1071400097000000E78040AE93057100228597000C
:107150000000E78060AD3C0017F7FF1F232CF7927B
:10716000834761002304F10083477100A304F10009
:10717000894717E7FF1F230FF77E8357810017E723
:10718000FF1F2313F75A0944A1AC154793F6470094
:10719000B336D00093F78703850685C32146638BFA
:1071A000C7066146638AC706130680026388C7065E
:1071B000130680036393C700914717E6FF1F23035D
:1071C000D67C97E6FF1FA38FF67A97E7FF1F238CE5
:1071D000E77A17E7FF1F034767559376070497E79A
:1071E000FF1F83C7B7548DEE1377770C9306700893
:1071F000630CD7021377F7078D46631ED70AB307D0
:10720000F040B7955B0093F7F70F938505D881A8F9
:107210001947ADBF854755B7894745B78D4771BFFA
:10722000930670086311D7021307300FB7150E00CD
:107230006389E7021307900DB7B504006383E70283
:107240001307700845BF9306800C6311D702B3077C
:10725000F040B775460093F7F70F938585CDB3D50A
:10726000F50297E7FF1F23ADB770F9B39306900CB3
:10727000631AD700B307F040916593F7F70F938532
:10728000C566F1BF9306A00C631BD700B307F0409F
:10729000B7153D0093F7F70F93850590C9B793068F
:1072A000B00CE319D7F4B307F040916593F7F70FEB
:1072B000938595D06DB78946631BD700B307F0401F
:1072C000B7750B0093F7F70F9385051B49BF8546EC
:1072D000631AD700B307F040DD6593F7F70F938586
:1072E00065E3B5BF09EBB307F0408D6593F7F70F82
:1072F000938575DCADB7F165938505209DB7834710
:107300002A00C18B99C7854717E7FF1F2307F76638
:1073100005BE97E7FF1F238207661DB6854717E75F
:10732000FF1FA302F76629BE3C0017E7FF1F2323B8
:10733000F7760947930700032314F10097E6FF1F30
:10734000238AE6622DBD639A0758A94763ECB744C8
:1073500017A70100130747948A05BA959C41BA976D
:10736000828717E4FF1F0344543C094A630C440F0F
:10737000636C8A0885476309F40A9307F00F17E7DF
:10738000FF1F0347275F63F6E70017E7FF1F23038D
:10739000F75E17EAFF1F034AEA5D930700041374C0
:1073A000FA0F63F447011304000497E7FF1F938764
:1073B000676E83AA0700228617E5FF1F1305C536EF
:1073C000D685330A8A40A29A97700100E78040ED83
:1073D00097E7FF1F2380475B97E7FF1F23AC576B9F
:1073E00097E7FF1F83C717591547639AE762B7E707
:1073F00000E03707400023A0E71801000100B7862E
:107400000040238086028DA58D47630CF40A9947BE
:10741000E315F4F697A701009387878E17E7FF1F00
:10742000232AF766A947A1BF17E7FF1F0347A767EE
:1074300097E7FF1F93870756494697A50100938555
:1074400025956306870097A50100938565903E8585
:1074500097700100E780C0E417E7FF1F232CA762A5
:10746000C94731BF97E6FF1F83C6E663054797E725
:10747000FF1F938727526394E6023E85130670022E
:1074800097A501009385458E97700100E78040E144
:1074900017E7FF1F2320A76093077002CDB53E8535
:1074A0001306300497A50100938545869770010067
:1074B000E78000DF17E7FF1F232EA75C9307300448
:1074C0007DBD97E5FF1F83C5452617A50100130560
:1074D000A59597700100E78000E8854A17EBFF1F2C
:1074E000034B6B5C97E5FF1F83C5252417A501009F
:1074F0001305859363185B0B97700100E780A0E587
:1075000097E7FF1F83C76722B5CBE368F4E617A4AC
:1075100001001304248C638C670117A40100130479
:10752000E48B6386470117A401001304A48C228511
:1075300097700100E780C0021375F50F93071500DF
:10754000860717E7FF1F2307F7448D4717E7FF1F3D
:10755000A302F74497E7FF1F9387C7430147BE86FF
:107560001376F70F89076365A60297E7FF1F23A32A
:10757000D75297E7FF1F83C7E74111B597970100DF
:107580009387477E17E7FF1F2326F7509147C5BB18
:107590003306E40003460600A380070005072380A6
:1075A000C7007DBF97700100E780E0DA97E7FF1F13
:1075B00083C7A717E1D7E362F4DC17940100130433
:1075C000647E638C5701179401001304247E638644
:1075D0004701179401001304E47E2285977001008F
:1075E000E78000F81375F50F93071500860717E776
:1075F000FF1F2301F73A8D4717E7FF1FA30CF7384A
:1076000097E7FF1F938707390147BE861376F70F69
:107610008907E37CA6F43306E40003460600A38052
:10762000070005072380C700D5B797E5FF1F83C56F
:10763000C50F179501001305E57F97700100E780DE
:1076400080D197E7FF1F83C7B73493E7470017E759
:10765000FF1FA30FF73283472A0017E7FF1FA30777
:10766000F7326FF0EFFD179501001305E57D977078
:107670000100E78020E697E7FF1F9387273183C744
:10768000070017E7FF1F2301F70A17E4FF1F034452
:10769000642E33348000A9B3179501001305057CCF
:1076A00097700100E78000E397E7FF1F83C7572E1D
:1076B00093E7070117E7FF1FA30CF72C83472A0066
:1076C00017E7FF1F2304F72C6FF08FF717950100C2
:1076D0001305057A97700100E780C0DF03470A00B1
:1076E0007D8B51EFB787004003C767021377C70B45
:1076F000136727002383E70203C7A7021377C70B8B
:10770000136727002385E70203C7E7021377C70B38
:10771000136727002387E70203C727031377C70BE5
:10772000136727002389E702854717E7FF1F230D0B
:10773000F70A17E7FF1F230BF71617E7FF1F2309A9
:10774000F72217E7FF1F2306F72297E7FF1FA38DF6
:10775000070897E7FF1FA38B071497E7FF1FA3896D
:10776000072097E7FF1FA386072097E7FF1FA38D3A
:10777000072097E7FF1FA38807326FF06FEC894758
:107780006312F70297E7FF1F83C747FA9146638C9E
:10779000D70863E0F604638EE70C6369F70A0547D0
:1077A0006380E70EFD5717E7FF1FA305F71C370798
:1077B0004000B7E700E023A0E71801000100B7860A
:1077C00000401306F0FC2381C60223A0E7106FF0EF
:1077D0008FD4130720086382E7086362F702130758
:1077E0001008E391E7FC378700408347670293F76F
:1077F000C70B93E727002303F7026FF06FE413072B
:1078000030086389E70213074008E39DE7F83787EC
:1078100000408347270393F7C70B93E7270023090B
:10782000F7026FF0EFE1378700408347270393F7B4
:107830003707F5B7378700408347E70293F7C70B51
:1078400093E727002307F7026FF08FDF37870040A9
:107850008347E70293F73707F5B737870040834739
:10786000A70293F7C70B93E727002305F7026FF0F2
:107870002FDD378700408347A70293F73707F5B717
:10788000378700408347670293F73707ADB71795EF
:1078900001001305E55E97700100E780A0C397E73C
:1078A000FF1F238307E8D5B3179501001305455E35
:1078B00097700100E78000C297E7FF1F239607E655
:1078C00097E7FF1F9387070B03C40700894763F3FC
:1078D000870009441374F40F21B613070002E393E1
:1078E000E7EC6399090A638FF5009307200263812F
:1078F000F508179501001305255D97700100E780D5
:1079000080A54DB5179501001305455997700100E5
:10791000E78040BC0144179B0100130B6B59A14A3F
:10792000B3078A0083C507005A85050497700100D4
:10793000E78060A2E31654FF17950100130505B612
:1079400097700100E78000B917E4FF1F034404DECD
:1079500011E497E7FF1F238C07DA59B48947E31333
:10796000F4E4854717E7FF1F2303F7DA6FF04FCDE5
:1079700017E6FF1F034676DB97E5FF1F83C5E5DAB1
:10798000179501001305455397700100E780A09CEF
:107990006FF00FCB638FF50493071002E39BF5F4B0
:1079A00097E5FF1F83C585D8179501001305C552BC
:1079B00097700100E780209A97E7FF1F23AC470DDF
:1079C00097E7FF1F9387C7FB944383D7470017E7C9
:1079D000FF1F034747FB17E6FF1F2327D6D41D448D
:1079E00097E6FF1F2394F6D497E7FF1F2381E7D480
:1079F000C5BA97E5FF1F83C565D317950100130529
:107A0000254F97700100E780009597E7FF1F2380BF
:107A100007D097E7FF1F239907D06FF0CFF62547D0
:107A2000E387E79C19476391E702B786004023800C
:107A30008602B7E700E03707400023A0E7180100FF
:107A40000100130600FC41B31307100A6391E7021B
:107A5000B786004023808602B7E700E03707400082
:107A600023A0E71801000100130680FCA9BB13073F
:107A7000A009E38FE7FC1307400AE38BE7FC130739
:107A80002002E386E7960547E383E796B7E700E041
:107A90003707400023A0E718E39109960100010091
:107AA000B786004023808602130620FC29BB17E717
:107AB000FF1F034737EC6308F71E63E7E7029547AC
:107AC000630EF70E99476308F704B78600402380DA
:107AD0000602B7E700E03707400023A0E7180100DF
:107AE00001001306A0FCC5B19307F005630AF70077
:107AF000930750096306F70093071002E317F7FC9A
:107B0000B7E700E03707400023A0E71801000100B5
:107B1000B786004051BF97E9FF1F83C9A9E59307C6
:107B20000004CE8A63F43701930A000497E7FF1F2D
:107B3000938747F603AA070013F4FA0F2286D2852B
:107B400017E5FF1F130545BE97600100E7804075EC
:107B5000B3878940529417E7FF1F230DF7E097E79B
:107B6000FF1F23A987F2638E0902B7870040238095
:107B70005703B7E600E03706400023A0C61801000F
:107B8000010003C72702134707042381E70203C745
:107B900027021377C70F2381E70223A0C6106FF0D7
:107BA0008F97B786004023800602B7E700E03707CB
:107BB000400023A0E71801000100FDB53787004011
:107BC0008347370097E6FF1F83C656DC93F7070805
:107BD000D58FA301F700B7064000B7E700E023A068
:107BE000D718010001001306A0FC2301C70223A03F
:107BF000D7106FF04F9297E7FF1F938727EAA6975A
:107C000083C7070093F7F70FD9CF97E7FF1F83C705
:107C100087E9D1EB17E7FF1F0347D7D5930700028A
:107C20006313F70897E7FF1F938707B003AB0700BD
:107C300097EAFF1F83CA8AAF17EAFF1F034A1AAFEA
:107C400097E9FF1F83C9A9AED2875687CE865A8689
:107C500097E5FF1F83C5A5AB179501001305C52A3E
:107C600097600100E780206F97E7FF1F23AA67D185
:107C700097E7FF1F238857D197E7FF1FA38447D1BA
:107C800097E7FF1F238137D197E7FF1FA38087A8BE
:107C9000B7E700E03707400023A0E7180100010024
:107CA000B7860040D1B3B7E700E03707400023A014
:107CB000E71801000100B786004025B52947238158
:107CC000E70209472383E7022385E7022387E702C8
:107CD0002389E7026FF08F8803C76700118B630267
:107CE000078A83C75700918BB5CF17E7FF1F03475C
:107CF00087DB85476313F70697E7FF1FA385E7C870
:107D000097E7FF1F238207AE97E7FF1F238007BA7D
:107D100097E7FF1F238E07C497E7FF1F238B07C436
:107D200097E7FF1FA38207AC97E7FF1FA38007B861
:107D300097E7FF1FA38E07C297E7FF1FA38B07C21A
:107D400097E7FF1FA38207C497E7FF1FA38D07D400
:107D5000B787004011476FF08F8217E7FF1FA30717
:107D6000F79A79BF854717E7FF1F230FF7A617E795
:107D7000FF1F230DF7B217E7FF1F230BF7BE17E70F
:107D8000FF1F2308F7BE69BF854717E7FF1F230DB5
:107D9000F7A417E7FF1F230BF7B017E7FF1F23090F
:107DA000F7BC17E7FF1F2306F7BC17E7FF1FA30D5C
:107DB00007A217E7FF1FA30B07AE17E7FF1FA309D3
:107DC00007BA97E7FF1FA38607BA8280411106C64C
:107DD00097000000E78080FBB78700402380070002
:107DE000130740FC2386E7001307C004A386E700BF
:107DF00017E7FF1F130747932398E70017E7FF1FB5
:107E000013078796239AE70017E7FF1F130707A2B8
:107E1000239CE70017E7FF1F130787AD239EE700AA
:107E200029472381E70209472383E7022385E702E5
:107E30002387E7022389E702A3810700930600F85E
:107E4000A380D700930690022380D700FD5623839A
:107E5000D7002381E700B706400037E700E0232082
:107E6000D71003C7170013671700A380E700B240BD
:107E700097E7FF1F239C07B041018280411106C68E
:107E800097000000E78080F0B7870040238007005C
:107E9000130700FC2386E7003147A386E70017E7B6
:107EA000FF1F130767882398E70017E7FF1F1307D3
:107EB000A78B239AE70017E7FF1F13072797239C39
:107EC000E70029472381E70209472383E702238547
:107ED000E702A3810700930600F8A380D70093066A
:107EE00090022380D700FD562383D7002381E7002B
:107EF000B706400037E700E02320D71003C717007C
:107F000013671700A380E700B24097E7FF1F239F86
:107F100007A641018280F1679387072017E7FF1FBB
:107F20002320F7A6854717E7FF1F231DF7A4A147C6
:107F300017E7FF1F2309F7A497E7FF1FA38507A4EF
:107F400097E7FF1F238207A497D7FF1F2381077C92
:107F500097D7FF1FA38C077A814717D5FF1F1305FB
:107F6000257BFD5517D6FF1F1306467B2947B30611
:107F7000F5002380B600B306F600238006008507CF
:107F8000E397E7FE97E7FF1F238807B097E7FF1FF8
:107F9000A38407B097E7FF1F238107B097E7FF1F70
:107FA000A38B079C97E7FF1FA389079C97E7FF1FF9
:107FB0002384079C97E7FF1F238F079A97E7FF1FEC
:107FC000238E079A97E7FF1FA388079A97E7FF1F5B
:107FD0002385079A97E7FF1FA38107AC828017E7E5
:107FE000FF1F034747AC85476316F70017030000E0
:107FF000670003E917030000670083DD411122C415
:1080000006C617E7FF1F034707AA85472E8613F406
:10801000F50FAA856317F70417E5FF1F13050585FC
:1080200097600100E780C02797E7FF1F238007883C
:10803000B787004023848702B7E600E03706400098
:1080400023A0C6180100010003C7A7021377C70FBA
:108050002385E702B240224423A0C6100145410116
:10806000828017D5FF1F1305257497600100E780F4
:10807000202397D7FF1F23890776B78700402382E5
:108080008702B7E600E03706400023A0C6180100CB
:10809000010003C767021377C70F2383E7025DBFA1
:1080A000411106C697000000E78020E7B240410179
:1080B000170300006700E3F2411106C697F0FFFFC7
:1080C000E780E0BD97D7FF1F83C7177295C797D585
:1080D000FF1F83C5857189C917D5FF1F130505715A
:1080E00097F0FFFFE780409C97D7FF1FA38E076E96
:1080F00097E7FF1F238A0788B2404101828041C968
:10810000D9C597E7FF1F83C76788D1C3011122CC68
:108110004AC84EC656C25AC006CE26CA52C42E8976
:10812000AA890144930A0004371B030063772403E0
:10813000B3078940C207C183BE8463F4FA00930485
:108140000004C204C180130A1BD497D7FF1F83C742
:10815000A7699DE37D1A631C0A00F2406244D24481
:108160004249B249224A924A024B0561828097F005
:10817000FFFFE780C0B2D1BF338589002694A68572
:10818000420497000000E780A0E7418045B7828065
:1081900097E7FF1F9387C79418429C4383D64500F7
:1081A0000345070083C5C700035646006396A50034
:1081B00083D5E700638DD502011106CE2386A70083
:1081C0002397D700B705CF00DC4B9385757D050756
:1081D0007D162EC2230001003AC42316C1002317C6
:1081E000D10099C30A858297F2400561828082801E
:1081F000DC4DDC4B81CFB7E70400904503A3870536
:10820000914517E5FF1F0345E58D028382806D715F
:108210003C083EC6B707E500232291103EC8AA8459
:108220003C083285232611103ECA232481102320C6
:1082300021112E8997300000E780405C2A849795B1
:1082400001009385E5CF17850100130565BE976092
:108250000100E7804010A285179501001305C5DED7
:1082600097600100E780200F294597600100E780B3
:108270006013B705CB009385757D680097100000EB
:10828000E7806065A285680097300000E78060495C
:10829000014781467000CA85268597200000E78047
:1082A000E08805CD2A8497950100938565C91785D7
:1082B00001001305E5B797600100E780C009A285BA
:1082C00017950100130505D997600100E780A00804
:1082D000294597600100E780E00C8320C11003244A
:1082E000811083244110032901105161828097D7A6
:1082F000FF1F9387E77E18429C43797122D406D6EC
:108300000348070083C807012A8483D64500035524
:1083100046006396080183D82701638DD80223881D
:10832000070105072399D7003708CC00DC4B130859
:10833000787D3ACC1307F5FF42CA23080100231EBB
:10834000E100231FD10099C7080832C62EC48297C6
:108350003246A245228597000000E78080EBB250AC
:108360002254456182806D713C083EC0B707E5002C
:108370003EC23C083EC42326111023248110232230
:108380009110231701002318010023190100231A5B
:108390000100231B010097B7FF1F83D7A70299E3B2
:1083A000C167FD172316F10097B7FF1F83D7A701F9
:1083B00091EB97D7FF1F9387A7729C439C43DC47A1
:1083C00083D7070017B4FF1F1304C4FF584C2317AB
:1083D000F10083574400484B2318F10031E1979591
:1083E00001009385E5BC17850100130565A497601E
:1083F0000100E78040F6179501001305A5BC9760C2
:108400000100E78040F5294597600100E78080F989
:108410008320C11003248110832441105161828084
:1084200097B7FF1F83C777FA89EBB7E70400BC57FC
:1084300082975C4C23AA0700E1BFFD1797B6FF1F88
:10844000A385F6F803560701834704014C470A85C4
:10845000230BF10097300000E780C02997D7FF1F5A
:10846000938707689C430147814688430A866C00CE
:1084700097100000E780806BAA8429C197950100BE
:10848000938505B3178501001305859A9760010050
:10849000E78060ECA68517950100130565B397602A
:1084A0000100E78040EB294597600100E78080EFFD
:1084B000584CB7E70400BC57484B9DBF97B7FF1F08
:1084C00083C7B7F0F5D7B7E70400BC4F1044854524
:1084D00017D5FF1F0345056182971DBF5C4EDC4B1E
:1084E000B9CFB1CD411122C41785010013054594C0
:1084F0002E84979501009385E5A906C69760010033
:10850000E78060E5A28517950100130525AF976008
:108510000100E78040E4294597600100E78080E89A
:10852000B7E704002244B24003A3870517D5FF1F15
:108530000345455B13064006914541010283828055
:10854000411122C417B4FF1F130484E51C4C06C656
:1085500089C7DC4399C34C488297584CB7E704005D
:10856000BC57484B82975C4CB240224423AA070078
:108570004101828017B7FF1F130787E48347070075
:108580009306F00B850793F7F70F63E9F60097B6AC
:10859000FF1F2387F6E2034507008280930700F858
:1085A000FDB7835745006386071001114AC817B904
:1085B000FF1F130929E152C4032AC90106CE22CCA8
:1085C00003274A0126CA4EC656C2F15735E31307A0
:1085D000D00DFD57636EC704B7E9040083A70907F0
:1085E0002A841305860042054181B284AE8A8297AF
:1085F000232AAA000325C9015C49A9E79795010030
:1086000093854597178501001305858297600100C2
:10861000E78060D417950100130585A697600100D7
:10862000E78060D3294597600100E780A0D7DD5738
:10863000F2406244D2444249B249224A924A3E85BB
:108640000561828093874400B705CF002319F500A8
:108650009385757D310597100000E780C0270325BD
:10866000C90183456400310597300000E780600B45
:108670000325C9012686D685310597300000E7809D
:1086800060077146A2854A8597600100E78040C176
:10869000504419CA83A78905854517D5FF1F03458F
:1086A00065448297814769B797000000E780E0CB77
:1086B000D5BFFD573E858280411126C297B4FF1F6A
:1086C000938444D0D84C22C437E404003C54484B33
:1086D00006C68297DC4C0323C4052244B240924470
:1086E00023AA070017D5FF1F0345C53F8545410154
:1086F0000283411126C297D4FF1F9384643E9C409D
:1087000006C622C44AC0D5C3DC43C5C35CC123002E
:10871000B5002A849795010093850581177501009E
:108720001305057197600100E780E0C22945976055
:108730000100E78020C79C4023A4070023A2070074
:1087400097B7FF1F9387C7C5DC4FDC4B91C72955EF
:1087500097000000E78000DF97B7FF1F938787C669
:10876000DC4FDC4B89C797000000E78020F537E934
:1087700004008327C905894517D5FF1F03458536A2
:1087800082978327C905914517D5FF1F0345853576
:1087900082979C4003A3470163090300228522447A
:1087A000B2409244024941010283B24022449244C1
:1087B0000249410182800111328506CE22CC26CAAF
:1087C0002E8497300000E7806003AA84978501001B
:1087D0009385C578177501001305856597600100BD
:1087E000E78060B7030784000356640083554400A4
:1087F000A686179501001305658297600100E78042
:1088000080B5294597600100E780C0B997B7FF1F81
:1088100083C767B9639D9700014597000000E78013
:1088200060D281450A8597000000E780C0ECF240E5
:108830006244D244056182806D7123248110232615
:1088400011102322911093F745002E84638707149B
:108850003C083EC0B707E5003EC23C083EC42317B3
:1088600001002318010023190100231A0100231B12
:10887000010097B7FF1F83D7A7B299E3C167FD1720
:108880002316F10097B7FF1F83D7A7B191EB97D7B6
:10889000FF1F9387E7249C439C43DC4783D7070053
:1088A00017B7FF1F1307C7AF2317F100544F8357A4
:1088B00047002318F100DC4AA1E797850100938562
:1088C000256E177501001305A55697600100E78016
:1088D00080A8178501001305E56E97600100E78009
:1088E00080A7294597600100E780C0AB134544008D
:1088F0008320C110032481108324411051618280A0
:1089000097B7FF1F83C737AA2555D9C3FD1717B6D9
:10891000FF1FA30AF6A803D6060183470701CC462A
:108920000A85230BF10097300000E780A0DC97D781
:10893000FF1F9387E71A9C4317B7FF1F130747A62C
:10894000978601009386066B88430A866C00971011
:108950000000E780A01DAA8451D997850100938566
:108960002564177501001305A54C97600100E78089
:10897000809EA68517850100130585659760010017
:10898000E780609D294597600100E780A0A12685CA
:1089900097000000E78000BB91BF93F725009DC7BB
:1089A000B7E70400BC474146814528088297255512
:1089B00097000000E78000B928089305F00F9700A2
:1089C0000000E78040D3134524001DB793F715003E
:1089D000014599DF97000000E780209913451400B6
:1089E00001BF5C4D411106C688C317D7FF1F23295D
:1089F000F70EB7E7040083A7070817050000130563
:108A0000E5E38297B24097D7FF1F238DA70C01455E
:108A10004101828001119307700F2316F10006CEE9
:108A200097D7FF1F83C7970D8DE7B7E7040083A78C
:108A3000870D17B6FF1F0346E69B6C0017D5FF1F77
:108A40000355050C82973335A00097D7FF1FA387E6
:108A5000A70AF2400561828041119397050122C463
:108A600006C626C2C1872E8463D40702B7E4040079
:108A7000FC5417B5FF1F0345E597829719C1BC54F5
:108A800082972165218DB240224492444101828027
:108A900093F715008DC7B7E7040083A7471A17B6E9
:108AA000FF1F1306269497D5FF1F9385650417B5FE
:108AB000FF1F03452594829713451400E9B793F7E8
:108AC000250099CFB7E70400BC4F13060064894521
:108AD00017B5FF1F0345059282971345240065B71C
:108AE00093F785009DC7B7E7040003A8871A13070B
:108AF000401F97B7FF1F83C7E78F814613064006C5
:108B0000994517D5FF1F0355A5FF0298134584000B
:108B10009DBF93F745000145BDD7B7E4040083A787
:108B2000041817D5FF1F0355A5FD8297BC4C1306EB
:108B30000064914517B5FF1F0345C58B8297134508
:108B4000440091B797D7FF1F83D787FB6398A7028D
:108B500017D7FF1F2317B7FA17D7FF1F2314C7FA1A
:108B600017D7FF1F2311D7FA2E861785010013058B
:108B70002568BE85175301006700E37D1785010056
:108B800013058568176301006700C3940357450008
:108B9000011106CE22CC97D7FF1F83D767F6178522
:108BA0000100130565666310F706C167F91717D74B
:108BB000FF1F2327F7F437E4040097D7FF1F23A3F1
:108BC00007F47C4C894517B5FF1F0345A5828297A2
:108BD0007C4C914517B5FF1F0345C581829797B718
:108BE000FF1F83C7376085CB8547A307F100832725
:108BF00044171306F10085451305503082971785F9
:108C000001001305A55497600100E780A08CF24095
:108C100062440561828097D7FF1F83C7E79C178551
:108C2000010013056557E5F38547A307F100832786
:108C300044171306F10085451305503082971785B8
:108C400001001305E552C1B77D15954763E0A71CE8
:108C5000178701001307474C0A053A951C4101117B
:108C600022CC06CE26CABA972E84828717850100A9
:108C70001305055A97600100E780C0851DAA03C748
:108C8000250099476311F7022E8597000000E780C1
:108C900020F083456400178501001305655897503F
:108CA0000100E780406B97B7FF1F238D07521785A0
:108CB00001001305A5587DBF03C72500954763191B
:108CC000F702C16717D7FF1F035787E3F91703D5CB
:108CD000A5006309F702B7E7040083A7C7178297C7
:108CE000178501001305855697500100E780807EA7
:108CF000854717B7FF1F2307F74E17850100130598
:108D000065578DBF97D7FF1F239CA7DE83D7E5004C
:108D1000B7E40400096617D7FF1F2314F7DE83D7D3
:108D200005011306069017A5FF1F0345A56C17D76D
:108D3000FF1F2319F7DC83D72501A14517D7FF1F94
:108D40002313F7DCBC4C8297BC4C1306006491459E
:108D500017A5FF1F0345056A82970356E400835554
:108D6000A400178501001305A54F97500100E78067
:108D7000805EBDBF1785010013058550E5BD83C525
:108D800025009147639CF50285471785010013056F
:108D9000A550A307F10097500100E780A073B7E743
:108DA000040083A747171306F100854513055030CB
:108DB0008297F2406244D24405618280994763926F
:108DC000F502228597000000E78080DC834564007F
:108DD000178501001305C54497500100E780A0578F
:108DE000C9BF9547639FF5008347140017850100AD
:108DF0001305854AE39007E8178501001305854BA5
:108E000095BD178501001305654BF9B782806D711B
:108E1000232481102326111023229110328401CDA6
:108E20008947630AF5028320C1100324811083243B
:108E3000411051618280178501001305E548AE8419
:108E400097500100E7800069A285268597C0FFFF43
:108E5000E7804066C9BFB7E70400FC472800829757
:108E6000178501001305054797500100E7808066CC
:108E70008347810039C41307000B6380E70213871F
:108E8000A7051377F70F8D4663EDE602A28528004C
:108E900097D0FFFFE78020D579B78547E3F587F8BE
:108EA00083459100177501001305C52DB335B0003A
:108EB00097B7FF1F238AB71A97500100E780A04990
:108EC0009DB703479100A207D98F35671307D75580
:108ED0006385E7086368F7022D671307B755638753
:108EE000E70631671307C755638AE7042967130745
:108EF000A7556394E702A285280097D0FFFFE7807B
:108F0000600815B739679306E765638DD70663E98F
:108F1000F6001307E7556380E706A28528003DB7F2
:108F20003D679306F7556386D7061307F766E39602
:108F3000E7FE97D0FFFFE780E020F5B50146A28568
:108F4000280097D0FFFFE78020F1F1BDA28528001F
:108F500097D0FFFFE7804001F9B58947E3F587EC3B
:108F60009305E4FFC205C1811305A10097A0FFFF8F
:108F7000E780C0114DBDA285280097D0FFFFE78094
:108F8000600155B5A285280097D0FFFFE780200C2F
:108F900059BD97D0FFFFE780A01471B5411122C4DD
:108FA00017A4FF1F13044446AA8617860100130660
:108FB00026182285C14506C697500100E780C05299
:108FC0000357440097A7FF1F938707452393E700A4
:108FD000035764002394E700B24022444101828099
:108FE000011106CE22CC97000000E78060FB37E439
:108FF00004008327841417A6FF1F1306E640D545F7
:1090000001458297832784179305F100130550309B
:1090100082978347F100A1C7A30701008327441764
:109020001306F100854513055030829783274417B6
:1090300017A6FF1F1306463ECD45130570308297D5
:109040008547A307F100832744171306F1008545E0
:10905000130550308297F240624405618280832775
:10906000441717A6FF1F1306263BCD451305703086
:10907000D5B761712324811A37E4040083270408DB
:109080002326111A2322911A2320211B232E311962
:10909000170500001305859C829717A9FF1F130968
:1090A0006935994785442300A900231CF100978561
:1090B00001009385E510930740061775010013051D
:1090C00025D7231CF1082308910097C9FF1F938916
:1090D000096297500100E780002883D509001785B1
:1090E00001001305A50597500100E780C02629451A
:1090F00097500100E780002B03D509008569970090
:109100000000E780E0E98327441710088545130530
:10911000503082978327441717A6FF1F1306C62FC8
:10912000CD451305703082978327441717A6FF1F7C
:109130001306862CB54513056030829783274417A4
:109140003008894513051031829783274417300969
:10915000894513052031829783274415938509C8D3
:109160000D45829783274415938509C81145829739
:10917000A3059100230691002308910002CD230C42
:1091800001008327841630099145130570408297AA
:10919000832784161306B100854513050040829786
:1091A0008327841670008545130510408297832716
:1091B000841630088545130520408297832784163E
:1091C00010088545130550408297832704157D5567
:1091D0008297832744137D5582977D5597A0FFFF83
:1091E000E78080358327440C829797A0FFFFE780B4
:1091F000C0108327841417A6FF1F1306E620D54549
:109200000145829789471306700F81452809230677
:10921000F1009790FFFFE78040EC8D4713060008B0
:1092200081452808230CF1089790FFFFE780E0EACA
:109230009147230CF100977701009387E7B098439B
:1092400083C747003AC8230AF10097D0FFFFE780A1
:1092500020F670008545054597A0FFFFE780E034C4
:1092600030099305700F094597A0FFFFE780E033B1
:109270003008930500080D4597A0FFFFE780E03216
:1092800010089545114597A0FFFFE7800032C167A0
:1092900017D7FF1F1307C786F9171CC32322070020
:1092A00017A5FF1F1305C51497A0FFFFE780C02E69
:1092B0008327C41D17D5FF1F1305058382973C48DC
:1092C00003450900854582978320C11A0324811A2A
:1092D0008324411A0329011A8329C1195D618280FF
:1092E000C16717D8FF1F0358A881F9176301F80851
:1092F0003DCDB5CD011126CAB7E4040083A7841281
:1093000022CC2E862315B10006CE2A840147814641
:10931000ED45428582972AC611ED17850100130598
:1093200025EB97500100E780E01AF2406244D244F6
:1093300005618280FC440356A100A28582972C001F
:1093400017C5FF1F0355C57B97A0FFFFE78080313E
:1093500069DD178501001305E5E897500100E780F6
:10936000601783A7C412ED45280082977DBF8280D5
:10937000011106CE22CC2DC9854717A7FF1FA302D6
:10938000F70897A7FF1F238F070637E404008327FA
:1093900084179305F1001305503082978347F1003D
:1093A000A9CBA3070100832744171306F1008545C5
:1093B0001305503082978327441717A6FF1F130603
:1093C000A603B5451305603082978547A307F100D2
:1093D000832744171306F100854513055030829703
:1093E000F24062440561828097A7FF1FA38B0700AC
:1093F00049BF8327441717A6FF1F1306E6FFB5458D
:1094000013056030E9BFC16717C5FF1F0355456FDE
:10941000F9176307F500B7E7040003A3C717028332
:10942000828001118547A307010017C7FF1F23078B
:10943000F76CB7E7040083A7471706CE1306F100C1
:109440008545130550308297F2400561828017935D
:10945000FFFFE702E3C32A8408452E89B28919C9B0
:1094600000C1971500009385A5866105973001001E
:10947000E780800181447D5A97100000E780E03941
:1094800063C7A404814497100000E780003A63C8D2
:10949000A40497C7FF1F938727679C43DC47B30744
:1094A000F94091872302F400638309048327C900EC
:1094B000B307F4409587A302F4001C4C89C79C476E
:1094C00099C3228582971793FFFF6700A3BF5C446F
:1094D000139714008504BA972390470171BF1C4865
:1094E000139714008504BA972390070069BF832758
:1094F00089000547B307F4409587A302F40083571A
:109500000400638EE7028DC309476384E7040D47B7
:10951000E395E7FA978701009387872E1CCC9787FE
:1095200001009387E72E11A8978701009387C7F45E
:109530001CCC97870100938727F55CC8BDBF978730
:109540000100938767E01CCC978701009387C7E0F1
:10955000EDB7978701009387672F1CCC9787010091
:109560009387C72FD9BF95E51793FFFFE702E3B3B2
:10957000004618448347940075839D8B6317F7005A
:1095800097100000E78060B448C41793FFFF67009E
:1095900003B482801793FFFFE70283AF138935007E
:1095A000C16442094111AA890144F1141359090106
:1095B000054A2EC697100000E7802026B245634872
:1095C000A400014541011793FFFF6700A3AF83A7E4
:1095D000090013171400BA9783D707006388B700F0
:1095E0006394970063742A010504E1B70545D9BF68
:1095F0001793FFFFE702E3A8AA892E89328BB6846E
:109600003A8ABE8A97A00000E78020FB71C92685B0
:1096100097200000E78020098D4763E7A7007D556C
:109620001793FFFF670063A983DB440097100000D6
:10963000E780A0242A8497100000E7804025930744
:10964000740031443305850263CDA70297100000F2
:10965000E780A02297100000E78020222A8497103C
:109660000000E780C022930774003144330585026F
:1096700063C3A70497100000E780202093074500EC
:1096800029A897100000E780802033058502130782
:10969000F0179307C017E35FA7FA2D55E3C277F9D8
:1096A00063040B02D6865286A6854A859720010060
:1096B000E78020BAB5B797100000E780401D33055A
:1096C00085029307C5FFD1BF832749001385C900D1
:1096D00083D5270097000000E78000EC61F581B793
:1096E00069553DBF97C7FF1F2392A74297C7FF1F2A
:1096F00093878741904381470C463307F500420723
:1097000041836393B70082805446139847008507CE
:10971000C2962390E600D5B797C7FF1F9387C73E31
:109720009C4303C58700828017C5FF1F0355053E74
:1097300082801793FFFFE7024397C1671387D7FF24
:10974000630BE502636AA700F1176300F5020145A8
:109750001793FFFF6700A3971387E7FF6302E502F4
:10976000FD171D8D13351500E5B797500000E780F4
:10977000C0267D15C5BF97500000E78040FBD5BFD0
:1097800097500000E78060F9EDB71793FFFFE702FD
:10979000C3914111AA8401442EC697100000E780AE
:1097A000C008B2456348A400014541011793FFFF7B
:1097B0006700E3919C48131514003E9583570500FC
:1097C000E385B7FE0504C9BF03485500814693F7FA
:1097D000F60F63E5070181473E85828058459397E0
:1097E0005600BA9703D727006316B70003D70700C0
:1097F000E304C7FE8506E1BF834645000147937732
:10980000F70F63E4D700814711A81C4513165700D2
:109810000507B29703D60700E313B6FE3E858280A4
:109820001793FFFFE702C38693170501C18797CA05
:10983000FF1F938A6A2D635BF00883A70A00C04765
:109840009C4703570400198D420541816368F50068
:10985000014422851793FFFF6700C38612052A94EF
:10986000CDBFDC4713944900014A3E94834744002E
:109870006341FA02014A834754006349FA028509A9
:10988000C20993D9090183A70A009847E3EBE9FCD1
:10989000C1B71C4413195A00A6853E994A85970002
:1098A0000000E780C0EE05E1050AC9B75C44131962
:1098B0005A00A6853E994A8597000000E78020ED72
:1098C00019E1050A4DBFE30C09FA61B7AA84814981
:1098D0005DBF1783FFFFE702437D1C452A8481E7B4
:1098E0009307C5001CC51C44231204001CC0930729
:1098F000F00F63EDB70093F5F50F22859720000078
:10990000E78020E21783FFFF6700637C93940501E3
:10991000C167C18063F9F500A68522859720000004
:10992000E78040E5C5B7C18193F5F50F2285972003
:109930000000E78000DFA685228597200000E780F1
:1099400040E0C9B797C7FF1F9387071C88438280F1
:109950001C4599C797C7FF1F23A8A71A01458280F6
:109960007D55828097C7FF1F9387071A98438347C7
:109970004500484792073E9582801783FFFFE70224
:10998000C372617100451C183EC6B70780013EC80E
:109990001C183ECA8357440002CE02D002CC231EBC
:1099A000F100834784002A8902D22301F1023C0896
:1099B0003ED402D697000000E78000FB83570500E5
:1099C0002316F10297500000E78060C42307A1022C
:1099D0005C4003556400F18313F717008347F102DD
:1099E00052055181F99BD98FA307F102971001000D
:1099F000E780807539CDAA840355050097A0000043
:109A0000E78080BC83D704002AD26800231CF100C1
:109A100083D72400231DF1001C4803D647008C4344
:109A200097200000E78000CD8347B400CA861786E0
:109A300001001306E68A8117A305F4006C004810A4
:109A400097200100E780E0805D611783FFFF6700DA
:109A500003682155D5BF1C45B1CF03C5A700894672
:109A600013576500630BD7028D46630ED7028546F8
:109A70006300D702130740063305E50203C7B700AA
:109A8000418B15CB83C7B700BD8B3355F540828022
:109A90001375F5031307803EC5B709671375F50302
:109AA00013070771D1BF372709001375F503130793
:109AB000077CD9B7014582801783FFFFE702E35E89
:109AC00003A98500630C09048347B900AE8493F7AA
:109AD000070E85C303459900930520030D810505F5
:109AE000B305B5028844610597300100E780E0A91D
:109AF00035A02E8597000000E78020F62A8419CD36
:109B000097000000E780605C8325C900B307B5407B
:109B100063FA87002E94B305A440E9F51783FFFF8D
:109B20006700E35A85457DBF1783FFFFE702E357D0
:109B30002A8403D50500011132C636C43AC22EC0AC
:109B400002CA02CC02CE97A00000E780E0A78245BF
:109B50002ACA22852ECC97000000E780E0E0035758
:109B60000500231EE10097500000E78040AAA246AE
:109B700032469247230FA10036874C08B2862285D1
:109B8000014697000000E780E0A605611783FFFF0C
:109B90006700E3531783FFFFE702235161711C182D
:109BA0003EC6B70780013EC81C183ECA3C080045A7
:109BB0003ED4AA8402CC02CE02D002D202D69700B2
:109BC0000000E78060DA8357050035592316F1025B
:109BD00097500000E780A0A32307A10209C4835780
:109BE000440081EB21594A855D611783FFFF6700BF
:109BF000034E035564005205518197100100E78020
:109C0000A0542A8965D18347B40093F7070E99C7FA
:109C10001305840197300100E78060998357440061
:109C2000231EF100834784002301F1025C400355A9
:109C30000900D98313F7070883471102231CA100E9
:109C400093F7F707D98FA300F10283572900231D4B
:109C5000F1005C40F18313F717008347F102F99B91
:109C6000D98FA307F10297A00000E780E0952AD2E0
:109C700035D9834794006800139757008347B40091
:109C8000FD8BD98FA305F4001C4803D647008C43F5
:109C900097200000E78000A6A6871777010013072A
:109CA0002764740005464C10268597000000E78065
:109CB00060942A890DD98347B400A685FD8BA3053E
:109CC000F40097000000E78060DF31BF1783FFFFDB
:109CD000E702A33D832485FE2A844111268597004F
:109CE0000000E78080D7834734FF93F7070E8DCBC2
:109CF0002AC6268597000000E78060C809CD834703
:109D000034FFB245FD8BA309F4FE91C5228597303F
:109D10000100E780808741011783FFFF6700233B35
:109D20007DD98327C4FF2685829775F5834734FF45
:109D300093F7070E91C7228597300100E7802087AF
:109D4000032584FE97000000E78000E5E9B717834C
:109D5000FFFFE70283329C4141112A8903C70700B4
:109D600089472E84935667006380F6040D46638806
:109D7000C6049307F0076304F7022E8597200000BE
:109D8000E780C0A7AA848149C16B130C490097C71B
:109D9000FF1F938767D79C43984763E4E904410119
:109DA0001783FFFF6700233103D745008547E3F89A
:109DB000E7FE2E8597200000E780A0A9E1B703D732
:109DC0004500E3FEE7FC2E8597200000E78000A316
:109DD000AA84228597200000E78060A4C204C98C71
:109DE0005DB7DC470355A900139A49003E9A9317C3
:109DF0000501C187635DF00083570A006397A702DE
:109E000063E774038327CA00034D5A002DA0A1679E
:109E10002167A98F1307F7EFE374F7FE6397090033
:109E200097000000E780209161FD85098DB78327A9
:109E30008A00034D4A00835DA90003576900216A27
:109E4000138BC7003AC6814A33CA4D01631E5D01B8
:109E500097C7FF1F9387C7CB9C43E1DBA28662862F
:109E6000814526858297D1B7A1679387F7EF930C39
:109E70004BFF63F24703B2455A8597F0FFFFE78037
:109E8000A0710DC103278B00104709CE10436382D8
:109E9000C4023107D5BFEE85668597000000E780D4
:109EA000008F71F993861A0093FAF60F130B0B02C9
:109EB00071BF835644005C43E3E9F6F622853AC657
:109EC00097100000E780807DA1679387D7042A8AD6
:109ED000035D4400324763E897008347D90093E766
:109EE00007F8A306F9001C4766852286E28582975B
:109EF000C1670844FD17337AFA00529508C023124F
:109F0000A40125B797C7FF1F938707C098438147D0
:109F100015C31447814763FFD500939745004C470D
:109F2000BE9519C903C7550081476375E600DC4536
:109F30001606B2973E85828003C745008147E37BC2
:109F4000E6FE16069C45F5B71783FFFFE7024314AC
:109F5000AA892E8A814497CAFF1F938AEABA83A7E7
:109F60000A00984763E6E4001783FFFF6700831544
:109F7000DC471394440001493E9413BB140083470B
:109F80004400634BF900014913BB1400834754009C
:109F9000634FF9008504E1B70844931759005287CD
:109FA000DA860146A2853E9582990509C9BF4844D3
:109FB000931759005287DA860546A2853E95829905
:109FC0000509E9B71783FFFFE702230E814517F55F
:109FD000FFFF1305054897C7FF1F239907B2970096
:109FE0000000E780A0F61783FFFF6700430E97C7C6
:109FF000FF1F938767B19C4395C31783FFFFE70259
:10A00000C30A814517F5FFFF1305A544970000001B
:10A01000E780C0F31783FFFF6700630B828017831D
:10A02000FFFFE702E30637E40400832784124111AF
:10A030002315E100AE893289368A3A868146014786
:10A04000ED45AA8482972AC621C90356A100D2856C
:10A0500097400100E780C0248327C413CE8526855E
:10A060008297058905C98327440D231421010146E0
:10A070002C00268582972A8401C9B7E7040083A7AC
:10A08000C712ED4528008297228541011783FFFF03
:10A09000670043034944D5B76554FDB75C41FD17DC
:10A0A0005CC182801783FFFFE7022300B7E704004B
:10A0B000FC5F829795473305F50281450D81178333
:10A0C000FFFF6700C3001783FFFFE70203FEB7E748
:10A0D0000400FC5F829795473305F5020D811783D5
:10A0E000FFFF6700C3FE1783FFFFE70203FCB7E72C
:10A0F000040083A7870B0355050082971783FFFF92
:10A100006700E3FC1783FFFFE70223FA035505000E
:10A110003287AE861796FF1F0356263697C5FF1F58
:10A120009385459F97000000E780A0EF1783FFFF0E
:10A130006700E3F91783FFFFE70223F7B7E704009F
:10A1400083A7C71782971783FFFF670043F817831A
:10A15000FFFFE70283F5B7E7040083A7871397C5DE
:10A16000FF1F9385259B829701451783FFFF67009B
:10A1700003F61783FFFFE70243F3B7E7040083A763
:10A18000C71F81451795FF1F0355252B82971783FE
:10A19000FFFF6700C3F31783FFFFE70203F1B7E791
:10A1A000040083A7871397C5FF1F9385A597829700
:10A1B00001451783FFFF670083F11783FFFFE70265
:10A1C000C3EEB7E7040083A7C71F81451795FF1F9C
:10A1D0000355A52C82971783FFFF670043EF178372
:10A1E000FFFFE70283EC2E8597800000E780E0AF59
:10A1F00097800000E780E0EC1783FFFF670023ED06
:10A200001783FFFFE70263EA97800000E780E0F62C
:10A210001783FFFF6700A3EB5C49E1175CC95CC5CE
:10A2200083572501A1072319F50083570501A107CD
:10A230002318F5008280F1473305F50297C7FF1F09
:10A24000938747909C433E9582808D476315F6081F
:10A2500003D74600854763F0E7081783FFFFE7024F
:10A26000C3E4368536842E8997100000E7800059B4
:10A2700029C98357440093140501C18063E39704FF
:10A28000228597100000E7806057FD142312940088
:10A290009307A0026300F5029307B0026307F5027B
:10A2A00093079002631FF500228597000100E78065
:10A2B000C08501A80146CA85228597A00000E780D5
:10A2C00060B01783FFFF670083E0228597100000CE
:10A2D000E780C003FDB7828097C6FF1F9386C686BE
:10A2E0009C42014599CF9843D44217C6FF1F232DA6
:10A2F000E6846396D70097C6FF1F23A9E6841385DB
:10A30000C7FE82801783FFFFE70223DA9700000071
:10A31000E780A04B7144330585029145979000007A
:10A32000E78020E911E565551783FFFF670023DA11
:10A3300097C7FF1F23A6A78097000000E780E0488B
:10A3400033058502914597900000E78080E661DD46
:10A3500097B7FF1F23A8A77E97000000E780E0467D
:10A3600097B7FF1F2398A77C97000000E780E04580
:10A3700097B7FF1F2391A77C97770100938787FBEF
:10A3800017B7FF1F232CF77A97070000938707E979
:10A3900017B7FF1F2322F77A014579B71783FFFF0D
:10A3A000E702A3D0AA8517B5FF1F1305A57897105C
:10A3B0000000E780C05B1783FFFF670043D117836E
:10A3C000FFFFE70283CE97000000E78060FD971053
:10A3D0000000E780405B97B7FF1F9387E7769C43B9
:10A3E00091CF1387C7FE19CB83D5C7FF17B5FF1FC2
:10A3F0001305057697200100E78020191783FFFFDA
:10A400006700E3CC1783FFFFE70223CA9700000031
:10A41000E780C0EC09CD834785002A8493F70704C1
:10A4200099EB0355E50097000000E78080F917835A
:10A43000FFFF6700C3C98347C5009304450117B9EF
:10A44000FF1F1309697085E3832709005CC997B76B
:10A45000FF1F23AB976E83274900F1FB97B7FF1FC0
:10A4600023A6976EE9B7FD172306F50061059780CF
:10A470000000E780C0D68307840063CB07048347CE
:10A48000840093E707F82304F400B7E704009C5F17
:10A4900082974205A94741813375F50283478400BD
:10A4A00093F707FCC98F2304F4008347D4003E953B
:10A4B0001C402318A40089CF984319CB8347C400BC
:10A4C0005040814585073305F502420541810297D9
:10A4D000832709005CC897B7FF1F23A797668327C8
:10A4E000490089E797B7FF1F23A297668347C400F7
:10A4F0009DDF8355040117B5FF1F13056565972080
:10A500000100E780800825B71783FFFFE702E3B962
:10A5100097C7FF1F938707899C4701448583858BD5
:10A5200085E3AE84B2853A8697100000E780804BC1
:10A530002A8419C597100000E780C041829408CC96
:10A5400022851783FFFF670083B81783FFFFE702A9
:10A5500023B441112E8932C6AA8997000000E780F2
:10A56000C031324713060502CA869705000093855D
:10A57000C5CC17B5FF1F1305E55B97000000E7800A
:10A58000E0F82A8425C99304C50097000000E780FD
:10A59000E0411946AA85268597100000E7808015BE
:10A5A0008545268597100000E7806011177501002A
:10A5B000130505D64E9583450500268597100000A6
:10A5C000E78020165C4831468145A1075CC85CC421
:10A5D00083572401E1172319F40083570401E1177D
:10A5E0002318F4001C4C3E859780FFFFE780E0AE07
:10A5F000A3042501228541011783FFFF670083AC77
:10A600001783FFFFE70263AA4111AA842EC632C452
:10A6100097100000E7806036004DB2452246834720
:10A6200084000CC050C093F7F70393E7070423049A
:10A63000F40023180400268597100000E78080317D
:10A6400083479400A9462317A40013D737000507B2
:10A650003307D7029D8B85072306F400A306E40089
:10A6600083C70401D8488507230FF7FE17B7FF1FDC
:10A670001307874D5843232A04009307440129E315
:10A6800017B7FF1F2324F74C17B7FF1F232EF74AD6
:10A6900017B4FF1F1304C44B228597200100E780E5
:10A6A00000E11C44858B5D8D19E58145228597204D
:10A6B0000100E78080ED41011783FFFF670023A1C0
:10A6C0001CC317B7FF1F2323F748D9B71783FFFF12
:10A6D000E702A39D97050000938565B701459700A4
:10A6E0000000E78000B001451783FFFF6700239E4D
:10A6F0001783FFFFE702639B97000000E78080B0AD
:10A700001783FFFF6700A39C8347C500A5E317835A
:10A71000FFFFE70283992A840355E50097000000B4
:10A72000E78000C821C18347840093F7F7FB230427
:10A73000F4001C4091C7DC4381C74C40014582971F
:10A7400097000000E78080B917B5FF1F130545404B
:10A7500097200100E780A0E50355E4009700000082
:10A76000E78020C61783FFFF670063968280178308
:10A77000FFFFE702839397B7FF1F9387E73C970597
:10A780000000938565C817B5FF1F1305653C23A01E
:10A79000070023A2070097200100E780E0CE17837F
:10A7A000FFFF6700C3921C4D91CFDC4381CF17831D
:10A7B000FFFFE702838F8345070082971783FFFF20
:10A7C0006700E390828097B7FF1F9387A73A9C4367
:10A7D00003C50700828097B7FF1F9387A7399C4363
:10A7E00003C51700828097B7FF1F9387A7389C4344
:10A7F00003C52700828097B7FF1F9387A7379C4325
:10A8000003C54700828097B7FF1F9387A7369C43F5
:10A8100003C53700828097B7FF1F9387A7359C43F6
:10A8200003C55700828097B7FF1F9387A7349C43C7
:10A8300003C56700828097B7FF1F9387A7339C43A8
:10A8400003C57700828097B7FF1F9387A7329C4389
:10A8500003C58700828097B7FF1F9387A7319C436A
:10A8600003C59700828097B7FF1F9387A7309C434B
:10A8700003C5A700828097B7FF1F9387A72F9C432C
:10A8800003C5B70011E11D45828097B7FF1F93876D
:10A89000672E9C4303C5C700828097B7FF1F93872D
:10A8A000672D9C4303C5D700828097B7FF1F93870E
:10A8B000672C9C4303C5E700828097B7FF1F9387EF
:10A8C000672B9C4303D50701828097B7FF1F9387AF
:10A8D000672A9C4303C52701828097B7FF1F938790
:10A8E00067299C4303D54701828097B7FF1F938751
:10A8F00067289C4303D56701828097B7FF1F938722
:10A9000067279C4303D58701828097B7FF1F9387F2
:10A9100067269C4303C5A701828097B7FF1F9387D3
:10A9200067259C4303C5B701828097B7FF1F9387B4
:10A9300067249C4303C5C701828097B7FF1F938795
:10A9400067239C4303C5D701828097B7FF1F938776
:10A9500067229C438857828097B7FF1F9387872180
:10A960009C4303D5C702828097B7FF1F9387872038
:10A970009C4303D5E70219E11305800C828097B749
:10A98000FF1F9387271F9C4303C50703828097B748
:10A99000FF1F9387271E9C43C85B828097B7FF1FCA
:10A9A0009387C71C8843828097B7FF1F9387471CF4
:10A9B0008843828019E17D558280F5DE984265DF0B
:10A9C000FDD917B7FF1F1307E73D1847AA87715531
:10A9D000058B631D072403C507001547E37DA7FC0E
:10A9E00003C737001305F0057D171377F70FE364EE
:10A9F000E5FC03C35700E30003FC83C86700E38C56
:10AA000008FA03C77700494579171377F70FE3640E
:10AA1000E5FA03C7A70011481305F7FF1375F50FF3
:10AA2000E36BA8F803CE97000D481305FEFF1375DE
:10AA3000F50FE362A8F803C8B700630908006518BA
:10AA40001378F80F1305600DE36705F703C5C7001A
:10AA5000794879151375F50FE36FA8F403C8D7008B
:10AA60000D457D181378F80FE36705F503D8070146
:10AA7000930E40175118420813580801E3ED0EF3E6
:10AA800003C8E7007D181378F80FE36605F303C8E1
:10AA900027017D181378F80FE36F05F103C88700CD
:10AAA000C54E75181378F80FE3E70EF103D8670168
:10AAB000856E938EBEE06D18420813580801E3ECD2
:10AAC0000EEF03D847016D18420813580801E3E45C
:10AAD0000EEF03D887017918420813580801E36C78
:10AAE00005ED03C8A7017D181378F80FE36505EDA0
:10AAF00003C5B7011D487D151375F50FE36DA8EA71
:10AB000003C5D701714879151375F50FE365A8EAF8
:10AB100003D5E7011308E00F7D1542054181E36C81
:10AB2000A8E803C50702494879151375F50FE364D2
:10AB3000A8E8C85301C937C834005915130858BFCD
:10AB4000E36BA8E603A8870237C53400130555BF99
:10AB50005918E36205E717B5FF1F232BC50003C68D
:10AB6000050117B5FF1F2327F5000545E375C5E46B
:10AB700003D82501D04933760603E31E06E203C657
:10AB80001501E30A06E217B6FF1F2321B6FE83C5AF
:10AB9000270001466387A50003C61700F145330669
:10ABA000B60283C707039305C00272971A071307FB
:10ABB000C70516031A9796084697B387B7024155FB
:10ABC0003E973297420741836362E8061773FFFF9F
:10ABD000E702A34D368597800000E780A0689700C4
:10ABE0000100E78020482A8497A00000E780805A6F
:10ABF0002A9497F00000E78060262A94979000003E
:10AC0000E780A0812A9497F0FFFFE780E06F2A9405
:10AC100097400000E78060932A9497700000E780D7
:10AC2000A09C22951773FFFF6700634A8280177309
:10AC3000FFFFE70283474111A307A10097A000008F
:10AC4000E780A0C59305F100170500001305E5B5E1
:10AC500097F0FFFFE780802F014541011773FFFF49
:10AC60006700E3461773FFFFE702A34117B4FF1F16
:10AC7000130444130328840079599368180097B487
:10AC8000FF1F23A514131378180063100802BA8459
:10AC9000BE89368B328A2E89AA8A97F0FFFFE78019
:10ACA000E0A77D15269519E531594A851773FFFFF1
:10ACB0006700A34097F0FFFFE78040A67D1526952B
:10ACC000A167E353F5FE97B7FF1F9387A744984307
:10ACD0003E8C814B01CB014597F00000E78020447A
:10ACE000933B15004A85DA865686D28597900000F8
:10ACF000E780C04D2A8911CD1C44F99B17B7FF1F6F
:10AD00002326F70A83270C00CDD3E3800BFA829722
:10AD100069BF268597B7FF1F23A8070897F0FFFF95
:10AD2000E780809C4146CE8517B5FF1F13050511AE
:10AD300097300100E780C05697D00000E780409927
:10AD40000325040B97D00000E780009D054597D0B0
:10AD50000000E78000A4054597000000E78060ED53
:10AD6000A9B797B7FF1F9387E7039C47858BEDC76C
:10AD70001773FFFFE702633317B5FF1F1305450A7B
:10AD800097B7FF1F23A0070297B7FF1F23AE070047
:10AD900097B7FF1F23AC070097200100E7802081B1
:10ADA00097500000E780E0F597100100E780A04C85
:10ADB00097100100E780A05297B7FF1F938707FD08
:10ADC0009C4391C7054597800000E780402097B7D6
:10ADD000FF1F938767E59C4399C741657D15977071
:10ADE0000000E78040A297F00000E780E03D97D0A8
:10ADF0000000E780808F97B7FF1F9387A70F9C43C2
:10AE0000139717016356070097F00000E78000AD25
:10AE100097B7FF1F23A4070297B7FF1F23A20702BC
:10AE200097B7FF1F23A0070297B7FF1F23AE0700A6
:10AE300097000000E780008C97000000E780007218
:10AE400097F0FFFFE780401897F00000E78040D6BA
:10AE50001773FFFF6700A327828097B7FF1F9387B1
:10AE600067F4884382801773FFFFE702032497800B
:10AE70000000E780607597800000E780C077177357
:10AE8000FFFF6700C3241773FFFFE70263202A84D4
:10AE90009304140201112E85B289A685214636C677
:10AEA0003A8997300100E780403D0DE9B246380805
:10AEB0002686CE851305940497500000E7806041F4
:10AEC00021462C084A8597300100E780003B133566
:10AED000150005611773FFFF6700C31E0145D5BF4D
:10AEE0001773FFFFE702631C9305450617B5FF1FA5
:10AEF000130585C897100100E78020691773FFFFCD
:10AF00006700E31C1773FFFFE702231A41112EC6E7
:10AF100097F0FFFFE780601BB24588C141011773BE
:10AF2000FFFF6700C31A1773FFFFE7026316AA84C7
:10AF30002E8497800000E780006CAA8985452285D1
:10AF400097000000E780E07D83C7E401138994083F
:10AF500099E313890403CE85228597000000E780DA
:10AF6000407C214693051902228597000000E78066
:10AF7000607897B7FF1F9387E7E28C43228597108D
:10AF80000000E780C08221469385840222859700D5
:10AF90000000E78020761773FFFF6700A312177386
:10AFA000FFFFE702030E397197F00000E780E0B47D
:10AFB0009305400661E997800000E7800060630226
:10AFC000051497B7FF1F83C7E7BC13B7170097B6E1
:10AFD000FF1F2381E6BC014499CFC16417B9FF1F4D
:10AFE000130949DC9309400EFD1497000000E78027
:10AFF000C0866342A40A97F0FFFFE780000D416915
:10B00000B7290900096AFD7A2A8B81447D19938941
:10B01000F97B130A0A71938A8AC797000000E780B8
:10B02000C08363D7A4041304400EB387840217B708
:10B03000FF1F130727D70324070B3E948357C40130
:10B040006382270B18403307EB4063EAE90083472C
:10B0500044008507B3874703D6976365F708014621
:10B060008145094597F0FFFFE780604EAA8B29E5EF
:10B0700097400000E780808385476317F506896560
:10B080009385057117B5FF1F130505AF97100100D4
:10B09000E780A04F95A0B30734030327090BBA97A5
:10B0A00003D7C7016308970003C75700A3820700AF
:10B0B0002382E700050415BF9305C500228597008C
:10B0C0000000E78080E65E85228697650100938513
:10B0D000652597F0FFFFE780E0525E85971000003E
:10B0E000E780608A850415BF97B7FF1F938787CBDA
:10B0F0009C478D83858BC1F721611773FFFF670024
:10B10000C3FB01468545094502D002D202D402D6CE
:10B1100097F0FFFFE780A043AA8479DD97F0000055
:10B12000E780E09C1389C4002A8481454A85970002
:10B130000000E780005F0C4041464A859700000010
:10B14000E780405B832944006385090C4E8502D863
:10B1500002DA02DC02DE97300100E78060402ACE8E
:10B16000141005462C0808184ECC97500000E780B4
:10B17000E00A1375F50F51ED8355840093E5250022
:10B180004A8597000000E780E05E11460C104A8572
:10B1900097000000E78000560146976501009385FF
:10B1A000E518268597F0FFFFE780C04526859700C4
:10B1B0000000E780407D5C40A1D3014685450D45F8
:10B1C00097F0FFFFE780A038AA841DD54840138977
:10B1D000C40097300100E780A0382AC64A8597004E
:10B1E0000000E780404C3246636FC5004C404A8502
:10B1F00097000000E780005001468145268597F0C2
:10B20000FFFFE7802040268597000000E780A077B9
:10B21000E5B583558400ADB71773FFFFE702E3E898
:10B2200097B7FF1F938707B89C471DC193E7870017
:10B2300017B5FF1F1305459417B7FF1F2328F7B64F
:10B2400097100100E78040321773FFFF670023E883
:10B25000DD9B17B7FF1F232BF7B497300000E78063
:10B26000E0647DF117B5FF1F1305059197100100EC
:10B27000E780E033D1BF1773FFFFE70283E0416946
:10B28000AA892E8AB28A368BBA8B814417BCFF1FDB
:10B29000130C4CB1930C400E7D1997F0FFFFE78023
:10B2A000C05B63C4A40001443DA03384940383279E
:10B2B0000C0B3E948357C401638627055A87D686B4
:10B2C0005286CE851305040397000000E780E0BB9B
:10B2D00001C923800B0022851773FFFF6700E3DDA0
:10B2E0008347F40185C35A87D6865286CE851305D7
:10B2F000940897000000E78040B909C5854723807E
:10B30000FB00D1BF850451BF835745006380071EF2
:10B310001773FFFFE702C3D701112A8497000000CB
:10B32000E780C04D09C985476309F50605611773B4
:10B33000FFFF670023D997E00000E780007C7DF5E0
:10B34000835744004947ED9BE392E7FEC1452285C0
:10B3500097000000E7804033AA8422859700000010
:10B36000E780204F0357440002CE91472A89631A91
:10B37000F700228597000000E780A0513C082ACC06
:10B380003ECE97E00000E78080765C55C5D3740818
:10B390004A86A6850545829751BF03574400D14789
:10B3A000E3F6E7F8032A0400C169014997BAFF1FD1
:10B3B000938A4A9F130B400EFD1997F0FFFFE78019
:10B3C000C049634FA90E2285032A0400970000009C
:10B3D000E780C042A1452A89228597000000E780C6
:10B3E000A02AAA84228597000000E780804A1440A2
:10B3F0002A86AA8978082685CA8597000000E780F2
:10B40000C0E7AA8405D503C7F40189476315F7008F
:10B410008347C10181DF5546D2851385640097308B
:10B420000100E780E0E7014597800000E780C01950
:10B4300001C583D7C401A5E797B7FF1F93878796F8
:10B440009C4793551900858913D73700058B01CF89
:10B450008983858B6399B70001452EC6970000004C
:10B46000E780C0DBB2454E8597800000E780601F13
:10B470000346C1012A849375190026859790000020
:10B48000E780E03935C1268597800000E780E01825
:10B49000268511C0014597800000E780004C973059
:10B4A0000000E780A0408547E312F5E883C7540019
:10B4B0001307F00FE38CE7E68507A382F400BDB520
:10B4C000B304690383A70A0BBE9483D7C401638BBB
:10B4D00037015546D2851385640097300100E78017
:10B4E000C0D955DD0509D1BD5DD86DB78280177310
:10B4F000FFFFE702E3B997800000E780000C05C179
:10B50000C164014417B9FF1F1309C9899309400E8B
:10B51000FD1497F0FFFFE7804034634EA40017A5A9
:10B52000FF1F1305656597100100E780E00317739F
:10B53000FFFF670023B9330534038327090B3E95CA
:10B540008357C50163889700231205009780000088
:10B55000E780A00C050475BF97B7FF1F938787840A
:10B560009C478D83858B8DE31773FFFFE702E3B361
:10B5700017A5FF1F1305456097100100E780200302
:10B580001773FFFF6700A3B482801773FFFFE70202
:10B59000C3B1970500009385C5A017A5FF1F13052C
:10B5A000A55D97100100E78020EE1773FFFF67008D
:10B5B00003B21773FFFFE70243AF8841B7E7040008
:10B5C000BC5B050542054181829709C5854723007B
:10B5D000F50005051773FFFF670063AF83C7F5FF2D
:10B5E0002E858507A38FF5FE828083C7F5FFFD17A3
:10B5F00093F7F70FA38FF5FE99EF1773FFFFE7029D
:10B60000C3AAB7E70400BC571385F5FF82971773E9
:10B61000FFFF6700C3AB82801C41035745008D8F3D
:10B62000BA951CC12312B5003E85828093D7850050
:10B63000A2051441DD8D835745001387E6FF18C12D
:10B6400089072312F50013D685004111238FB6FE1A
:10B65000A38FC6FE4101828018419307F7FF1CC1EA
:10B660008357450085072312F500A30FB7FE82809C
:10B67000835745008D8F2312F5001C41BE950CC1E8
:10B680002E858280AA8703D7470008410D8FAA958F
:10B690002392E7008CC38280184108453305A740F8
:10B6A000828083574500035765001D8F1C41084564
:10B6B0003385A7403305A74082801773FFFFE70259
:10B6C000C39E41112EC62A8497000000E780A0FD8A
:10B6D000B2456373B50001A0835744000840BE958E
:10B6E0002312B4003E9541011773FFFF6700239EAC
:10B6F0001773FFFFE702639B41112E84B28532C6A8
:10B7000097000000E780A0FB3246A2859730010039
:10B71000E78000B941011773FFFF6700439B177370
:10B72000FFFFE70283982E84854597000000E7809D
:10B7300000F9230085001773FFFF67004399177313
:10B74000FFFFE702839641112317B1008945970057
:10B750000000E780C0F68347E1002300F50083473F
:10B76000F100A300F50041011773FFFF6700239666
:10B770001773FFFFE702639393D78500A20541117A
:10B78000DD8D2317B100894597000000E78020F385
:10B790008347E1002300F5008347F100A300F50093
:10B7A00041011773FFFF670083921773FFFFE702E2
:10B7B000C38F1397850193D78501C166938606F0E1
:10B7C000D98F13D78500758FD98FA2053707FF0052
:10B7D000F98D4111DD8D2EC6914597000000E7805F
:10B7E00000EE6C00114697300100E78060AB41012C
:10B7F0001773FFFF6700A38D1773FFFFE702E38A4C
:10B800001C41854503C4070097000000E78080E6DF
:10B8100022851773FFFF6700838B1773FFFFE70213
:10B82000C3881C414111894503C7070083C717001E
:10B830002307E100A307F10097000000E78080E301
:10B840000355E10041011773FFFF67004388177339
:10B85000FFFFE70283851C414111894503C70700AB
:10B8600083C717002307E100A307F100970000003A
:10B87000E78040E08357E100410113D58700A2072C
:10B880005D8D420541811773FFFF67004384177385
:10B89000FFFFE70283810C4141112A8411466800B1
:10B8A00097300100E780C09F9145228597000000F6
:10B8B000E78040DCB247C166938606F013978701A4
:10B8C00013D58701598D13D78700758F598DA2071E
:10B8D0003707FF00F98F5D8D41011763FFFF670098
:10B8E000037F1C45BE950CC18280AE87944391E6D0
:10B8F000584101EF0CC15CC1828003C75700136738
:10B900001700A382E700B687D5B70CC3EDB7AA87A7
:10B91000084119CD1841D44398C36313D500D8C347
:10B920002A87034657009376160081E623200700F6
:10B930008280944381CA8C4203A847008CC36393DE
:10B940000601CCC3799A14C3A302C7003687D1BFBE
:10B950001C45DC471D8DB777DBB6938777DB098500
:10B960003305F502420541818280F147B385F50236
:10B9700048452E9582808347450085072302F500C0
:10B9800082801763FFFFE70243722A8409E417638A
:10B99000FFFF6700C37383474400F5DBFD1793F790
:10B9A000F70F2302F400E5F71C4403D7270005072F
:10B9B0002391E700DC4399C3228582974C4889CDC7
:10B9C00083475400898B99E71C4422859C479C43FC
:10B9D0009C478297232A04000040232004007DB75F
:10B9E0001763FFFFE702636C8357250041112EC6E2
:10B9F00081EB0144228541011763FFFF6700236D3E
:10BA0000035705008147F146E305F7FEB385D702EA
:10BA1000404585072E948345440008C4F5F5B24798
:10BA2000AA8481E7232A040009A81C456C0022850A
:10BA30009C439C43829748C84DDD85472312F40000
:10BA4000B24723200400231804002319F4005C48A3
:10BA50005CC483D72400FD172391F40061BF1763F2
:10BA6000FFFFE702836497A7FF1F9387E7128843CE
:10BA70002326050023240500410597100100E780D7
:10BA800000B31763FFFF670083641763FFFFE702DC
:10BA9000C36117A4FF1F130424101C40411199CF48
:10BAA0009C472300B5002AC65CC197000000E780D0
:10BAB00040FB1C40DC4399C3324582974101176328
:10BAC000FFFF6700C3600347450029E3584DAA877D
:10BAD0007D551DCF1763FFFFE702235D1CC3DC47C5
:10BAE00097A6FF1F23AAE60AF15613050701239024
:10BAF000D700970500009385050297100100E780A5
:10BB0000A09801451763FFFF6700635C7D55828045
:10BB100082801763FFFFE7024359011161468145A7
:10BB200028009760FFFFE780405B97A7FF1F938780
:10BB3000A7069C4328009305F00FDC473EC69700FC
:10BB40000000E780C0F405611763FFFF670023581A
:10BB500097A7FF1F938747049C43D847A167938704
:10BB6000C702631EF70A397106DE22DC26DA80007E
:10BB70004AD84ED652D456D23285B28497000000AD
:10BB8000E780C0C7AA89268597000000E78020C902
:10BB90002318A4FC268597000000E78040C82319DD
:10BBA000A4FC268597000000E78060C783D7440087
:10BBB0000A8A231AA4FC858393F7F70F230EF4FC5B
:10BBC0008607BD0793F7073F3301F1408A8A014991
:10BBD0008347C4FD6367F902CE85130584FC232CDB
:10BBE00054FD97000000E78080EA5281130104FCB5
:10BBF000F2506254D2544259B259225A925A216197
:10BC00008280268597000000E78060C193171900A5
:10BC1000D69705092390A7001379F90F55BF8280A5
:10BC200097A7FF1F938747F79C43D847A167938740
:10BC3000A702631AF70A397106DE22DC26DA8000D1
:10BC40004AD84ED652D456D23285B28497000000DC
:10BC5000E780C0BAAA89268597000000E78020BC4B
:10BC6000FD572318A4FC26852319F4FC9700000037
:10BC7000E780E0BA83D744000A8A231AA4FC8583AC
:10BC800093F7F70F230EF4FC8607BD0793F7073FE2
:10BC90003301F1408A8A01498347C4FD6367F90291
:10BCA000CE85130584FC232C54FD97000000E7800B
:10BCB00000DE5281130104FCF2506254D254425906
:10BCC000B259225A925A216182802685970000003B
:10BCD000E780E0B493171900D69705092390A700D1
:10BCE0001379F90F55BF828097A7FF1F9387C7EA83
:10BCF0009C43D847A16789076310F70A397106DEAC
:10BD000022DC26DA80004AD84ED652D456D232856A
:10BD1000328997000000E78060AEAA894A859700C3
:10BD20000000E780C0AF835749000A8A2318A4FCAB
:10BD3000858393F7F70F230CF4FC8607BD0793F771
:10BD4000073F3301F1408A8A8144834784FD63E7DA
:10BD5000F402CE85130584FC232A54FD97000000CD
:10BD6000E780E0D25281130104FCF2506254D254B5
:10BD70004259B259225A925A216182804A859700CB
:10BD80000000E780C0A993971400D69785042390FC
:10BD9000A70093F4F40F55BF828097A7FF1F9387E6
:10BDA000A7DF9C43D847A1679387E704631EF70A80
:10BDB000397106DE22DC26DA80004AD84ED652D40B
:10BDC00056D23285B28497000000E78020A3AA896A
:10BDD000268597000000E78080A42318A4FC268510
:10BDE00097000000E780A0A3231AA4FC26859700F3
:10BDF0000000E780C0A283D744000A8A2319A4FC6C
:10BE0000858393F7F70F230EF4FC8607BD0793F79E
:10BE1000073F3301F1408A8A01498347C4FD6367C4
:10BE2000F902CE85130584FC232C54FD97000000F5
:10BE3000E780E0C55281130104FCF2506254D254F1
:10BE40004259B259225A925A21618280268597001E
:10BE50000000E780C09C93171900D697050923902E
:10BE6000A7001379F90F55BF828097A7FF1F93870B
:10BE7000A7D29C43D847A1679387C704631AF70AE0
:10BE8000397106DE22DC26DA80004AD84ED652D43A
:10BE900056D23285B28497000000E7802096AA89A6
:10BEA000268597000000E7808097FD572318A4FCA3
:10BEB0002685231AF4FC97000000E780409683D77C
:10BEC00044000A8A2319A4FC858393F7F70F230EF5
:10BED000F4FC8607BD0793F7073F3301F1408A8AD8
:10BEE00001498347C4FD6367F902CE85130584FCCD
:10BEF000232C54FD97000000E78060B952811301A4
:10BF000004FCF2506254D2544259B259225A925A05
:10BF100021618280268597000000E780409093177A
:10BF20001900D69705092390A7001379F90F55BF7B
:10BF3000828097A7FF1F938727C69C43D847A16796
:10BF4000DD076317F7041763FFFFE7020316797134
:10BF50003285328497000000E780408A2AC6228515
:10BF600097000000E780A08B2311A1022285970093
:10BF70000000E780A088B2452300A10228089700AE
:10BF80000000E780C0B045611763FFFF670023141E
:10BF9000828097A7FF1F938727C09C43D847A1673C
:10BFA000938787046317F7041763FFFFE702E30F24
:10BFB00079713285328497000000E78020842AC698
:10BFC000228597000000E78080852311A102228549
:10BFD00097000000E7808082B2452300A102280874
:10BFE00097000000E780A0AA45611763FFFF670084
:10BFF000030E828097A7FF1F938707BA9C43D847F9
:10C00000A1679387A7046312F7021763FFFFE70294
:10C01000C30901112800814597000000E78020A78F
:10C0200005611763FFFF6700830A828097A7FF1FE0
:10C03000938787B69C43D847A167938757026319B4
:10C04000F7021763FFFFE70243060111328597F0FD
:10C05000FFFFE780A07A2308A10081452800970010
:10C060000000E780C0A205611763FFFF6700230699
:10C07000828097A7FF1F938727B29C43D847A16769
:10C080009387E702631BF7041763FFFFE702E301EF
:10C0900001113285328497F0FFFFE7804078AA844F
:10C0A000228597F0FFFFE7808077854709E92285A1
:10C0B00097F0FFFFE78080744205B337A0002800A7
:10C0C0008145231891003ECA97000000E780209C1C
:10C0D00005611763FFFF670083FF828097A7FF1F3B
:10C0E000938787AB9C43D84799476313F708176337
:10C0F000FFFFE70283FB79713285328497F0FFFFFF
:10C10000E780C06F2AC6228597F0FFFFE780207185
:10C110002310A102228597F0FFFFE780206E230104
:10C12000A102228597F0FFFFE780406DA301A102E5
:10C13000228597F0FFFFE780606C2302A102228531
:10C1400097F0FFFFE780806B2313A102228597F011
:10C15000FFFFE780A06AB2452314A10228089700D8
:10C160000000E780C09245611763FFFF670023F678
:10C17000828097A7FF1F938727A29C43D847A16778
:10C180009387C7036313F7081763FFFFE702E3F121
:10C1900079713285328497F0FFFFE78020662AC6E6
:10C1A000228597F0FFFFE78080672310A102228598
:10C1B00097F0FFFFE780A0662311A102228597F088
:10C1C000FFFFE780A0632302A102228597F0FFFF13
:10C1D000E780C062A302A102228597F0FFFFE780FB
:10C1E000E0612303A102228597F0FFFFE780006151
:10C1F000B245A303A102280897000000E780208928
:10C2000045611763FFFF670083EC82801763FFFFC0
:10C21000E702A3E901112A8497F0FFFFE780005E9F
:10C22000AA84228597F0FFFFE780605F228597F060
:10C23000FFFFE780C05E035744008D4763F7E700C8
:10C24000228597F0FFFFE780805D228597F0FFFF52
:10C25000E780E05C2800A68597000000E780208347
:10C2600005611763FFFF670083E697A7FF1F9387AA
:10C27000A7929C43D847A167FD07631FF700176388
:10C28000FFFFE70283E2328597000000E78040F875
:10C290001763FFFF6700A3E3828097A7FF1F9387C1
:10C2A000A78F9C43D847A167E5076315F708176375
:10C2B000FFFFE70283DF79713285328497F0FFFF59
:10C2C000E780C0532AC6228597F0FFFFE7802055FC
:10C2D000228597F0FFFFE78080542310A10222857A
:10C2E00097F0FFFFE780A053520551812311A1026F
:10C2F00022852302010297F0FFFFE7802050A3026E
:10C30000A102228597F0FFFFE780404F2303A1029F
:10C31000228597F0FFFFE780604EB245A303A1029C
:10C32000280897F0FFFFE780807645611763FFFFDD
:10C330006700E3D9828097A7FF1F9387E7859C4317
:10C34000D847A1679387E703631FF7001763FFFFD1
:10C35000E702A3D5328597000000E78060EB176302
:10C36000FFFF6700C3D6828097A7FF1F9387C7820E
:10C370009C43D847A16793874704631EF70217635E
:10C38000FFFFE70283D279713285328497F0FFFF95
:10C39000E780C0462AC6228597F0FFFFE780204845
:10C3A000B245280897F0FFFFE780606E456117638C
:10C3B000FFFF6700C3D182809797FF1F9387C77DD8
:10C3C0009C43D847A167938787026310F7041763DC
:10C3D000FFFFE70283CD79713285328497F0FFFF4A
:10C3E000E780C0412AC6228597F0FFFFE780004121
:10C3F000B2452300A102280897F0FFFFE7802069DB
:10C4000045611763FFFF670083CC82801763FFFFDE
:10C41000E702A3C9011197F0FFFFE780203EAA853C
:10C42000280097F0FFFFE780806605611763FFFF34
:10C430006700E3C99797FF1F938707769C43D84708
:10C44000A167D107631FF7001763FFFFE702E3C58A
:10C45000328597000000E780A0FB1763FFFF6700AD
:10C4600003C782809797FF1F938707739C43D84722
:10C47000A167C507631FF7001763FFFFE702E3C269
:10C48000328597000000E780A0F81763FFFF670080
:10C4900003C482809797FF1F938707709C43D847F8
:10C4A000A167B907631FF7001763FFFFE702E3BF48
:10C4B000328597000000E780A0F51763FFFF670053
:10C4C00003C182809797FF1F9387076D9C43D847CE
:10C4D000A167AD07631FF7001763FFFFE702E3BC27
:10C4E000328597000000E780A0F21763FFFF670026
:10C4F00003BE82809797FF1F9387076A9C43D847A4
:10C5000089476318F7021763FFFFE70203BA0111B7
:10C51000328532C897F0FFFFE780402EAA852800B9
:10C5200097F0FFFFE780A05605611763FFFF6700E4
:10C5300003BA82809797FF1F938707669C43D8476B
:10C54000A1678D076311F7041763FFFFE702E3B5E7
:10C5500001113285328497F0FFFFE780202A13060D
:10C560006100AA844C00228597300000E780C02338
:10C570002800A68597F0FFFFE780605105611763EB
:10C58000FFFF6700C3B482809797FF1F93870761FF
:10C590009C4381CFDC4391CB1763FFFFE702E3B0FD
:10C5A00082971763FFFF670083B282801763FFFFE4
:10C5B000E702A3AF79713C08AE843ED2A165B7070C
:10C5C0000A002A843ED448103C08DD053ED636C415
:10C5D00032C63AC297D0FFFFE780E02F12474810DB
:10C5E000BA8597F0FFFFE780C01332464810B28546
:10C5F00097F0FFFFE780E014A2464810B68597F059
:10C60000FFFFE7800012501001478146A685228572
:10C6100097D0FFFFE780805145611763FFFF6700F8
:10C6200003AB1763FFFFE70243A801117C00032956
:10C63000C501AE843ECAA165B70707002A843ECC77
:10C6400048087C00C5053ECE97D0FFFFE780A028B4
:10C650008345D900480897F0FFFFE780800C500819
:10C6600001478146A685228597D0FFFFE780004CD1
:10C6700005611763FFFF670083A51763FFFFE702EC
:10C68000C3A283C7950093F7F707A384F50097002B
:10C690000000E78040F91763FFFF670043A31763BB
:10C6A000FFFFE70283A079713C08AE843ED2A1650A
:10C6B000B70709002A843ED448103C0893854504F6
:10C6C0003ED632C636C497D0FFFFE780C020A246D0
:10C6D0004810B68597F0FFFFE780A0043246481067
:10C6E000B28597F0FFFFE780C005501001478146F3
:10C6F000A685228597D0FFFFE780404345611763F9
:10C70000FFFF6700C39C1763FFFFE702039A83C71D
:10C71000950041112A8493F7F707A384F500328529
:10C720002EC697F0FFFFE780800F85672AC46370ED
:10C73000F50297700000E78020E92246B24509ED36
:10C7400011478146228597000000E78060E641019D
:10C750001763FFFF6700A39701478346F501DDB725
:10C760001763FFFFE702C39201113C003ECAB707FF
:10C770000A003ECC3C003ECE83C79500AA89328594
:10C7800093F7F707A384F5002E8497F0FFFFE78067
:10C7900000098567637DF504A165AA8493858504F6
:10C7A000480897D0FFFFE7800013268597700000A8
:10C7B000E78080E12A8929E19145480897F0FFFF49
:10C7C000E78020F6A685480897F0FFFFE78060F72E
:10C7D000CA85480897F0FFFFE780A0F4014781462B
:10C7E0005008A2854E8597D0FFFFE7802034056171
:10C7F0001763FFFF6700038D8145480897F0FFFF2F
:10C80000E78020F20349090275BF1763FFFFE702C3
:10C81000238879711C103ECAB7070F003ECC404DEB
:10C820001C10AA84AE894808994532C636893ECE86
:10C8300097D0FFFFE780200A32464808B28597F07C
:10C84000FFFFE78000EE630C0902A545480897F05A
:10C85000FFFFE780C0E62546CA8597200100E780F4
:10C8600020A4500801478146CE85268597D0FFFF3A
:10C87000E780C02B45611763FFFF6700A3848355E2
:10C88000C402480897F0FFFFE780A0EB0355E402DD
:10C89000814505C5854785456301F502C167FD17DB
:10C8A0009305F00F630BF5007D1597700000E7808E
:10C8B000208E9305150093F5F50F480897F0FFFFBC
:10C8C000E78020E683450403480897F0FFFFE780F0
:10C8D00040E583451403480897F0FFFFE78060E4D4
:10C8E00083552403480897F0FFFFE78080E58355D0
:10C8F0004403480897F0FFFFE780A0E49DB7175373
:10C90000FFFFE702837A83C795008146014693F7CC
:10C91000F707A384F50097000000E78040EF175366
:10C92000FFFF6700C37A1753FFFFE70203787971AF
:10C930003E841C103ECA2E89B7070F00A1653ECC6D
:10C94000FD051C10AA84480842C03AC23ECE36C437
:10C9500032C697D0FFFFE78000F832464808B2851C
:10C9600097F0FFFFE780E0DBA2464808B68597F026
:10C97000FFFFE78000DD12474808BA8597F0FFFF08
:10C98000E78020DC0248630C08029145480897F0D4
:10C99000FFFFE780C0D21146A28597200100E78003
:10C9A0002090500801478146CA85268597D0FFFF11
:10C9B000E780C01745611753FFFF67004371894542
:10C9C000480897F0FFFFE78080CF834704002300EB
:10C9D000F50083471400A300F500E1B71753FFFFEC
:10C9E000E702036B83C7950001112A8A93F7F707C3
:10C9F000A384F5003285AE8432C697F0FFFFE7804E
:10CA000000E232462A89328597F0FFFFE78000DF97
:10CA100085676373F902AA894A8597700000E780E9
:10CA2000A0BA2A8419ED114781464A86A685528507
:10CA300097000000E780C0B705611753FFFF67004C
:10CA400063689387E9FF93F7F70F0547E366F7FEFF
:10CA50008347F50195EB8947E380F9FE8346F401AE
:10CA6000528501474A86A68597000000E78040B4BA
:10CA7000A167D90748083ECC230A010002CE9700DF
:10CA80000000E780A0B04DBF639EE7008947639E2A
:10CA9000F90093071020231FF50097700000E7802E
:10CAA000C0B76DBF0947E39BE7FA8D47E398F9FAF2
:10CAB000228597700000E78080DF9797FF1F93879C
:10CAC000E72C9C4399E79797FF1F9387E7159C43B3
:10CAD00099C703D5040097800000E780A0CE231FEC
:10CAE000040022855DBF1753FFFFE702035C0111BD
:10CAF0003C003ECAB7070B003ECC3C003ECE83C78D
:10CB000095002A89328593F7F707A384F500AE8450
:10CB100097F0FFFFE780A0D093170501C187635A04
:10CB2000F006A1652A849385E502480897D0FFFFA7
:10CB3000E78060DAA285480897F0FFFFE78060C0D1
:10CB40009797FF1F9387470E9C43A9EB014493756A
:10CB5000F40F480897F0FFFFE780A0BC935584408E
:10CB600093F5F50F480897F0FFFFE78080BB9355DA
:10CB7000044193F5F50F480897F0FFFFE78060BA8E
:10CB8000014781465008A6854A8597D0FFFFE78078
:10CB9000E0F905611753FFFF670063534165854660
:10CBA0000546A2857D1597500000E78060BD59DDE0
:10CBB000510597000100E780808F1304400633443D
:10CBC000850271B71753FFFFE702234E0111B70724
:10CBD00006003EC683C7950021642A8993F7F707AC
:10CBE000A384F500AE8428009305A4040AC40AC8EF
:10CBF00097D0FFFFE78020CE300001478146A68511
:10CC00004A8597D0FFFFE78060F297E0FFFFE7805B
:10CC1000801513049404480822CC230A010002CE94
:10CC200097000000E780809605611753FFFF6700BB
:10CC3000034A1753FFFFE702A345C1642A89014451
:10CC40009799FF1F93890916130A8002FD1497E034
:10CC5000FFFFE78080C16347A40001451753FFFF32
:10CC600067004346B307440303A7C90ABA9703D72B
:10CC700007006306970083D7270063842701050414
:10CC8000F9B70545E1BF1753FFFFE70263402A8A62
:10CC90002E8999C123A0050081498144979AFF1FDD
:10CCA000938A0AF0614B97E0FFFFE78040C263C7B9
:10CCB000A4004E851753FFFF6700C340338464030D
:10CCC00083A70A003E948357040099E76304090090
:10CCD000232089008504C1BF4146D2851305440045
:10CCE00097100100E780605975F5A289E5B71753E1
:10CCF000FFFFE702E33939717C083ED4B7070A0029
:10CD00003ED67C083ED883C795002A8A328593F7A1
:10CD1000F707A384F5002E8932C697F0FFFFE7805E
:10CD200000B085676373F5083246AA84328597F0B0
:10CD3000FFFFE780A0AC8547AA8963E8A706A16545
:10CD400093858504281097D0FFFFE780C0B826851B
:10CD500097700000E78040872A8429ED91452810CC
:10CD600097F0FFFFE780E09BA685281097F0FFFF74
:10CD7000E780209DCE85281097F0FFFFE780609A1E
:10CD8000014781463010CA85528597D0FFFFE78062
:10CD9000E0D9A1679387770448183EDC230A010293
:10CDA00002DE97F0FFFFE780607E21611753FFFFEF
:10CDB000670043318145281097F0FFFFE7806096B8
:10CDC000A685281097F0FFFFE780A0979797FF1F91
:10CDD000938707349C4381CB22856389090097D0D0
:10CDE0000000E78040248345040271B797D000001B
:10CDF000E780C022CDBF1753FFFFE702632983C737
:10CE000095004111AA8993F7F707A384F5003285AD
:10CE1000AE84328A97F0FFFFE78060A08567637F6A
:10CE2000F5022A8997600000E780007A2A849146FB
:10CE300031C58347F50105476387E70291C70D4771
:10CE40006366F704AD461DA89305050303250A0094
:10CE5000414697100100E78040420DE94101175318
:10CE6000FFFF670023269305950803250A00414626
:10CE700097100100E7806040814669F54A86A685E3
:10CE80004E8597000000E780C081C9BF83250A0056
:10CE90001305940897700000E780A02919C1C146C6
:10CEA000F1BF9797FF1F938767EE9C4399E797978A
:10CEB000FF1F938767D79C4399C7228597800000FF
:10CEC000E780208A69FD8547A30FF400228597B08B
:10CED0000000E7806084228597600000E780E073AF
:10CEE0004E8581464A86A68597F0FFFFE780607BE6
:10CEF000A1679387570448003EC42302010002C67D
:10CF000097F0FFFFE780806891BF1753FFFFE702AC
:10CF1000431783C795004111AA8993F7F707A384A4
:10CF2000F50032852E89B28A97F0FFFFE780208FC7
:10CF300085676374F50EAA8497600000E780C06877
:10CF40002A840DED416B014A979BFF1F938B8BE564
:10CF5000130C400E7D1B19A833048A0383A70B0B07
:10CF60003E948357C40163836705050A97E0FFFF7A
:10CF7000E780A08EE342AAFE95460DA08357C50127
:10CF8000639697029305050303A50A00414697108F
:10CF90000100E780802E994611E181462686CA85E8
:10CFA0004E8597F0FFFFE780C06F85A883A50A0034
:10CFB0001305040397700000E780A017C14679FDB0
:10CFC0002285231E940097A00000E780E07422854C
:10CFD00097600000E78060649797FF1F938747136F
:10CFE0009C43A9C323000402228597D00000E78058
:10CFF00040F04E8581462686CA8597F0FFFFE78080
:10D00000406AA1679387070448003EC423020100D9
:10D0100002C697F0FFFFE780605741011753FFFFFB
:10D020006700A30989472300F402E1B7397106DEDE
:10D0300022DC4AD8800052D456D25AD026DA4ED6B4
:10D040005ECE2E8A32892A8B97D0FFFFE780E07D63
:10D050000605710541998A8A3301A140232224FCE7
:10D06000231404FC97D0FFFFE780207C83479A00BD
:10D070000605350593F7F7072315A4FCA304FA006A
:10D080004A85232624FC97E0FFFFE7804079931729
:10D090000501C1876340F0025681130104FCF25080
:10D0A0006254D2544259B259225A925A025BF24BFC
:10D0B00021618280AA844A8597E0FFFFE78020767D
:10D0C000AA894A8597E0FFFFE7806075A16593858F
:10D0D000C5022A89130544FC97C0FFFFE780A07FA3
:10D0E000268597C0FFFFE780E073854511C94A8612
:10D0F000CE8597C0FFFFE780606DAA8B21E9894547
:10D10000130544FC97E0FFFFE780A061A6851305A7
:10D1100044FC97E0FFFFE780C062CE85130544FC26
:10D1200097E0FFFFE780E061CA85130544FC97E0C4
:10D13000FFFFE780006101478146130644FCD2856A
:10D140005A8597D0FFFFE780609EB9B781451305E8
:10D1500044FC97E0FFFFE780C05CA685130544FC14
:10D1600097E0FFFFE780E05DCE85130544FC97E084
:10D17000FFFFE780005DCA85130544FC97E0FFFFD1
:10D18000E780205C814497D0FFFFE780006AE3D40A
:10D19000A4FA83A70B0113971400BA9783D507004D
:10D1A00099C5130544FC97E0FFFFE780805985048B
:10D1B000D9BF797106D622D44AD000184ECE52CCAF
:10D1C00056CA26D25AC8AE893289AA8A97D0FFFF9A
:10D1D000E780A0650605690541990A8A3301A140E7
:10D1E000232A24FC231C04FC97D0FFFFE780E06384
:10D1F00083C7990006052D0593F7F707231DA4FCA7
:10D20000A384F9004A85232E24FC97E0FFFFE780E2
:10D21000006193170501C187634FF000528113012C
:10D2200004FDB250225492540259F249624AD24A41
:10D23000424B45618280AA844A8597E0FFFFE780E0
:10D24000005EA1659385A5022A89130544FD97C058
:10D25000FFFFE7804068268597C0FFFFE780805C7E
:10D26000854509C9CA8597C0FFFFE78020592A8BE9
:10D2700029E18945130544FD97E0FFFFE780604AF7
:10D28000A685130544FD97E0FFFFE780804BCA8524
:10D29000130544FD97E0FFFFE780A04A0147814660
:10D2A000130644FDCE85568597D0FFFFE7800088A2
:10D2B000B5B78145130544FD97E0FFFFE780604661
:10D2C000A685130544FD97E0FFFFE7808047CA85E8
:10D2D000130544FD97E0FFFFE780A046814497D007
:10D2E000FFFFE7808054E3DBA4FA83270B01139749
:10D2F0001400BA9783D5070099C5130544FD97E03C
:10D30000FFFFE78000448504D9BF1753FFFFE70202
:10D31000C3D983474500404DD5EFFD575DC48346D3
:10D32000940009476363D70A0346B400854663EE59
:10D33000C6088306E40063CA06085C45F9562390D4
:10D34000D7009797FF1F83C7E78599E3A304E400FD
:10D350009797FF1F9387478D9C4381E78947A306D3
:10D36000F4009797FF1F9387A7DA9C4381E78947CB
:10D370002306F4009705000093854506AA8413054B
:10D38000040197F00000E7802010FD57231AF402F3
:10D3900081471CDC01489797FF1F23A1878097874F
:10D3A000FF1F9387E77F232E040304C0804397D099
:10D3B000FFFFE780C05161463306C50281452285E3
:10D3C0009750FFFFE78060D181473E851753FFFFED
:10D3D0006700E3CFFD57D5BF1753FFFFE702E3CC4C
:10D3E0002A840355450297600000E780E01D19E597
:10D3F000231E04001753FFFF670063CD8357E4012A
:10D40000F5DB930504FF174501001305E52B97E0B5
:10D410000000E780E014F9BF1753FFFFE702E3C8FD
:10D420002E89A16541119385E5032A8436C432C64D
:10D43000BE843AC297C0FFFFE780E04912472285C9
:10D44000BA8597E0FFFFE780C02D32462285B2857E
:10D4500097E0FFFFE780E02EA2462285B68597E0A1
:10D46000FFFFE780002E630309029145228597E0C4
:10D47000FFFFE780C0241146A68597100100E780D2
:10D4800020E241011753FFFF670063C489452285ED
:10D4900097E0FFFFE780A02283C704002300F50088
:10D4A00083C71400A300F500E9BF1753FFFFE7028D
:10D4B000C3BF83C79500444D054793F7F707A3847F
:10D4C000F5001C42411183C707006367F7062E84ED
:10D4D0002A89B1C003C7D400630FF7021787FF1F63
:10D4E00013078774184305C3A386F40097A00000B0
:10D4F000E780404A83C7D40099E741657D1597408E
:10D500000000E780403083D72403918B89C797E0E0
:10D510000000E780C0134A85A28597F0FFFFE780EF
:10D520008010A167C10748003EC42302010002C663
:10D5300097F0FFFFE780800541011753FFFF670069
:10D5400003B91753FFFFE70243B603D745008D47E2
:10D55000AA8441112E8432892E8563E3E70297E085
:10D56000FFFFE780C02BAA8523000900268597C00E
:10D57000FFFFE780A02841011753FFFF670023B595
:10D5800097E0FFFFE780A0292AC6228597E0FFFFEA
:10D59000E780E028B24585472A862300F9002685E2
:10D5A00097C0FFFFE7808022F9B7397106DE22DCE1
:10D5B00026DA80004ED652D456D24AD85AD05ECE01
:10D5C000AE89B284AA8A97D0FFFFE78000250605BE
:10D5D0001305250241990A8A3301A140232224FC24
:10D5E000231404FC97D0FFFFE780202383C7990012
:10D5F00006054D0593F7F7072315A4FCA384F9004E
:10D600002685232624FC97E0FFFFE780402193171F
:10D610000501C1876340F0025281130104FCF250FE
:10D620006254D2544259B259225A925A025BF24B76
:10D6300021618280AA8B03AB040097C0FFFFE780C3
:10D64000601E51E583D7440001498544F11793B723
:10D650001700A301F4FC834734FCA165C9C7938577
:10D66000E504130544FC97C0FFFFE780C026A685AC
:10D67000130544FC97E0FFFFE780A00ADE85130551
:10D6800044FC97E0FFFFE780C00B834734FC114662
:10D6900091E30946DA85130544FC97E0FFFFE78034
:10D6A00060058144630A0900416B7D1B97D0FFFF31
:10D6B000E780A01663CCA40201478146130644FC10
:10D6C000CE85568597C0FFFFE7804046B1B7A68557
:10D6D000130634FC97000000E780E0E69334150061
:10D6E0002A8986048DBF9385C504A5BF8327C900F9
:10D6F00013971400BA9783D5070063886501130553
:10D7000044FC97E0FFFFE780C003850445B717534B
:10D71000FFFFE702039779711C103EC4B7070F00A3
:10D720003EC61C103EC883C79500AA8A328593F76F
:10D73000F707A384F500AE89328497E0FFFFE78006
:10D74000000E93170501C187635AF0062A8A2285C5
:10D7500097E0FFFFE780A00C2A895285032B040085
:10D7600097C0FFFFE780000C39ED835744008144E8
:10D770000544F11793B71700A303F1008345710027
:10D78000DA872287CA865286280097000000E78041
:10D79000E0C8014781463000CE85568597C0FFFF1F
:10D7A000E780C038A1679387D70348083ECC230A97
:10D7B000810026CE97F0FFFFE78040DD45611753DB
:10D7C000FFFF6700838FA28513067100970000009A
:10D7D000E78060D7AA84094455D13544E30055FB5E
:10D7E0004A8597F0FFFFE78000450D4441D9014489
:10D7F00097D0FFFFE7806002634DA400C16B014436
:10D80000FD1B97D0FFFFE7804001634EA400154445
:10D81000B5B7DC4413171400BA9783D707006383A6
:10D8200027030504F1B7D84493171400BA9703D718
:10D830000700631B770123902701268597A000002E
:10D84000E78080DB01441DBF050465BF1753FFFF60
:10D85000E702038483C7950041112A8A93F7F707EB
:10D86000A384F50032852E89328497E0FFFFE7809C
:10D8700000FB93170501C1876353F006AA8922852F
:10D8800097E0FFFFE780A0F92311A1004E85832ACE
:10D89000040097C0FFFFE780E0F839E583574400B4
:10D8A00085440144F11793B71700A300F100034822
:10D8B000110003572100D6875285CE862686CA8559
:10D8C00097F0FFFFE7806006A167F10748003EC4BC
:10D8D0002302910022C697F0FFFFE78020CB410191
:10D8E0001743FFFF6700037EA28513061100970010
:10D8F0000000E78040C52A84894455D98357210018
:10D9000011678544BA97C2071167C1831307F7EF00
:10D91000E36FF7F89787FF1F938747479C4381CBB7
:10D9200085451305210097500000E7802075835539
:10D9300021002285814497C0FFFFE78040E525D97B
:10D9400023100500228597A00000E78040CD85B711
:10D950001743FFFFE702E37283C7950041112A8B4B
:10D9600093F7F707A384F50032852E8A328497E077
:10D97000FFFFE780C0EA93170501C1876351F006F6
:10D98000AA8A228597E0FFFFE78060E92A89568509
:10D99000832B040097C0FFFFE780C0E831E5835781
:10D9A000440081440544F11793B71700A301F10027
:10D9B00003483100DE875A854A87D6862286D2857B
:10D9C00097F0FFFFE78060F6A167ED0748003EC4CF
:10D9D0002302810026C697F0FFFFE78020BB4101AC
:10D9E0001743FFFF6700636DA285130631009700A0
:10D9F0000000E78040B5AA8409445DD99167CA97C1
:10DA0000C2071167C1831307F7EF0544E362F7FA12
:10DA1000CA8597C0FFFFE78080D7014451F981494B
:10DA200097D0FFFFE78060E063DBA90098489397F9
:10DA30001900BA9703D7070005EF2390270197D065
:10DA4000FFFFE78080DE1544E384A9F6268597A0D2
:10DA50000000E780C0BC9787FF1F938727339C4354
:10DA60000144B9D74A8597500000E780C05889B76C
:10DA700085097DB71743FFFFE702836179713E8413
:10DA80007C083EC82E8AB7071400A1653ECAE5058A
:10DA90007C08AA89080836C4428932C6BA8AC68474
:10DAA0003ECC97C0FFFFE78000E3CA85080897E0F7
:10DAB000FFFFE78000C732460808B28597E0FFFF06
:10DAC000E78020C8A246630A09049D45080897E03C
:10DAD000FFFFE780C0BE1D4681459740FFFFE780FE
:10DAE000C05F63890A089145080897E0FFFFE78057
:10DAF00000BD1146A68597000100E780607A1008F6
:10DB000001478146D2854E8597C0FFFFE78000021E
:10DB100045611743FFFF6700E35AB685080897E0A1
:10DB2000FFFFE78000C21C400808D8439355C70197
:10DB3000858912075183B205D98D97E0FFFFE780F1
:10DB400040C01C40080883C5870097E0FFFFE780BE
:10DB500040BD1C40080883C5A70097E0FFFFE78091
:10DB600040BC1C40080883C5970097E0FFFFE78092
:10DB700040BB85BF8945080897E0FFFFE78020B4D8
:10DB800083C704002300F50083C71400A300F50039
:10DB9000BDB71743FFFFE702A34F83C795004111AD
:10DBA000AA8993F7F707A384F5003285AE843284FF
:10DBB00097E0FFFFE780A0C693170501C187635D6B
:10DBC000F0042A89032A040097C0FFFFE78080C57C
:10DBD00019E9835744000548F11793B71700A307C5
:10DBE000F100814631A81306F100A28597000000DC
:10DBF000E78060951DC51C459DC783D64700014839
:10DC00000347F10093078500D2884A86A6854E8592
:10DC100097000000E78040E641011743FFFF6700DF
:10DC2000634A09487DBF1D486DBF1743FFFFE702E8
:10DC3000234665715C083EC4B7077B013EC65C089D
:10DC40003EC883C795002A8A328593F7F707A384D5
:10DC5000F500AE8997E0FFFFE78040BA8357E10007
:10DC6000E1C78945280097C0FFFFE780C0C681450E
:10DC7000280097E0FFFFE780C0AA97C0FFFFE7807A
:10DC8000A0CC9787FF1F9387A7489C431784FF1F4B
:10DC9000034444F1AA843334800099C313642400FC
:10DCA0009787FF1F938747F89C4399C313644400E9
:10DCB0009787FF1F9387870D9C4399C31364840044
:10DCC00083D504002800014997E0FFFFE78060A7A3
:10DCD00083D52400280097E0FFFFE78080A683D546
:10DCE0004400280097E0FFFFE780A0A597D0FFFF42
:10DCF000E780A0AE93150501C181280097E0FFFFE2
:10DD0000E78020A4A285280097E0FFFFE78060A3BA
:10DD10009C446360F902014781463000CE855285FC
:10DD200097C0FFFFE78080E059611743FFFF67005E
:10DD30006339DC441314490028003E9497E0FFFF48
:10DD4000E78060968347440003475400890706072D
:10DD5000BA978607E36AF5FC835524002800814AB8
:10DD600097E0FFFFE780E09D83454400280097E0AF
:10DD7000FFFFE780009B83455400280097E0FFFFEA
:10DD8000E780209A8347440063C9FA00814A8347A9
:10DD9000540063C1FA020509A5BF1C4413975A0039
:10DDA0002800BA9783D50700850A97E0FFFFE78030
:10DDB0004099C9BF032BC40093975A0028003E9B8B
:10DDC00083552B00850A97E0FFFFE78080978355F6
:10DDD0000B00280097E0FFFFE780A0964DBF174398
:10DDE000FFFFE702832C5C4993E717005CC997A00B
:10DDF0000000E78020B61743FFFF6700432D17435D
:10DE0000FFFFE702832A2E84814597F0FFFFE7801A
:10DE1000C0E705C583570500FD172310F50009C4A9
:10DE2000835725002310F40097000000E78060FB73
:10DE300001451743FFFF6700832931457DD8231033
:10DE40000400C5BF1743FFFFE702832483C7950083
:10DE500041112A8A93F7F707A384F50032852E89AA
:10DE6000328497E0FFFFE780809B93170501C1870D
:10DE70006356F006AA89C145228597E0FFFFE78037
:10DE8000A0802A8B4E85832A040097C0FFFFE7807D
:10DE9000609931E983574400231101000544F117CB
:10DEA00093B71700A300F100814403481100035702
:10DEB0002100D6875285CE862286CA8597F0FFFF3D
:10DEC000E780A0A6A1679387170248003EC42302FB
:10DED000810026C697E0FFFFE780406B41011743B2
:10DEE000FFFF6700231E13061100A28597F0FFFFB6
:10DEF000E7806065AA8409E523110100094475B72C
:10DF0000930521005A8597000000E78080EF835732
:10DF100021002A84D9DB9787FF1F938727E79C433B
:10DF200081CB85451305210097500000E78000153F
:10DF3000835521002685314497C0FFFFE780208567
:10DF40002DD523100500268597900000E780206DD1
:10DF50000144A1BF1743FFFFE702231541112E899A
:10DF60006C00AA8402C697F0FFFFE78000D20DC1C3
:10DF70000357050005072310E50097000000E78020
:10DF800040E681473E8541011743FFFF67002314A8
:10DF90003247954765DBCA85268597300000E780C4
:10DFA000400DC147E34005FE3244854741462310FA
:10DFB000F40083570900A685130544002311F400DB
:10DFC00097000100E780C02D228545BF1743FFFF62
:10DFD000E702030C83C795004111AA8A93F7F7075C
:10DFE000A384F5003285AE89328497E0FFFFE78095
:10DFF000008393170501C1876356F0062A8AC1453D
:10E00000228597D0FFFFE7802068AA845285032BE2
:10E01000040097C0FFFFE780E08031E983574400A8
:10E02000231101008544F11793B71700A300F100F5
:10E0300001440348110003572100DA875685D28630
:10E040002686CE8597F0FFFFE780208EA167938715
:10E05000070248003EC42302910022C697E0FFFF5A
:10E06000E780C05241011743FFFF6700A305A28567
:10E070001306110097F0FFFFE780E04C2A8409E5C2
:10E0800023110100894475B7268593052100970067
:10E090000000E78060ECAA8449FD835521002285B9
:10E0A00097B0FFFFE780A06E49F5014997C0FFFFD9
:10E0B000E780A077635DA900184893171900BA9705
:10E0C00003D707000DEF035721002390E70097C007
:10E0D000FFFFE7808075630625039787FF1F9387FF
:10E0E000E7CA9C4399C70355210097500000E78079
:10E0F00080F0228597900000E78060521DBF0509DF
:10E1000075B795443DB705C19307F00F630FF50050
:10E11000C547630CF5009307F5FF05453315F5007A
:10E120004205418182800145828041657D15828062
:10E13000B9E91743FFFFE70243F7034506033284BB
:10E1400097000000E78060FC9305803EB305B502B0
:10E15000C205C18181CD0357E402854763F8E7001A
:10E160001305040197E00000E78020428357E40292
:10E1700041677D176385E700FD172317F4021743F6
:10E18000FFFF6700C3F482801743FFFFE70263EFDE
:10E19000004283C79500444D0349140093F7F707E5
:10E1A000A384F50083470400220911673369F9004D
:10E1B000A167B347F90041112A8BAE8A63ECE70EE1
:10E1C000834724001307C00EB91793F7F70F637343
:10E1D000F71003473400C14763EEE70E834744005E
:10E1E0001307E00793C707086371F70C834984009E
:10E1F00083477400A209B3E9F900856763F7F90A58
:10E20000034A6400834754004E85220A336AFA00A9
:10E2100097500000E780403B61C123962403834B65
:10E220003400137AFA00239A340323887403239961
:10E23000440393890401631C090023A60402239864
:10E2400004024E8597E00000E78060363DA0034958
:10E2500024004A8597000000E78020EB2397A40262
:10E26000834744004E85A388F402E38D0BFCE30B47
:10E2700009FC97E00000E780202F97900000E780DE
:10E28000007381460146D6855A8597E0FFFFE780F7
:10E290000058A167938797033EC4230201004800FA
:10E2A00002C697E0FFFFE780602E41011743FFFFA2
:10E2B0006700A3E08544A2862686D6855A8597E026
:10E2C000FFFFE780C054A167938797033EC42302F2
:10E2D0009100F1B7BD44C5B79144F1BF1743FFFFAB
:10E2E000E70203DB01111C08404D3EC2B7070F00D7
:10E2F0003EC41C083EC62A89AE8997C0FFFFE7804E
:10E30000A0DA585C1C5C6346B70E6394E50063E2D8
:10E31000A70E3385A740B3B7A700B305B7401306D0
:10E32000803E81469D8D97000100E78080B7931461
:10E330000501C180A1659385C503480097B0FFFF23
:10E34000E78060598145480097D0FFFFE780603D36
:10E3500083550404480097D0FFFFE780803E835533
:10E360002404480097D0FFFFE780A03D814589CC79
:10E37000C167FD179305F00F6388F4002685975059
:10E380000000E780E0E0AA85480097D0FFFFE78023
:10E39000403903554404814501CDC167FD179305FC
:10E3A000F00F6307F50097500000E78060DEAA8554
:10E3B000480097D0FFFFE780C036834564044800DB
:10E3C00097D0FFFFE780E03583457404480097D07D
:10E3D000FFFFE7800035500001478146CE854A8522
:10E3E00097B0FFFFE780807405611743FFFF670068
:10E3F00063CD814481B71743FFFFE70203CB83C797
:10E40000950093F7F707A384F50097000000E780D5
:10E4100020ED1743FFFF670083CB1743FFFFE702A1
:10E4200023C783C795004111404D93F7F707A38495
:10E43000F5002A8A3285B284AE8997D0FFFFE78043
:10E44000003E2A8B268597D0FFFFE780403D2A8932
:10E45000268597D0FFFFE780603A93170B0163CAC8
:10E460000702E177CA97C207C183116763E3E70236
:10E4700093070910C207C1831307B00F637BF7002E
:10E4800093170901C187AA8A634AF000C54763FE52
:10E49000570141011743FFFF6700C3C297B0FFFF59
:10E4A000E780C028E31725FFD5B763080B02630692
:10E4B0000902814463890A02B7077F0023106405BB
:10E4C000231124057CC0568597000000E780E0C337
:10E4D0009304803EB304950239A0B7077F00232040
:10E4E00004047CC081440355240497E00000E780C5
:10E4F000A0A3A1C497C0FFFFE78000BB269593D7D8
:10E50000F44133379500AE97BA9708DC5CDCCE85D2
:10E51000528597000000E780A0DC99E023220404E4
:10E52000A1679387B70348003EC42302010002C6D7
:10E5300097E0FFFFE7808005A9BF814701481CDC09
:10E54000232E0403E9B71743FFFFE70203B697C082
:10E55000FFFFE780C037E1473305F502914597504B
:10E560000000E78000C5E55711C59777FF1F23A975
:10E57000A76281473E851743FFFF670043B5854784
:10E580001777FF1F2300F76282801743FFFFE70220
:10E59000C3B19777FF1F9387676080433DC0835760
:10E5A00004046390A70683572404639CB704368948
:10E5B000B28497C0FFFFE78020AF5C5C63C3B70401
:10E5C0006395B7001C5C63EEA7028347640463F3A2
:10E5D000F400A6872303F4048347740463F39700CD
:10E5E000A687A303F4048357440441677D1763851A
:10E5F000E70085072312F4043C4481C7CA852685B9
:10E6000082971743FFFF670083AC9777FF1F9387BD
:10E61000E7589C43014599C303C58700828017438F
:10E62000FFFFE70283A80111B70707003EC683C7B3
:10E630009500584D0AC493F7F7070AC8A384F5005C
:10E640002A89AE8411CB1C4283C707002304F7003C
:10E6500097900000E780003421649305540228005D
:10E6600097B0FFFFE780202797000000E78020FA9F
:10E67000AA85280097D0FFFFE780A00A3000014755
:10E680008146A6854A8597B0FFFFE780204A13049C
:10E690004402480822CC230A010002CE97E0FFFF83
:10E6A000E780C0EE05611743FFFF670043A21743F1
:10E6B000FFFFE702839F01117C003ECAB7070700F6
:10E6C0003ECC7C003ECE83C795002E84AA8493F76F
:10E6D000F707A384F500A16593855502480897B014
:10E6E000FFFFE780401F97000000E78040F2AA8507
:10E6F000480897D0FFFFE780C002500801478146D5
:10E70000A285268597B0FFFFE78040420561174349
:10E71000FFFF6700C39B9777FF1F938727489C43A2
:10E72000094599C303C5970082809777FF1F938798
:10E73000E7469C43094599C303C5D7008280977774
:10E74000FF1F9387A7459C43014599C303C5A700B5
:10E7500082801743FFFFE702A3930111B707080068
:10E760003EC683C79500404D0AC493F7F7070AC811
:10E77000A384F5002A89AE8429C41442854703C7BF
:10E78000060063E0E70A83479400094681496380F5
:10E79000C702B307F740A304E400B339F00083C70E
:10E7A00016002305F40097900000E780A01E035791
:10E7B0002403058B19C76386090097D00000E78002
:10E7C00000E9216493058402280097B0FFFFE780E9
:10E7D000801097000000E78040F4AA85280097D0B9
:10E7E000FFFFE78000F497000000E78080F5AA852E
:10E7F000280097D0FFFFE780C0F201478146300034
:10E80000A6854A8597B0FFFFE78040321304740263
:10E81000480822CC230A010002CE97E0FFFFE780E0
:10E82000E0D605611743FFFF6700C3891743FFFF69
:10E83000E702A38701117C003ECAB70708003ECC5F
:10E840007C003ECE83C795002E84AA8493F7F707F9
:10E85000A384F500A16593858502480897B0FFFF62
:10E86000E780600797000000E78020EBAA85480852
:10E8700097D0FFFFE780E0EA97000000E78060ECB8
:10E88000AA85480897D0FFFFE780A0E95008014714
:10E890008146A285268597B0FFFFE7802029056184
:10E8A0001743FFFF6700A3829777FF1F9387072F08
:10E8B0009C43014599C303C5B70082801733FFFF0E
:10E8C000E702A37E0111B70707003EC683C7950084
:10E8D000404D0AC493F7F7070AC8A384F5002A89B4
:10E8E000AE8405C81C42054783C707006368F70666
:10E8F0000347B400630FF700A305F40097900000EE
:10E90000E78040098347B400B9CF97D0FFFFE78085
:10E9100040BE21649305B400280097B0FFFFE78054
:10E9200080FB97000000E78060F8AA85280097D058
:10E93000FFFFE78000DF014781463000A6854A855A
:10E9400097B0FFFFE780801E2904480822CC230AE5
:10E95000010002CE97E0FFFFE78040C30561173357
:10E96000FFFF6700C37697D0FFFFE78020BF55B752
:10E970001733FFFFE702637301117C003ECAB7073C
:10E9800007003ECC7C003ECE83C795002E84AA842F
:10E9900093F7F707A384F500A165AD05480897B084
:10E9A000FFFFE78040F397000000E78020F0AA8592
:10E9B000480897D0FFFFE780C0D65008014781463E
:10E9C000A285268597B0FFFFE780401605611733C3
:10E9D000FFFF6700C36F9777FF1F9387271C9C4338
:10E9E000094599C303C5C70082801733FFFFE702BB
:10E9F000C36B01117C00AE843ECAA165B707070056
:10EA00002A843ECCD1057C0048083ECE97B0FFFF5B
:10EA1000E78060EC97000000E78020FCAA854808AA
:10EA200097D0FFFFE780E0CF500801478146A685D9
:10EA3000228597B0FFFFE780600F05611733FFFF66
:10EA40006700E3681733FFFFE702236683C795007B
:10EA500093F7F707A384F50097000000E78020F9FB
:10EA60001733FFFF6700A3661733FFFFE702436218
:10EA700083C795000329C501411193F7F707A384C4
:10EA8000F5001C4283C90700854763E6370797777F
:10EA9000FF1F9387E7679C432E84AA8485CF970046
:10EAA0000000E78080F389476306F50263040902EA
:10EAB0008347C9006380370323063901979000001C
:10EAC000E78040ED83572903898B89C797D00000E1
:10EAD000E780E0B72685A28597000000E78020F157
:10EAE000A167CD0748003EC42302010002C697E09B
:10EAF000FFFFE780A0A941011733FFFF6700835C98
:10EB00009777FF1F938787099C431D4599C303C5CA
:10EB1000E70082801733FFFFE70223590111B7078F
:10EB200007003EC683C79500584D0AC493F7F70700
:10EB30000AC8A384F5002A89AE8415C71C4283C77E
:10EB4000070093968701E18663C4060685466381C4
:10EB5000D7068346E7006388F6002307F7009790FF
:10EB60000000E78020E321649305E400280097B0CB
:10EB7000FFFFE78040D697000000E780A0F8AA8555
:10EB8000280097D0FFFFE780C0B9014781463000D9
:10EB9000A6854A8597B0FFFFE78040F9350448080D
:10EBA00022CC230A010002CE97E0FFFFE780009EFF
:10EBB00005611733FFFF670083511733FFFFE7023B
:10EBC000C34E01117C003ECAB70707003ECC7C0053
:10EBD0003ECE83C795002E84AA8493F7F707A384BB
:10EBE000F500A165B905480897B0FFFFE780A0CE02
:10EBF00097000000E78000F1AA85480897D0FFFF42
:10EC0000E78020B2500801478146A285268597B04B
:10EC1000FFFFE780A0F105611733FFFF6700234B7B
:10EC20001733FFFFE702C346AA8401441779FF1F89
:10EC3000130909F7E14997C0FFFFE78040C9634422
:10EC4000A400014519A833053403832709003E9524
:10EC5000835725006397970011051733FFFF67005F
:10EC600063460504C9BF032E8500630A0E1217739D
:10EC7000FF1F1303A311032303006315030029439C
:10EC80006390061203234E01631503001D4363992D
:10EC900007101733FFFFE702C33EC689428A3E8949
:10ECA000BA8AB684328BAE8B2A84B5E103554E0006
:10ECB00019E501431A851733FFFF67000340A16779
:10ECC000A98F116763FBE70097000000E78080F5DC
:10ECD000814597F0FFFFE780C0120844B70700E0C6
:10ECE0005841F98F18455CC1B707001FF98F1CC543
:10ECF0005C4991C7610597E00000E780408BE38A9B
:10ED000009FA228597900000E78060C65DB73285DA
:10ED100097C00000E78040430D4349DD1C44116764
:10ED200003D54700A167A98F63FBE70097000000A8
:10ED3000E78040EF814597F0FFFFE780800C0323D9
:10ED4000840093164B01D1828347B30003566300BE
:10ED50008588FD8BA305F300FD777D8E558EFD76AE
:10ED6000FD16B204F18E83274301C58E2312730171
:10ED70002313D3002304530123052301A3044301D8
:10ED8000BDDF228597B0FFFFE78020CDAA8508442C
:10ED9000B5D1610597D00000E780207F8DB71D4376
:10EDA0001A8582801733FFFFE702832E0569AA8444
:10EDB000AE89328A0144FD5A7D1997C0FFFFE78072
:10EDC000C0A56347A40001451733FFFF6700832FE9
:10EDD000D84493171400BA9703D70700631F37036B
:10EDE0002390570163070A00268597900000E7806B
:10EDF000A0809C449DC383D76700B3F72701639E1F
:10EE00003701D28801488147014781460146814543
:10EE1000268597000000E78040E5050479BF173399
:10EE2000FFFFE702E32679711C103EC4B7070F000D
:10EE30003EC61C103EC883C79500AA8A328593F748
:10EE4000F707A384F5002E89328497D0FFFFE7806F
:10EE5000009D93170501C187635AF006AA89228590
:10EE600097D0FFFFE780A09B2A8A4E85032B0400E2
:10EE700097B0FFFFE780009B39ED83574400814442
:10EE80000544F11793B71700A303F1008345710000
:10EE9000DA872287D2864E86280097E0FFFFE78038
:10EEA000E057014781463000CA85568597B0FFFF7D
:10EEB000E780C0C7A1679387F70348083ECC230AC1
:10EEC000810026CE97D0FFFFE780406C4561173365
:10EED000FFFF6700231FA2851306710097E0FFFF65
:10EEE000E7806066AA84094455D1528597E0FFFF08
:10EEF000E78060D40D4459D90546D2852685970010
:10EF00000000E78060EA2A8451B71733FFFFE70269
:10EF1000C319835507000346270041112A842E8513
:10EF200032C62EC497E0FFFFE780E0D001C9324629
:10EF3000A245228597000000E78000E741011733D2
:10EF4000FFFF6700C3181733FFFFE702831383C770
:10EF500095004111AA8A93F7F707A384F50032853B
:10EF6000AE89328497D0FFFFE780608B931705014D
:10EF7000C1876357F00AC1452A8A228597C0FFFFDF
:10EF8000E78080702A8D228597D0FFFFE780208957
:10EF90002A89228597D0FFFFE7804086930705F8EE
:10EFA00093F7F70F1307E007AA8B637BF706228519
:10EFB00097D0FFFFE78080842A8C228597D0FFFFBF
:10EFC000E780C083AA8C5285032B040097B0FFFF13
:10EFD000E780408539E983574400231101008144CB
:10EFE000F11793B71700A300F10005440347110080
:10EFF00083562100938784005685DA8822885286BA
:10F00000CE8597F0FFFFE78020A7A167E9074800BA
:10F010003EC42302810026C697D0FFFFE780005739
:10F0200041011733FFFF6700430913061100A28552
:10F0300097E0FFFFE7802051AA8409E52311010032
:10F0400009446DB7930521006A8597F0FFFFE780BB
:10F05000A0F02A8441FD835521009356C900131660
:10F06000490185486688E2875E87858A51822685C0
:10F0700097000000E78060BF2A848DBF1733FFFF31
:10F08000E702230083C7950041112A8B93F7F70706
:10F09000A384F5003285AE89328497C0FFFFE780F4
:10F0A000007893170501C1876352F00A2A8A2285E6
:10F0B00097C0FFFFE780A076AA8A228597C0FFFF4E
:10F0C000E780E0752A89228597C0FFFFE7800073FB
:10F0D000930705F893F7F70F1307E0072A8C637778
:10F0E000F706228597C0FFFFE7804071AA8C228532
:10F0F00097C0FFFFE78080702A8D5285832B040024
:10F1000097A0FFFFE780007239E5835744008544EC
:10F110000144F11793B71700A301F1000347310031
:10F12000930784005A85DE882688D6865286CE8547
:10F1300097F0FFFFE78040948D4748003EC42302CC
:10F14000910022C697D0FFFFE7804044410117336A
:10F15000FFFF670083F6A2851306310097E0FFFFEB
:10F16000E780603E2A84894455D99356C900131616
:10F17000490185486A88E6876287858A5182D685F3
:10F1800097000000E78060AEAA8449BF1733FFFFF5
:10F19000E70203F02A8981440144617A916A177B6E
:10F1A000FF1F130BABBE97B0FFFFE780006863C77C
:10F1B000A40022851733FFFF6700C3F083270900EF
:10F1C00093991400CE9703D50700330745014207F2
:10F1D00041836364570305C103270B0019C78545A5
:10F1E0003E8597400000E78060E983270900050419
:10F1F000CE972390070085047DB797000000E78035
:10F2000060A2832709000504CE972390070065D5E7
:10F21000814597F0FFFFE780C0BEF1BF1733FFFFC6
:10F22000E70203E783C7950041112A8A93F7F7079E
:10F23000A384F50032852E89328497C0FFFFE780D2
:10F24000005E93170501C187635AF004AA89832AD7
:10F25000040097A0FFFFE780E05C31E5835744009E
:10F2600085440144F11793B71700A301F100034847
:10F270003100D68752850147CE862686CA8597D02B
:10F28000FFFFE780806AA167F50748003EC42302BC
:10F29000910022C697D0FFFFE780402F410117332E
:10F2A000FFFF670023E2A2851306310097E0FFFF0E
:10F2B000E78060292A8489445DD99777FF1F938767
:10F2C000E7AC9C4381CF044997B0FFFFE780E0554E
:10F2D000AA85268597400000E78040DA13050401DF
:10F2E00097000000E780C0EA228597800000E78051
:10F2F00000338144ADBF1733FFFFE70283D883C7D4
:10F3000095004111AA8A93F7F707A384F500328587
:10F31000AE8932842311010097C0FFFFE78020509F
:10F3200093170501C1876354F0062A8AC1452285D7
:10F3300097C0FFFFE7804035AA8B5285032B04005E
:10F3400097A0FFFFE780004E21E9835744008544E2
:10F350000144F11793B71700A300F100034811000F
:10F3600003572100DA875685D2862686CE8597D028
:10F37000FFFFE780805BA1679387270248003EC4B8
:10F380002302910022C697D0FFFFE7802020410191
:10F390001733FFFF670063D2A2851306110097E0C1
:10F3A000FFFFE780401A2A8489444DD99777FF1FD1
:10F3B0009387C79D98433E8901CF044997B0FFFFCB
:10F3C000E780A046AA85268597400000E78000CB0D
:10F3D0001305040197000000E78080DB97B0FFFF72
:10F3E000E780A04495443DD9930521005E8597F0C0
:10F3F000FFFFE78060B6AA8435F11C48035721005F
:10F4000022852390E70097800000E7804021832732
:10F410000900A9D70355210097400000E780A0BD4F
:10F4200035BF1733FFFFE702C3C583C795004111FE
:10F43000AA8A93F7F707A384F5003285AE89328450
:10F4400097C0FFFFE780A03D93170501C187635177
:10F45000F0062A8A228597C0FFFFE780403C2A8970
:10F460005285032B040097A0FFFFE780A03B31E506
:10F470008357440085440144F11793B71700A30153
:10F48000F10003483100DA8756854A87D2862686FE
:10F49000CE8597D0FFFFE7804049A167F907480074
:10F4A0003EC42302910022C697D0FFFFE780000EE2
:10F4B00041011733FFFF670043C0A28513063100E7
:10F4C00097E0FFFFE78020082A8489445DD991678F
:10F4D000CA97C2071167C1831307F7EF8544E36238
:10F4E000F7FA9777FF1F9387678A9843BE8B01CF00
:10F4F000044997B0FFFFE7804033AA8526859740EF
:10F500000000E780A0B71305040197000000E78022
:10F5100020C897B0FFFFE780403195443DD11C489B
:10F52000228581442390270197800000E780200FE7
:10F5300083A70B00B9D74A8597400000E780A0ABAE
:10F5400089B71733FFFFE70243B62A844105B28427
:10F5500097000000E780C0C311C522859780000096
:10F56000E780E00B81460146A68522859780000052
:10F57000E780C04E1C4C89C7DC4799C3228582971F
:10F580001733FFFF6700A3B49767FF1F93870761D7
:10F590009C43014599C31385070182809767FF1F2C
:10F5A0009387C75F884382801733FFFFE702E3AF8B
:10F5B0009317C600DD8DC2054111C1812A8432C670
:10F5C00097C0FFFFE780E0173246228511829375CE
:10F5D000F60F97C0FFFFE780C01441011733FFFF0C
:10F5E0006700E3AE1733FFFFE70283AA79713C0897
:10F5F0003ED2B7070C003ED43C083ED683C79500E8
:10F60000AE842A8993F7F707A384F500A165938553
:10F610003504481097A0FFFFE780E02BC165FD157A
:10F620000144176AFF1F130AEA77930A400EAE8956
:10F630002E8B2EC697B0FFFFE7802022420593173E
:10F6400004014181C183B24563E9A702C167FD1787
:10F650006387F500481097C0FFFFE780800E5010C9
:10F6600001478146A6854A8597A0FFFFE780004CA9
:10F6700045611733FFFF6700E3A433075403832773
:10F680000A0BBA9703D6C701630A3601638A3501AC
:10F69000481097000000E78060F1DA85050451BF4B
:10F6A000B285EDBF1733FFFFE702A39D79717C0898
:10F6B0003EC8B70711003ECA7C083ECC83C7950000
:10F6C000AA89328593F7F707A384F5002E8997C09E
:10F6D000FFFFE780C01485676378F504A165AA84FD
:10F6E0008905080897A0FFFFE780E01E2685974060
:10F6F0000000E78060ED133415000A04A2850808B5
:10F7000097C0FFFFE780E001A685080897C0FFFFCC
:10F71000E780200325CC014781461008CA854E8525
:10F7200097A0FFFFE780804045611733FFFF670028
:10F73000C398B30754030327CA0ABA9703D707002D
:10F74000631C970003D627006380650508089700AF
:10F750000000E780A0E5DE8505042EC697B0FFFF18
:10F76000E780A0104205931704014181C183B2458F
:10F77000E3E1A7FCC167FD17E38FF5F8080897C020
:10F78000FFFFE78000FC41BFB285F9B7C165FD15F9
:10F790000144176AFF1F130AEA60930A80022E8B46
:10F7A000AE8B65BF1733FFFFE702239018418347F5
:10F7B000170083460700A207D58FD207D183239075
:10F7C000F50083472700034717008D45A207D98F0F
:10F7D00091832310F60097C0FFFFE780A0E917335D
:10F7E000FFFF6700C38E1733FFFFE702638AC16420
:10F7F00001441769FF1F1309E95A93098002FD1498
:10F8000097B0FFFFE78060066347A4000145173308
:10F81000FFFF6700238B330534038327C90A3E9516
:10F8200083570500E38597FE0504D9BF1733FFFF13
:10F83000E70203862A8AAE89B284B68A974000001E
:10F84000E78080D819E591473E851733FFFF6700B1
:10F8500063872A894E8597C00000E780E08E2A845E
:10F86000638E0A048D476DD103570500C547E31D1C
:10F8700047FD0347F9018546AD47E317D7FC8347AA
:10F88000450081CF4146A6855D0597F00000E780E1
:10F89000C09E814755D9AD4745BF13096501230275
:10F8A000E500CA85268597100000E780606231C1B7
:10F8B000A547E38B0AF82302040079B705C18357F3
:10F8C0000500E39247F94146A685190597F0000027
:10F8D000E780A09A81472DD99947BDB74E859700FB
:10F8E0000000E78080F02A84954739DD1309550030
:10F8F0004DBF4146A6852310440123113401130551
:10F90000190097F00000E780A099228597800000F9
:10F91000E780A0EA81470DBF1723FFFFE702E378E6
:10F9200079717C003ECCB7070A003ECE7C003ED009
:10F9300083C79500B2842E8493F7F707A384F5005C
:10F940001306A1002A892C00268597000000E78075
:10F95000A0E5A16528088D0597A0FFFFE780A0F727
:10F9600090408355A1000355810085469700000013
:10F97000E78000ECAA84AA85280897C0FFFFE780EB
:10F9800040DA0356A1008355810028089700000043
:10F99000E780C0C1300801478146A2854A8597A00B
:10F9A000FFFFE780A018854748103ED4230291024C
:10F9B00002D697D0FFFFE78060BD45611723FFFFA8
:10F9C0006700E3701723FFFFE702236E79717C0065
:10F9D0003ECCB7070A003ECE7C003ED083C79500E0
:10F9E000B2842E8493F7F707A384F5001306A100D1
:10F9F0002A892C00268597000000E780E0DAA165BF
:10FA000028088D0597A0FFFFE780E0EC9040835524
:10FA1000A10003558100814697000000E78040E186
:10FA2000AA84AA85280897C0FFFFE78080CF0356E5
:10FA3000A10083558100280897000000E78000B7E7
:10FA4000300801478146A2854A8597A0FFFFE780DD
:10FA5000E00D48102302910202D402D697D0FFFF96
:10FA6000E780C0B245611723FFFF67004366172395
:10FA7000FFFFE702836397000000E78060DB172346
:10FA8000FFFF6700C3649767FF1F93876711884371
:10FA900082801723FFFFE70243618357250041114E
:10FAA000AE842A842307B10017F5FFFF130525460E
:10FAB0006C002316F10097A0FFFFE780204991C456
:10FAC000228597800000E780E0D6FD572310F400E0
:10FAD000130620028145130554009720FFFFE7809D
:10FAE000C05F41011723FFFF6700635E1723FFFF1D
:10FAF000E702035A79717C003ECCB7070A003ECE7C
:10FB00007C003ED083C79500AA89AE8493F7F7079F
:10FB10003285A384F5001306A1002C009700000095
:10FB2000E78080C803558100114497400000E780BA
:10FB3000A0A915C50355A100014497B00000E780B6
:10FB4000A06011CD03570500835781004544631819
:10FB5000F700854597000000E780E0F30144216944
:10FB600093053900280897A0FFFFE780C0D6A2853B
:10FB7000280897C0FFFFE780C0BA0356A10083554D
:10FB80008100280897000000E78040A23008014764
:10FB90008146A6854E8597A0FFFFE78020F9481093
:10FBA0004AD42302810202D697D0FFFFE780009E4D
:10FBB00045611723FFFF6700E3501723FFFFE702AC
:10FBC000234D9767FF1F938767FD2A8488432E89FB
:10FBD00015C5035745038357C4016311F702232654
:10FBE000050223180502410597D00000E780209CFC
:10FBF0006306090097800000E78060DB8144976915
:10FC0000FF1F9389291A130A800297B0FFFFE7802C
:10FC1000C0C563C4A4049767FF1F9387E7009C4394
:10FC200099C70355C40197200000E780C0BD630752
:10FC30000900228597800000E780C0A01306400ECF
:10FC4000814522859720FFFFE7802049FD57231E2D
:10FC5000F4001723FFFF6700E3463385440383A7BF
:10FC6000C90A3E95035705008357C4016317F7007F
:10FC7000CA8597000000E78000E2850479B7172362
:10FC8000FFFFE702E34083C795004111AA8993F77C
:10FC9000F707A384F5003285AE8497C0FFFFE780A5
:10FCA00000B885676378F5042A8997400000E780EB
:10FCB000A091014401CD83D704003144638827011A
:10FCC000854597000000E78080EF01444E85A286BD
:10FCD0004A86A68597D0FFFFE780A09CA1679387FF
:10FCE000170448003EC42302810002C697D0FFFFDC
:10FCF000E780C08941011723FFFF6700A33C17235A
:10FD0000FFFFE702E3389767FF1F938727E98043E8
:10FD100029C4014597C00000E780002181470148C0
:10FD2000C1641CDC232E0403232004041769FF1F75
:10FD30001309490701449309400EFD1497B0FFFFD2
:10FD4000E780A0B1634FA400814517F5FFFF1305BD
:10FD5000857F97A0FFFFE780601F1723FFFF6700E5
:10FD60006336330534038327090B3E958357C5015A
:10FD700063879700854597000000E78040E405040D
:10FD800075BF9357050113D78700A380F50093171C
:10FD90000501C183A1832380E5002381F500A381B0
:10FDA000A50082801723FFFFE70223302300050010
:10FDB00083C71500A300F50083C725002301F500C4
:10FDC00083C73500A301F50083C745002302F50072
:10FDD00083C75500A302F50083C76500930595000E
:10FDE000A30305002303F5002304050032859700D3
:10FDF0000000E78040F91723FFFF6700432D17231A
:10FE0000FFFFE702E3284111E9540DCD85CD93F9B9
:10FE1000C5FF2E842A89AA84338AA900B7EA040080
:10FE200063189A020D88854411CCB7E704009C5FE3
:10FE300082972AC622866C003305390197E00000BC
:10FE4000E7800046268541011723FFFF67008327CF
:10FE500083A78A039104829793170501C183A18325
:10FE6000A38EF4FE93570501238FF4FEA183238E06
:10FE7000A4FEA38FF4FE6DB763E6D5021723FFFF40
:10FE8000E702A322B28741113686BE8536C697E0C7
:10FE90000000E780E040B246410136851723FFFFAE
:10FEA0006700E322814636858280838705001387B9
:10FEB000F5003D05FD8793F77708834607007D151C
:10FEC0008606B58FA300F5006307B7007D1783474B
:10FED00017009D83DDB782801723FFFFE702E31C35
:10FEE000B7E7040083A7070932872A863A858297F5
:10FEF000133515001723FFFF6700631D15C18147E8
:10FF00008DC11723FFFFE702431A414697E0000027
:10FF1000E780003985473E851723FFFF6700231BD5
:10FF200081473E8582801DCD1723FFFFE702E3173F
:10FF3000414681452A849720FFFFE780001A414609
:10FF40008145130504039720FFFFE780001901474F
:10FF5000C1672322040438C87CC805451723FFFF66
:10FF60006700E3160145828081473DCDB5CD17235B
:10FF7000FFFFE7028313B2842E89130680058145B3
:10FF80002A849720FFFFE7804015CA8524C4268570
:10FF900097000000E780C0F6414681452285972002
:10FFA000FFFFE78080133044A28522859700000080
:10FFB000E780C0F293040401A28526859700000023
:10FFC000E780E0EEA6851305040297000000E780B5
:10FFD00000EE228597000000E78020F585473E85EA
:10FFE0001723FFFF6700A30E3E8582801723FFFFC4
:10FFF000E702030A4111E9540DCD85CD93F9C5FF00
:020000040001F9
:100000002E842A89AA84338AA900B7EA0400639857
:1000100044030D88814411CCB7E704009C5F8297AC
:100020002AC622866C003305390197E00000E7807C
:100030002027268541011723FFFF6700A30883A718
:100040008A039104829793170501C183A183A38E2C
:10005000F4FE93570501238FF4FEA183238EA4FEA3
:10006000A38FF4FE6DB765CD1723FFFFE7024302B0
:10007000B28411E605451723FFFF6700A3042A8415
:100080002E890145EDD93C487848B3E6E700E5D62E
:100090009386F7FFB3B7F6007D17032A4404BA9797
:1000A00034C87CC863050A06C14913050A03B3892D
:1000B00049412295637D3601B2862E86A68597003A
:1000C0000000E780A0DB7C40BE9464C065B7CE86AC
:1000D0002E86CE8597000000E78040DAC114D294C6
:1000E0004E9923220404A2879306040103C7070044
:1000F00003C607038507318FA38FE7FEE398F6FE5B
:100100003044A285228597000000E78020DD2699F3
:10011000C1493306994063EC9900A9DCA686A685FF
:100120001305040397000000E78040D579BF81479D
:10013000B306F4003307F6000347070083C5060043
:1001400085072D8F2380E600E39437FF3044A28596
:10015000228597000000E78060D8C1145DBF01458B
:1001600082800DC11723FFFFE70223F413068005E9
:1001700081459720FFFFE78040F605451723FFFFE5
:100180006700E3F401458280814749C5C1C5172353
:10019000FFFFE70283F1FC4141462E84AA84639964
:1001A000C70413860501A2878146C14503C707001E
:1001B00003C507038507298F3305D60003450500CE
:1001C0008506298FA38FE7FEE392B6FE3044A28511
:1001D000268597000000E78060D022859700000008
:1001E000E78060F885473E851723FFFF670023EE11
:1001F000138507031D8E814522959720FFFFE78019
:10020000C0ED7C40130700F813060402A297238870
:10021000E70251BF3E8582801723FFFFE702E3E834
:100220006D712E84B284AA859010280036899700BB
:100230000000E780A0D309EDD55725A050400C4021
:10024000280097000000E78040E27DD5FD142104DE
:10025000F5F42C004A8597000000E78020F38147E1
:1002600061DD3E8551611723FFFF670043E61723D9
:10027000FFFFE70283E341112EC432C62C0005467E
:1002800097000000E78080F941011723FFFF670016
:1002900003E41723FFFFE70243E101112A842EC67E
:1002A00002C802CA02CC02CE97E00000E780402BD1
:1002B000B2462A86A285080897000000E78060FB06
:1002C0001375F50F05611723FFFF670043E0172340
:1002D000FFFFE70283DD7971B2872A842146230874
:1002E000B10013051101BE853AC436C697E000007F
:1002F000E78000FBB2469305910136859700000028
:10030000E78060A82285141035460C08970000008D
:10031000E78020F62A84224701E921460C103A851D
:1003200097E00000E780C0F7228545611723FFFFB3
:100330006700E3D91723FFFFE70223D77171AE846B
:10034000AA850A85328497000000E78060BB11C946
:100350000A86A685228597000000E78020B881479D
:1003600011E1C5473E854D611723FFFF670023D686
:100370001723FFFFE70263D01D712A8AB289BE846A
:1003800035468547130511012E8CB68A3A8BC28CEF
:10039000468D2308F10097E00000E78060F0101020
:1003A0000C085285231F010097000000E780C0F869
:1003B0002A843DEDA1476313FD089307900591E062
:1003C000E5473546E2851305110113990A01230813
:1003D000F1001359090197E00000E78060EC135722
:1003E000890093978A00D98F90080C085285231FA3
:1003F000F10097000000E78020F42A8415E9A1E4C9
:100400009387FA0091831379F9003EC663130900BC
:100410004149668B8144C14B854DB247639F970C20
:100420006A868C0033855C0197E00000E78040E736
:10043000228525611723FFFF6700E3C79307900418
:10044000C9F0A547BDBF834701050947C14B230834
:10045000F10083471105A58FA308F10093872400BD
:10046000814463E1FB04014714083386E6008C08ED
:10047000B386E400BA95DA9683C6060083C5050004
:100480000507AD8E2300D600E390E7FE4147639C4D
:10049000E70490080C08528597000000E780C0E947
:1004A00025D181A0B3069B00BA871008B305F600DA
:1004B00090083E9603C5060003460600850785069C
:1004C000298E2380C500E39277FF998F90080C084E
:1004D0005285BE9497000000E78000E689470147F7
:1004E00049D12A84B1B790083E9603460600140805
:1004F000BE962380C600850759BFB247850463872F
:10050000971481471808B306F70098083E9733867A
:10051000F90003470700034606008507318F238053
:10052000E600E39177FF90080C08528597000000E1
:10053000E78080E05DF53546E2851305110123086B
:10054000B10197E00000E780A0D513970401418333
:10055000939784002183D98F10180C085285231F8C
:10056000F10097000000E78020DD25FD814710188D
:100570003387F9003E960347070003460600B3069B
:10058000FB008507318F2380E600E39277FF65A8A3
:100590001808B306F70098083E973386F90003471A
:1005A0000700034606008507318F2380E600E3E15C
:1005B00027FFCA87639E770990080C085285970029
:1005C0000000E78060D711FD81479800B306F7006F
:1005D000900818103E973E96034707000346060012
:1005E0008507318F2380E600E39177FF3546E2856A
:1005F000130511012308B10197E00000E78040CA0C
:10060000139704014183939784002183D98F101895
:100610000C085285231FF10097000000E780C0D12D
:10062000E31105EC814710183387F9003E96034724
:10063000070003460600B306FB008507318F2380C1
:10064000E600E3E227FFC109410BC1BB814785B743
:100650009408BE9683C6060018083E972300D7006C
:10066000850789BF638006321723FFFFE702E3A0F7
:1006700059712A84BE89B28B85473546130511020C
:100680002E8B468C4289BA8A368A2300F10297E083
:100690000000E780E0C010180C102285231701022B
:1006A00097000000E78040C963180512A147631F47
:1006B000FC069307900563930900E5473546DA8504
:1006C0001305110293140A012300F102C18097E07F
:1006D0000000E780E0BC93178A0013D78400D98F0D
:1006E00090080C1022852317F10297000000E78084
:1006F000A0C47DE1639209049307FA00BD88918349
:1007000091E0C144C207C183DE8C814A3EC6414D9F
:10071000B24763E2FA0E6286B3854B01881097E018
:100720000000E78080B54DC93D557DA0930790043A
:10073000E39609F8A54759B7834701050947C14C16
:100740002300F10283471105B3C7F900A300F102AA
:1007500093872900814963E1FC0481461810330620
:10076000D7008C083387D900B69556970347070002
:1007700083C5050085062D8F2300E600E390D7FE94
:1007800041476390E70690080C102285970000000F
:10079000E78080BA35D189A0B3863A01BA871010B4
:1007A000B305F60090083E9603C506000346060012
:1007B00085078506298E2380C500E39297FF33873E
:1007C000EC4090080C102285BA9997000000E78051
:1007D000A0B68947014741D165611723FFFF670034
:1007E000838D90083E96034606001410BE96238023
:1007F000C600850779B7B247850A93990A01939D88
:100800008A0093D909016391570F85473546DA85E8
:10081000130511022300F10293D9890097E000002B
:10082000E78000A8B3ED3D0190000C10228523174E
:10083000B10397000000E78020B059FD8147A689E9
:1008400063EA970626860C084A8597E00000E78051
:1008500020A581471810B306F700100898083E97A6
:100860003E9603470700034606008507318F238025
:10087000E600E3E197FE639FA90590080C1022852E
:1008800097000000E78040AB21F981479810B3063C
:10089000F700900818183E973E9603470700034656
:1008A00006008507318F2380E600E391A7FF410909
:1008B000C10CB9BD18089000B306F7003E96338707
:1008C000FC0003470700034606008507318F23809D
:1008D000E600B5B798084E97034707001C10CE975F
:1008E0002380E700850941BF85473546DA85130532
:1008F00011022300F10293D9890097E00000E780FC
:10090000209AB3ED3D0190000C1022852317B1030E
:1009100097000000E78040A2E31005EC814718082B
:100920009000B306F7003E963387FC0003470700AC
:10093000034606008507318F2380E600E391A7FF79
:1009400041460C084A8597E00000E78060958147A2
:100950001810B306F700100898083E973E96034714
:100960000700034606008507318F2380E600E391E8
:10097000A7FF90080C10228597000000E780C09B1D
:100980001DD599BD7D5582801713FFFFE702E371E6
:1009900001112A842E8593055100328902C002C2BA
:1009A00002C402C69304740097F0FFFFE780A03DE5
:1009B0001D46A6851305910097E00000E780408E54
:1009C00010088A854A8597000000E780E09619EDB7
:1009D00093071400180883C607000346070085071D
:1009E0000507B18EA38FD7FEE397F4FE05611713B9
:1009F000FFFF6700C36D1713FFFFE70263692E84D3
:100A00008C414111AA89838715003289914463D3AF
:100A10000700A1449757FF1F9387876F9C43A1C787
:100A2000C1CA8D472310F10083C725004A852301E1
:100A3000F10083C73500A301F10083C745002302FD
:100A4000F10083C75500A302F10083C76500930539
:100A50009100A30301002303F1002304010097F098
:100A6000FFFFE78040320C404A860A8597F0FFFF7F
:100A7000E78080330328040083564400A6881D08BD
:100A800081470147E51642868A854E85970000001A
:100A9000E780408E2A8919E5A685228597B0FFFF59
:100AA000E780E0C14A8541011713FFFF67008361BA
:100AB0004A860A8597F0FFFFE780002F6DB717136E
:100AC000FFFFE702E35C2E848C414111AA898387F2
:100AD00015003289914463D30700A1449757FF1F43
:100AE000938707639C43A1C7C1C68D472310F100BC
:100AF00083C725004A852301F10083C73500A30180
:100B0000F10083C745002302F10083C75500A3020B
:100B1000F10083C7650093059100A303010023033F
:100B2000F1002304010097F0FFFFE780C0250C408F
:100B30004A860A8597F0FFFFE78000278356440026
:100B4000032804008A85858EC2061D08C1822312EF
:100B5000D400A68881470147E51642864E85970056
:100B60000000E78060B041011713FFFF6700835565
:100B70004A860A8597F0FFFFE78000234DBF1713D1
:100B8000FFFFE7028352B335B000011185052A89C2
:100B90001315F601336515012308B1009305110102
:100BA00036843AC632C03EC442C297F0FFFFE780A7
:100BB000801DA2471248425593D68700230BF100AF
:100BC0009305910193578800A30AD100A30BF1006C
:100BD000230C010197F0FFFFE780E01A324702463D
:100BE00003280400B337E000835644009207914481
:100BF00011C2A1444A85A68842860C0897F0FFFFDF
:100C0000E78040772A8919E5A685228597B0FFFFFE
:100C1000E780E0AA4A8505611713FFFF6700234BB1
:100C20001713FFFFE702C34601113EC68647B335DF
:100C3000B0008505AA891315F6015D8D2308B10062
:100C40009305110136843A89B28442C446C297F0B2
:100C5000FFFFE780401322489248164593578800CB
:100C6000A30AF1009305910193D78800230B01019A
:100C7000A30BF100230C110197F0FFFFE780A010F8
:100C80003247104083564400B337E00092070328F0
:100C90000900914891C0A1480C084E8597000000BA
:100CA000E780809CAA8401E9835544004A8597B077
:100CB000FFFFE780C0A0268505611713FFFF6700CF
:100CC0006340AA959307F00F17170100130747A376
:100CD0006317B50013C5F7FF1375F50F828005057F
:100CE0008346F5FFB58FBA9783C70700D5B703577B
:100CF000450014419307F00F17160100130646A094
:100D0000369742074183139506014181631BE50035
:100D1000AD8FB29703C50700130515F31335150002
:100D20008280850603C5F6FFA98FB29783C70700A7
:100D3000D9BF1713FFFFE7024337B28736842E86E9
:100D4000BA86AA853E85BA8497F0FFFFE780605295
:100D5000634F0500228597E00000E78060802A86C7
:100D6000A686A285268597F0FFFFE780805017139F
:100D7000FFFF6700C3351713FFFFE70263315D71A3
:100D80002A8BAE8A17150100130505952C00B28435
:100D9000368ABA893E8997F0FFFFE780C04F2A84E0
:100DA0005DE134104146DA85280097F0FFFFE780C7
:100DB000404C2A8449E98547A303F100A6C2930762
:100DC00071002408BEC4A68685470D462C1828103D
:100DD00002DC02DED6C0BEC697F0FFFFE78000440B
:100DE0002A8435E183477102A6860D4693F7F707FB
:100DF0002300FA00C1473EDE2C188947281026DC64
:100E0000A303F10097F0FFFFE78040412A8405ED3E
:100E10004146A6854E8597D00000E78060488D4703
:100E2000A6860D462C182810A303F10097F0FFFFAB
:100E3000E780C03E2A8401E94146A6854A8597D0CD
:100E40000000E780E045228561611713FFFF67001E
:100E500063271713FFFFE702432597F700009387E7
:100E600027EF984383C7470079712A89AE84171505
:100E700001001305E5860C083AC42306F10097F03B
:100E8000FFFFE78040412A8405ED14104146CA85E2
:100E9000080897F0FFFFE780C03D2A8415E1140899
:100EA00015462C00081097F0FFFFE780803C2A844D
:100EB00001E921462C08268597D00000E780403EB6
:100EC000228545611713FFFF670063201713FFFF9B
:100ED000E702A31D97F70000938787E79C47797186
:100EE000AA842E8417150100130505800C083EC640
:100EF00097F0FFFFE780203A0DE914104146A685E0
:100F0000080897F0FFFFE780C03605E11408114696
:100F10006C00081097F0FFFFE780A03519E58347C4
:100F2000F10193F7F7032300F40045611713FFFF66
:100F30006700E3191713FFFFE70223173688A1485C
:100F400081470147E54697F0FFFFE780A04217136E
:100F5000FFFF6700C3171713FFFFE702031536886B
:100F6000A14881470147E54697F0FFFFE780C06F42
:100F70001713FFFF6700A3151713FFFFE702E31224
:100F800001112A842E850C0832C697F0FFFFE780F6
:100F9000803009ED3247970601009386667310088A
:100FA000C145228597000000E780E0D8056117134E
:100FB000FFFF6700C3111713FFFFE702030F411183
:100FC000C1472EC032C48A8509463EC23EC697F04C
:100FD000FFFFE780A02441011713FFFF6700230FE5
:100FE0001713FFFFE702630C4111AE8613061009C9
:100FF000AA850A8502C002C202C402C697F0FFFF9A
:10100000E780202741011713FFFF6700430C1713E8
:10101000FFFFE70283093287970601009386466D3A
:101020002E869305000297000000E780C0D01713BA
:10103000FFFF6700C3091713FFFFE702030779717A
:10104000C1472ACC2ED032D42C080D4628003ECEE3
:101050003ED23ED602C402C602C802CA97F0FFFFC3
:10106000E780C01B45611713FFFF67004306171396
:10107000FFFFE70283030111AA842E8417050100F4
:10108000130585678A8597F0FFFFE780C02015E587
:1010900014084146A6850A8597F0FFFFE780601D8A
:1010A00009ED8347E1010347F101A207D98FCA0780
:1010B000C9836177D98F2310F40005611713FFFFEF
:1010C0006700E30015CD1713FFFFE70203FE9757F4
:1010D000FF1F938767B190439755FF1F938505B115
:1010E0001755FF1F130545AC97D00000E78000C5DA
:1010F0001755FF1F130545AB1713FFFF670023FDAF
:101100001755FF1F130545AA82808DCD1713FFFFCA
:10111000E702A3F99757FF1F938707AD9443011187
:101120002E840A869755FF1F938545AC97D0000003
:10113000E78040C60A850294014505611713FFFF49
:101140006700E3F87D5582801713FFFFE702E3F5A0
:1011500097D00000E78080D19757FF1F23A6A7A84C
:1011600017F5FFFF1305E5C997B00000E780C074CD
:101170001713FFFF6700A3F51757FF1F130707A9F2
:101180009317150008433E95FD572310F500828004
:101190001713FFFFE70263F12A84084009E51713DC
:1011A000FFFF6700C3F21C4158401CC06313E500F9
:1011B0005CC08347550023200500F99BA302F5007E
:1011C00097A0FFFFE780207CC9BF1713FFFFE7024E
:1011D00023EC9757FF1F938767A598432A8411CB69
:1011E0008347350093F7070289C7035505008945F2
:1011F00002971305440197B00000E780403B8355F8
:1012000004000355E40097300000E780A00C485824
:1012100019C597A0FFFFE7800077232A0402130572
:10122000840397000000E780E0F68144B14997907D
:10123000FFFFE780C06D63CBA40283473400232007
:10124000040493F727FCA301F40000489790FFFFE4
:10125000E780E06C13161500814522859710FFFF8B
:10126000E780A0E71713FFFF6700C3E5B3873403E8
:101270000329040385043E994A8597000000E7800E
:1012800060F12304090065B78347350093F707022F
:1012900099E3014582808357E500E39CB7FEC1676F
:1012A000FD176316F60005458280054599A81713BA
:1012B000FFFFE70283DF93170601C187B2842A8408
:1012C00001496359F002835705009DCB01456367CF
:1012D000F600034584003E953325A6001375F50FEF
:1012E0000DA01C4813171900BA9783D70700E38E87
:1012F00097FA05099790FFFFE7806062E343A9FE34
:1013000001451713FFFF670083DC1713FFFFE70298
:1013100023D8AE89AA849790FFFFE78000562A84DD
:1013200097D0FFFFE780A02EAA860147130684010D
:1013300097050000938585E41755FF1F1305458D1C
:101340009790FFFFE780801C2A8925C98C441304ED
:10135000C50022859E0593F5050897A0FFFFE7804D
:10136000403CCC4083877400E18163DD070493E552
:101370000508228597A0FFFFE780A03A0D469385D8
:101380004400228597A0FFFFE780C03683D5040084
:10139000228597A0FFFFE780E03D83D524002285CA
:1013A00097A0FFFFE780003D03D6490083A5090011
:1013B000228597A0FFFFE780E0334A851713FFFFE0
:1013C000670043D093F5F5076DB71713FFFFE702EA
:1013D000C3CD01112A84328532C697A0FFFFE78072
:1013E000E0279780FFFFE78060348357040017579A
:1013F000FF1F1307279B3246231BF100930700F8BA
:10140000A30DF1001C471843231AA1008983858B83
:10141000B307F740B28548083ECE231C0100230DD8
:10142000010097000000E78080EE05611713FFFFC1
:101430006700E3C91713FFFFE70283C500410145B9
:101440003DC49304C40026853289AE8997A0FFFF6E
:10145000E780C02495452A8A2685035B040197A06E
:10146000FFFFE7802021268597A0FFFFE780603EF1
:101470008D45AA8A268597A0FFFFE780A01F2685B5
:1014800097A0FFFFE780E03C5C48420A135A0A013C
:10149000D2975CC423186401814763983A014605DA
:1014A0004D81330625419337160013F5F70F1713B7
:1014B000FFFF670023C11713FFFFE70283BC8969A1
:1014C0002A8BAE8B328AB68A81440144314CFD1995
:1014D0009790FFFFE780A04363CDA4009790FFFFA4
:1014E000E780E045018D33B5AA001713FFFF6700C1
:1014F000C3BC3389840383270B003E9963170A001A
:101500008347890085043E94E1B703560A00DE85CF
:101510004A8533F6C90097000000E780E0F16DD1FD
:101520000545E1B71713FFFFE70223B801112A842D
:101530007C000355E5003ECAB70707003ECC7C009F
:101540003ECE97200000E78020082A89854548087C
:1015500097A0FFFFE78020399945480897A0FFFF33
:10156000E780E015AA844A8597200000E780A0085C
:101570002380A4009757FF1F9387C7829C4341662F
:10158000130606F09396870113D78701558F93D6DC
:101590008700F18E558FA207B706FF00F58FD98F10
:1015A00011462C00138514003EC497D00000E7803C
:1015B00020CF5008A38204008945228597000000AF
:1015C000E780E0E019C9AA851305840397A0FFFF0F
:1015D000E780E0313C4085073CC005611713FFFF01
:1015E0006700E3AE1713FFFFE70223AC9790FFFFFE
:1015F000E780E0342A8405049790FFFFE7802033DA
:101600003305A402F14791453305F5029720000008
:10161000E78020BA11E565551713FFFF670023AB7C
:101620009747FF1F23ACA75E9790FFFFE78020310D
:101630002A8405049790FFFFE780602F3305A402FA
:101640008945060597200000E780A0B669D5974731
:10165000FF1F23ADA75A9790FFFFE780402E2A84F3
:1016600005049790FFFFE780802C3304A40297477E
:10167000FF1F239F87589790FFFFE780402C2A8405
:101680009790FFFFE780A02A930714003385A702F5
:101690009747FF1F239FA75697070100938787C986
:1016A0001747FF1F232AF7560145BDB71713FFFF42
:1016B000E702039EAA842E8901449749FF1F93895C
:1016C000696E130A80069790FFFFE7804026634704
:1016D000A40001451713FFFF6700C39E33054403B1
:1016E00083A709024A86A6853E9597000000E780F9
:1016F000E0B919E10504C1BF0545E9BF1713FFFFB4
:10170000E7022398AA8A2E8BB28B368C3A8A8144C0
:1017100001448149974CFF1F938CCC68130D8006C0
:101720009790FFFFE780A02063C9A40011E08549DE
:101730004E851713FFFF670043983389A40383A7DF
:101740000C025E86D6853E994A8597000000E780A8
:10175000E0B31DC19790FFFFE780601E0544636DF5
:101760004501D2866286DA851305090397000000D9
:10177000E780A0D411C1854985045DB71713FFFF29
:10178000E7020391C16441112A8901449749FF1F6F
:1017900093894961130A8006FD1436C632C42EC2ED
:1017A0009790FFFFE780A01892452246B246634813
:1017B000A400014541011713FFFF6700A390330503
:1017C000440383A709023E9509C683473500C18BB0
:1017D0009DC791C68347350093F707028DC3630603
:1017E00099008357E500639C27010357050001CB4F
:1017F00063E7E50083478500BA97E3CDF5FA050472
:1018000069BF1713FFFFE702A388C1642A89014457
:101810009749FF1F93890959130A8006FD14979071
:10182000FFFFE780C0106346A4001713FFFF6700A7
:1018300063893305440383A709023E958357E50076
:10184000638A97006304990063962701970000005C
:10185000E780E0970504E1B71713FFFFE702E38194
:1018600089692A8AAE8A328BB68B8144174CFF1F56
:10187000130C4C53930C8006314DFD199790FFFFCC
:10188000E780E00A63C6A4001713FFFF6700A38286
:101890003389940383270C028355CA015A863E99E3
:1018A0004A8597000000E780609E31C1814D15A0F8
:1018B0003384AD038327090303D60B00D68533F6A3
:1018C000C9003E94228597000000E780E0B609E950
:1018D000850D9790FFFFE7808003E3CBADFC01A867
:1018E000228597000000E780E08A23040400850435
:1018F00071B71703FFFFE702C3784169AA8A014A5B
:10190000174BFF1F130B0B4A7D19C14B054C9790CA
:10191000FFFFE780C0016346AA001703FFFF6700CF
:10192000C37993098006B3073A0383290B02BE9952
:1019300083D7E900638E270163842A01639A5701E4
:1019400003A4890301E84E8597000000E780C0BD2D
:10195000050A75BF83570401639977099304C4008E
:10196000268597A0FFFFE78060D385452A8D2685D1
:10197000835C040197A0FFFFE780C0CF268597A076
:10198000FFFFE780A0E762056185635905048D4587
:10199000268597A0FFFFE780E0CD8945268597A0A3
:1019A000FFFFE78020CD8945268597A0FFFFE780D0
:1019B00060CC8545268597A0FFFFE780E0CC834774
:1019C0000500094793F7F707639AE70099452685CD
:1019D00097A0FFFFE78040CBA30285014848337DF5
:1019E0002D01231894016A9548C40040A1BF170334
:1019F000FFFFE702836B37E404008327041D82970F
:101A00009747FF1F83C707271725FF1F130545AEFD
:101A1000A300F5008327441C82978327841C8146FA
:101A20001306F00F8145014582971703FFFF6700FA
:101A3000036A1747FF1F1307E71318439745FF1F54
:101A400083C545239747FF1F938747218346870315
:101A5000034697036397D5009747FF1F238CC72042
:101A6000828083C587010347A7036317B6009747A2
:101A7000FF1F2381E720828003C687016317C70009
:101A80009747FF1F2388D71E828083C687011307CD
:101A900050026319D700930760021747FF1F230BFB
:101AA000F71C828083C68701130660026315D60087
:101AB00093077002DDB783C7870155BF9747FF1FA4
:101AC0009387C719D44B0947638DE6081703FFFFB7
:101AD000E702A35D1749FF1F130989153E84834759
:101AE0000900918B9DCFB7E4040083A7041D829762
:101AF00083A7441C1745FF1F13050514829783A76E
:101B0000841C81461746FF1F034606158145014583
:101B1000829721C583470900ED9B1747FF1F2309C3
:101B2000F7108347040093F7F70F85CB91471747CA
:101B3000FF1F232FF71297000000E78080EB97002C
:101B40000000E78040EFB7E70400BC4F41469145F5
:101B50001745FF1F0345051182971703FFFF670015
:101B6000035782801703FFFFE70223548D4741117B
:101B70006306F504C5476308F50285476310F5025F
:101B80009747FF1F238AA70EB7E70400BC4B9305B6
:101B900000101745FF1F0345E50C8297410117030D
:101BA000FFFF6700C35285471747FF1F2306F70C47
:101BB000B7E70400BC4B93050020E1BF9747FF1F28
:101BC0009387C709D44B1147638DE600B7E704003C
:101BD00083A7071D8297B7E70400BC4B9305000459
:101BE0004DBF05491747FF1F2324270983C7070057
:101BF00032C62E8493F7F70FD5D3B7E4040083A73A
:101C0000041D7D141374F40F8297E37689FCB245AA
:101C1000994703C61500E3F0C7FCFC4409061745C5
:101C2000FF1F1305A5058297BC48930500081745BB
:101C3000FF1F03452503829779BF1703FFFFE702C4
:101C4000C3461747FF1F130767014047184B1C4047
:101C50009746FF1F23AAF6006316E4001747FF1FED
:101C60002326F700130584FE9790FFFFE78000AA64
:101C7000035564FF9780FFFFE780807297A0FFFF06
:101C8000E78060D01703FFFF670063441703FFFF7F
:101C9000E702A3419747FF1F938747FCD84BDC47D8
:101CA00089C797000000E78080F985471747FF1F25
:101CB0002320F7FC9747FF1F9387C7EB9C439305AF
:101CC00000021745FF1F0345E5F983C78703174740
:101CD000FF1F2301F7FAB7E70400BC4B82971703F5
:101CE000FFFF6700C33E9747FF1F23ABA7F6828025
:101CF0001703FFFFE702C33937E404007C4CA1451A
:101D00001745FF1F034505F682977C48A1451745F7
:101D1000FF1F034525F59744FF1F938424F4829702
:101D2000DC4489EB97000000E78080D91703FFFFB0
:101D30006700433903D567FF9780FFFFE780406660
:101D4000AA896DD1D84891476310F7027C4C914520
:101D50001745FF1F034505F182977C4891451745BC
:101D6000FF1F034525F0829703A9490103D4090108
:101D70008947B7E904001747FF1F232BF7EE83A716
:101D8000091D21044204829783C784011715FF1F90
:101D90001305057661191717FF1FA30BF77483A7A7
:101DA000491C418082979747FF1F238707EC83A731
:101DB000C91C814609469375F40F4A85829711E93B
:101DC0009747FF1F83C787FB89C79710FF1FE780CF
:101DD00000DFB7E70400BC4F2146A1451745FF1FB0
:101DE000034545E8829799B71703FFFFE702E32B06
:101DF00093F7052001112E8481CF97000000E78022
:101E000020E91345042005611703FFFF6700232C19
:101E100093F70510A9CF9744FF1F938424E4DC486F
:101E200097000000E78020C11747FF1F130787D4E2
:101E3000184383C78401034787036318F700DC4412
:101E400089C797000000E78080DF85471747FF1F9D
:101E50002320F7E2B7E70400BC4B930500021745C7
:101E6000FF1F034525E082971345041069BF93F7D0
:101E70000508BDC79747FF1F83C757E0E9171946F5
:101E80009745FF1F9385A5DF1305D10093F4F70F46
:101E90001749FF1F034989DE97C00000E7804040D3
:101EA00093970401C1831747FF1F1307A7DD231D65
:101EB000F100231CF1009747FF1F938727DA3ACEE2
:101EC0003ACAD8432306010009CBDC4393158901A4
:101ED00054080D46E185680082971345040825B72C
:101EE00093F72500A5C39747FF1F938727D7D84BA4
:101EF00089476306F7029747FF1F83C767D313F726
:101F0000270011EF918B99CFB7E70400BC4F130660
:101F1000000A89451745FF1F0345C5D4829713451D
:101F20002400D5B59747FF1F9387C7C49C4383C739
:101F300087031747FF1F230FF7D297000000E780A2
:101F400060DBF1BF93F7050281CB97000000E780CB
:101F500060DA1345040245BD93F7850081CB9700F5
:101F60000000E780E0D21345840071BD93F71500AF
:101F700081CB97000000E780A0B41345140061B541
:101F800093F7450081CB97000000E78060B31345CD
:101F9000440095BD93F7050495C39747FF1F83C77A
:101FA000E7CB91CB97000000E780A0A491471747AB
:101FB000FF1F232FF7CA13450404B1B593F705019A
:101FC0000145E38207E49747FF1F938727C9D84B52
:101FD00091476310F7049747FF1F938767C59C439A
:101FE00013D727008583D98F858B91E7B7E7040046
:101FF00083A7071D8297B7E70400FC4F914517455B
:10200000FF1F034525C6829785471747FF1F2321DA
:10201000F7C613450401C5BB9747FF1F2380A7D60A
:1020200082801703FFFFE70243089747FF1F23AD96
:1020300007C29747FF1F23AB07C285471744FF1FFF
:10204000130444B31747FF1F2324F7C21C4083C760
:1020500087031747FF1F230FF7C09790FFFFE78005
:10206000409329C59717FF1F23A8A7481C401705B1
:1020700000001305A5D783C787031747FF1F230B4E
:10208000F7BE1717FF1FA305F7469747FF1FA38744
:1020900007BCB7E7040083A7070882979747FF1F8D
:1020A0002382A7BC1703FFFF67006302B7C7898EAF
:1020B000938767ED1717FF1F2320F74445BF174786
:1020C000FF1F0347A7B9795555E79747FF1F938728
:1020D000E7B803C7170005079746FF1FA380E6B8B8
:1020E00003C717008D463377D7029746FF1FA38794
:1020F000E6B683C617001747FF1F1307A7A71843A5
:1021000093F6F60FA9EE834787031747FF1F2303B4
:10211000F7B685471747FF1F2302F7B49747FF1FFE
:10212000938707B19C430145998BA9E71703FFFFEC
:10213000E702A3F737E404007C48C1451745FF1FB9
:10214000034545B282973C4885451745FF1F034527
:1021500065B1829701451703FFFF670043F783C707
:10216000170085466395F6008347970379BF834739
:10217000A70361BF82809747FF1F83C727AEA1CF08
:102180001703FFFFE70263F237E404009747FF1FDE
:10219000238607AC7C4885451745FF1F034585AC62
:1021A00082977C4C91451745FF1F0345A5AB82974D
:1021B0007C4891451745FF1F0345C5AA82973C48B7
:1021C000C1451745FF1F0345E5A982970145170340
:1021D000FFFF6700C3EF795582801703FFFFE70217
:1021E000C3EC2A84035565FF9780FFFFE780401BFF
:1021F0009747FF1F938787A6D847BE841DEF979008
:10220000FFFFE78080779C48232004009DEB9747E1
:10221000FF1F23AD87A49747FF1F23A787A4B7E716
:102220000400BC4B89451745FF1F0345A5A38297B2
:1022300001451703FFFF670083E9630A870018431E
:1022400075BF80C39747FF1F23A287A2C9BF7955D7
:10225000CDB71703FFFFE70243E59747FF1F9387BB
:1022600027B288432326050023240500510597A0A3
:102270000000E780C0331703FFFF670043E5170343
:10228000FFFFE70283E21744FF1F130464AF1C4003
:10229000411199CF9C472302B5002AC61CC1970063
:1022A0000000E78040FB1C409C4B99C3324582975D
:1022B00041011703FFFF670083E11703FFFFE702F8
:1022C000C3DE4111444D328532842EC69790FFFF04
:1022D000E780C0522AC422859790FFFFE7802054F0
:1022E00003A84400630C0800B2458357440018401B
:1022F000224683D54500AA86268502984101170308
:10230000FFFF6700C3DC1703FFFFE70203DA404D5E
:102310001DC808C097050000938565031305440197
:1023200097A00000E78040169747FF1F938747A5B7
:102330009C43014589E79747FF1F23A387A4170301
:10234000FFFF6700C3D87D55DDBF1703FFFFE7021E
:10235000C3D5011168009305F00F02C602C802CA76
:1023600002CC02CE97000000E780A0F105611703C0
:10237000FFFF6700C3D59747FF1F938767A09C4364
:10238000D847A1679D076319F7021703FFFFE7020C
:10239000C3D1011132859790FFFFE7802046230AC1
:1023A000A1008145680097000000E78080ED05618D
:1023B0001703FFFF6700A3D182809747FF1F938712
:1023C000279C9C43D847A167938777036319F7023B
:1023D0001703FFFFE70263CD011132859790FFFFDE
:1023E000E780C041230AA1008145680097000000F2
:1023F000E78020E905611703FFFF670043CD828076
:102400009747FF1F9387C7979C43D8479547631605
:10241000F7041703FFFFE70243C901113285328435
:102420009790FFFFE780803D230AA10022859790C7
:10243000FFFFE780C03E83574400231BA100814576
:102440003ECC1C4068003ECE97000000E78060E371
:1024500005611703FFFF670083C78280930785FF2D
:102460008DC38327C5FF91CFDC4B81CF1703FFFFBF
:10247000E702A3C3032585FF82971703FFFF6700C9
:1024800003C582801703FFFFE70223C22A84328537
:102490009790FFFFE7808036BD4763EBA7001844A5
:1024A0009377F5000345B70041995D8DA305A7001B
:1024B0001703FFFF6700A3C11703FFFFE702E3BE97
:1024C00001117C003ECAB70707003ECC7C003ECE1F
:1024D0005C4DA9C72A8413858700AE8497A00000AD
:1024E000E780E0FCA1652A899D0548089770FFFFF9
:1024F000E780603E9305803EB345B902480893F5F6
:10250000F50F9790FFFFE780C021014781465008F3
:10251000A68522859770FFFFE7804061056117035C
:10252000FFFF6700C3BA1703FFFFE70203B8970076
:102530000000E780A0F81703FFFF670043B9170307
:10254000FFFFE70283B601117C00AE843ECAA1659D
:10255000B70707002A843ECC48087C0093857503A2
:102560003ECE9770FFFFE78000371C44480883C5C4
:10257000B700BD899790FFFFE780A01A5008014778
:102580008146A68522859770FFFFE780205A056166
:102590001703FFFF6700A3B31703FFFFE702E3B0D2
:1025A0002A84AE8497000000E78000EEA68522858D
:1025B00097000000E780E0F81703FFFF670023B1F2
:1025C0001703FFFFE70263AE97000000E78060F7A4
:1025D0001703FFFF6700A3AF1703FFFFE702E3AC9A
:1025E0000329C5014111630809022A843285B28496
:1025F0009790FFFFE78080202AC626859790FFFFEF
:10260000E780E021832749002A8691C7DC4781C7FC
:10261000B2452285829741011703FFFF670023AB74
:102620001703FFFFE70263A8444D91CC2A8432854B
:102630009790FFFFE780A01EDC40AA8589C79C47D2
:1026400099C3228582971703FFFF670043A81703EA
:10265000FFFFE702E3A3032AC5014111630D0A0648
:102660002E89AA849545328532849770FFFFE780D2
:102670008026854522859790FFFFE7804004AA8940
:10268000CA8522859790FFFFE780A00B83274A0029
:102690008DCBDC439DC722859790FFFFE780A0008C
:1026A00083274A00104083564400DC437115A3077A
:1026B000A100B2961307F1004E86CA85268582973F
:1026C00001C52380090001A88345F1002285979068
:1026D000FFFFE780C0FE41011703FFFF6700839EF5
:1026E0001703FFFFE702639C65711C083EC2B70732
:1026F00080013EC41C0832893EC62A84AE849700FD
:102700000000E780A0ED4A859790FFFFE780201149
:102710008357A1008DC3AA85500022859700000031
:10272000E78020F3014781465000A68522859770F7
:10273000FFFFE780A03F59611703FFFF6700239960
:102740001703FFFFE702C39465711C088329C501C5
:102750003EC2B70780013EC41C082A84AE84328979
:102760003EC697000000E780E0EB638A09024A85D5
:102770009790FFFFE780A00A8357A100AA8585C331
:102780005000228597000000E780A0EC01478146B9
:102790005000A68522859770FFFFE7802039596198
:1027A0001703FFFF670003921703FFFFE702E38FA2
:1027B00065711C083EC2B70780013EC42A841C080C
:1027C00032853EC6AE849790FFFFE7804005835771
:1027D000A1008DC3AA855000228597000000E780E4
:1027E00040E7014781465000A68522859770FFFF8C
:1027F000E780C03359611703FFFF6700438D17035C
:10280000FFFFE702838A444D81EC8347450093B77D
:102810001700B307F0403E851703FFFF6700238BC7
:102820001845FD576DDB97070000938747032A84FF
:102830005CCB970500009385A5C21385840097A003
:102840000000E78060C480C003474400814761F70F
:102850001737FF1F232897527DBF1703FFFFE7029B
:1028600023838329C501411103298500814763879B
:10287000090A0324090191452A8A22859770FFFFDE
:10288000E7806005854522859790FFFFE78020E37C
:102890008945AA8A22859790FFFFE78040E2AA84B3
:1028A0009770FFFFE780400A83A749002A8B8DCBF2
:1028B0009C439DC722859790FFFFE780C0DE83A7DA
:1028C0004900A306A1001040835644009C4313070F
:1028D000D100B296D6851306E1005285829709CDC4
:1028E00083570B002380F400A183A380F40023808E
:1028F0000A00A306010039A88357E100228523803E
:10290000F4008345D100A183A380F4009790FFFFDA
:10291000E780E0DA8347D100B337F0000347B9001E
:10292000920701453D9BD98FA305F900410117F39B
:10293000FEFF6700237917F3FEFFE70203774111DB
:102940000DED9737FF1F9387E743804315C8044079
:10295000130984009DC95C4099C79C4B89C7268593
:102960002EC68297B2459307803EB385F5024A850D
:1029700097A00000E78060C121A0404DAA8469F8BB
:10298000410117F3FEFF670083744A8597A000009A
:10299000E780E0C15C40EDD7DC4BFDD32685829714
:1029A000C5B717F3FEFFE70243702A84328597907C
:1029B000FFFFE780A0E4AA85228597000000E7805A
:1029C000C0F717F3FEFF6700837017F3FEFFE702FF
:1029D000C36D2A84AE8497000000E780C0FCA68502
:1029E000228597000000E78060AD17F3FEFF6700C7
:1029F000036E08413355B5000589828017F3FEFF49
:102A0000E702A36A1734FF1F1304C4391C5C0111C9
:102A1000231701008D83858BA303F1008327040B0B
:102A2000231801002319010003D7C7013ECA3C0047
:102A30002314E1007D572315E1000357C4023ECC67
:102A400002CE2316E1009770FFFFE78020CE835768
:102A5000E101231EA10093F707E093E71710231F5E
:102A6000F1009737FF1F83C7873695C30547014598
:102A7000638AE7008347840393E727001737FF1F24
:102A8000230EF734056117F3FEFF670043648147A7
:102A900017F70000130707E6854613067100854502
:102AA000480897900000E780408F69FD83478403C2
:102AB000F59B1737FF1F2303F73285471737FF1F93
:102AC0002307F730C1B717F3FEFFE702035B973D1B
:102AD000FF1F938D2D2D03A6CD0639712A898147BD
:102AE0008144930600023357F600058B01C7850425
:102AF00093F4F40F8507E398D7FE83A70D0B2317F4
:102B000001022318010203D7C7013EDA3C10231447
:102B1000E1027D572315E10203D7CD023EDC2319E4
:102B200001022316E10202DE9770FFFFE78000C07A
:102B30008357E103231EA102014593F707E093E7C2
:102B40001710231FF1029737FF1F83C74728B9EFDC
:102B50009737FF1F83C797283EC69739FF1F938972
:102B600069240144014D9D4A054B954B173CFF1FBD
:102B7000130C8C2A973CFF1F938C8C2903DAC90510
:102B8000630B0A00EA856318590366859700000005
:102B9000E78060E61DC5050DA1478909E310FDFE2C
:102BA0002DE49737FF1F23A707260145216117F35F
:102BB000FEFF67004350628597000000E780A0E3B6
:102BC00079D93247B3878400E3FCE7FC9C00130605
:102BD000140006043E9413178A0093578A00D98F75
:102BE000C207C183A30EF4FCA183230FF4FC03A747
:102BF0000D07B317AB01D98F1737FF1F232CF72011
